:020000040800F2
:10800000A8C20020A1810008A9810008DD9F000806
:10801000AD810008AF810008B181000800000000B8
:10802000000000000000000000000000B381000814
:10803000B581000800000000B7810008B981000880
:10804000BB810008BB810008BB810008BB81000820
:10805000BB810008BB810008BB810008BB81000810
:10806000BB810008BB810008BB810008BB81000800
:10807000BB810008BB810008979200089B92000812
:10808000BB8100089F920008BB810008BB810008EB
:10809000BB810008BB810008BB810008BB810008D0
:1080A000BB810008BB810008BB810008BB810008C0
:1080B0003D9D0108BB810008BB810008BB81000811
:1080C000BB810008BB810008BB810008BB810008A0
:1080D000BB8100081DA6010821A6010825A60108EC
:1080E00053960008BB810008BB810008BB810008D3
:1080F000BB810008BB810008BB810008A392000877
:10810000BB810008BB810008BB810008BB8100085F
:1081100015A6010819A60108BB810008BB8100084B
:10812000BB810008BB810008BB810008BB8100083F
:10813000BB810008BB810008BB810008BB8100082F
:10814000BB810008BB810008BB810008BB8100081F
:10815000BB810008A7920008AB92000829A601087D
:10816000BB810008BB810008BB810008BB810008FF
:10817000BB810008BB810008BB810008BB810008EF
:10818000BB810008BB810008DFF810D000F0BEFB07
:1081900000480047EDC20108AFF30080A8C20020EC
:1081A0000648804706480047FEE7FEE7FEE7FEE791
:1081B000FEE7FEE7FEE7FEE7FEE7FEE7E19C0108DB
:1081C000898100082DE9F0410024061B254671F144
:1081D000000605DA01240027D0EB070067EB010158
:1081E000161E73F1000605DA0027D2EB07020125FF
:1081F00067EB030300F077FA86460E4617469C4667
:10820000AC4204D00025D0EB050E65EB010624B18D
:108210000020D2EB000760EB030C704631463A4673
:108220006346BDE8F081202A06DBCB17203A41FAED
:1082300002F043EAE07306E041FA02F3D040C2F1F3
:108240002002914008431946704740EA01039B070A
:1082500003D009E008C9121F08C0042AFAD203E0BB
:1082600011F8013B00F8013B521EF9D27047421E43
:1082700012F8013F002BFBD111F8013B02F8013B42
:10828000002BF9D17047421C10F8011B0029FBD1CB
:10829000801A704730B505460020034600E05B1C9D
:1082A000934205D2EC5CC85C201A01D1002CF6D1B7
:1082B00030BD2DE9FE4F804681EA0300C00F0C4619
:1082C000009021F0004123F00045B8EB0200A941E5
:1082D00005D24046214690461C460B46024623F0F6
:1082E0000040104347D0270DC7F30A00C3F30A51DB
:1082F0000290401A019040286BDAC3F3130040F457
:10830000801B0098924620B10023D2EB030A63EB56
:108310000B0B01985946C0F14002504600F014FA88
:1083200006460D4650465946019AFFF77CFF10EB72
:1083300008006141002487EA115284EAE7731A4376
:1083400040D0009A62B3019A012A4FEA075215DC25
:10835000001B61EB02014FF0004202EA0752CDE937
:108360000042001C41F5801132462B4600F051FAC4
:1083700003B0BDE8F08F40462146F9E7001B61EBF2
:108380000201001C41F5801300185B412018A2F582
:10839000001747EB030140EAD570B6196D4111E0B3
:1083A0006D084FEA360645EAC0754FEA0752001BD2
:1083B00061EB0201001C41F5801149084FEA3000D1
:1083C0000019514132462B4603B0BDE8F04F00F092
:1083D00011BA0098012240000023D0EB020263EBA7
:1083E000E073009821464FEAE074B8EB000061EBBF
:1083F0000401E9E783F000435BE781F0004158E7BF
:108400002DE9FE4F81EA030404F0004421F000410D
:1084100000944FF0000B23F0004350EA01045ED0BB
:1084200052EA03045BD0C3F30A54C1F30A552C4447
:10843000A4F2F3340194A0FB0254C1F3130141F4FC
:108440008011C3F3130343F4801301FB024400FBC8
:10845000034E840A970A44EA815447EA8357A4FBEF
:10846000076802958D0A05FB07854FEA932C04FBEC
:108470000C542705029D4FEA065847EA1637B5EB1C
:1084800008056EEB070C870E920E47EA811742EA49
:108490008312A7FB0201B6EB0B0164EB00042B0D6A
:1084A00043EA0C335E1844EB1C50DA465146E7FBB6
:1084B0000201C5F313044FEA0B3343EA14534FEAA6
:1084C0000432019C43EA0603A4F10C040294009CCC
:1084D000CDE900B400F09DF903B0BDE8F08F0020B5
:1084E0000146F9E72DE9F04D81EA030404F0004B61
:1084F00021F0004514464FF0000A23F0004150EAF5
:10850000050220D054EA01021DD0C5F30A570246E5
:10851000C5F31303C1F31300C1F30A5640F48015E9
:1085200043F48013A7EB0608101BD64608F2FD386B
:1085300073EB050002D308F1010801E092185B41DA
:10854000B8F1000F03DA00200146BDE8F08D0020ED
:108550004FF48011064684460EE0171B73EB0507A7
:1085600005D3121B63EB050306434CEA010C4908D3
:108570004FEA300092185B4150EA0107EDD152EA10
:10858000030012D082EA040083EA0501084305D003
:10859000101BAB4106D20122002306E000224FF05F
:1085A000004302E06FF0010253101AEB06004CEB9F
:1085B000085110EB0A0041EB0B01BDE8F04D00F053
:1085C00019B90EB5C10F80EAE0700844CA0700214E
:1085D00040F233438DE80E000A460B4600F019F9CD
:1085E00003B000BD0EB540F2334102910021CDE948
:1085F00000110A460B4600F00CF903B000BD3EB571
:10860000CA17CB0F002450405140C0186141DA070F
:1086100040F233430094CDE901232246234600F083
:10862000F8F803B030BD70B5C1F30A5201F000454F
:108630000024C1F3130140F2FF3341F480119A4248
:1086400001DA002070BD40F233439A42A2F2334275
:1086500003DC524200F087F800E090402C43F1D058
:10866000404270BD70B5C1F30A5201F000450024CC
:10867000C1F3130140F2FF3341F480119A4202DA50
:108680000020014670BD40F233439A42A2F23342C9
:1086900003DC524200F067F801E000F055F82C438B
:1086A000F0D00023D0EB030063EB010170BD01F0BB
:1086B000004330B421F0004150EA010206D00A0D17
:1086C000A2F56072C1F31301002A02DC30BC002065
:1086D0007047440F44EAC104C100E01830BC00EB0D
:1086E000C25000F050B82DE9F05F054600209246D8
:1086F0009B4688460646814640241BE02846414664
:108700004746224600F02FF853465A46C01A914178
:1087100010D311461846224600F016F82D1A67EBC2
:1087200001084F4622460120002100F00DF817EB0A
:1087300000094E41201EA4F10104DFDC4846314609
:108740002A464346BDE8F09F202A04DB203A00FA7F
:1087500002F1002070479140C2F1200320FA03F398
:10876000194390407047202A04DB203A21FA02F096
:108770000021704721FA02F3D040C2F1200291405B
:108780000843194670470029A8BF7047401C49009C
:1087900008BF20F00100704710B4B0FA80FC00FA66
:1087A0000CF050EA010404BF10BC704749B1CCF191
:1087B000200421FA04F411FA0CF118BF012121431D
:1087C0000843A3EB0C01CB1D4FEA00614FEA1020D8
:1087D00042BF002010BC704700EBC350104400297A
:1087E000A4BF10BC7047401C490008BF20F0010026
:1087F00010BC704710B5141E73F1000408DA401C59
:1088000041F1000192185B411A4301D120F00100AF
:1088100010BD2DE9F04D92469B4611B1B1FA81F29F
:1088200002E0B0FA80F220329046FFF78DFF044656
:108830000F4640EA0A0041EA0B0153465A460843F4
:1088400013D0114653EA010019D0C8F14002504636
:10885000FFF789FF05460E46504659464246FFF748
:1088600073FF084305D0012004E020463946BDE8E7
:10887000F08D0020054346EAE0762C4337430A9802
:108880006305E40AA0EB08000022FD0A44EA47540D
:108890000A3002D500200146E9E7010510196941B7
:1088A000DDE9084500196941BDE8F04DA2E770B562
:1088B00021F0004303430CD0C1F30A550024D5EB4B
:1088C000040564EB0403D617AD1AB34102DB0020A4
:1088D000014670BD201841EB025170BD30B5041E39
:1088E00071F1000404DB4FF00044404264EB0101ED
:1088F000141E73F1000405DB1C464FF00043524286
:1089000063EB0403994208BF904230BD064C074D0B
:1089100006E0E06840F0010394E80700984710344F
:10892000AC42F6D3FFF734FCD8F10108F8F10108A6
:108930002DE9F04D00231A461B1A8A4103DB002063
:108940000146BDE8F08DC1F30A52C1F3130141F4B1
:1089500080154FF0000BD10702D100186D41521E57
:108960000027044640F2FF11384601EB620A3E46FA
:108970008046024600204FF48011FFF7F4FEC21932
:108980007141BB1846EB0100B4EB030C75EB000C16
:1089900004D3E41A65EB000517460E46241908F1C6
:1089A00001006D4180463428E3DDF91946EB0600ED
:1089B000091BA84103D24FF0FF32134601E0002209
:1089C00013461BEB070046EB0A51BDE8F04DFFF7DD
:1089D00011BF000030B5041E71F1000404DB4FF03C
:1089E0000044404264EB0101141E73F1000405DBF6
:1089F0001C464FF00043524263EB04038B4208BF16
:108A0000824230BD70B58C1810F8015B15F0070379
:108A100001D110F8013B2A1106D110F8012B03E017
:108A200010F8016B01F8016B5B1EF9D12B0705D41F
:108A30000023521E0DD401F8013BFAE710F8013B68
:108A4000CB1A921C03E013F8015B01F8015B521E84
:108A5000F9D5A142D8D3002070BD027803E010F808
:108A6000013B1A44D2B2491E89B2F8D2104670476F
:108A700070B5ADF5287D00260D46ADF89462ADF8D1
:108A8000986200EB40012D4800EBC104608AA842C7
:108A900051D9ADF898624AE0A089228A284481B26F
:108AA000274800F0B1F8ADF894626A46208A0BE0DE
:108AB000BDF894326168C95CBDF89432D154BDF8F8
:108AC0009412491CADF89412BDF894128842EFD864
:108AD000401E81B21046FFF7C0FF1A498870228AF3
:108AE0000DF1FF31515C814219D1ADF894620CE077
:108AF000BDF894126068BDF89422405CA168885467
:108B0000BDF89402401CADF89402208ABDF894127E
:108B1000401E8842ECDC01200DF5287D70BD6420EC
:108B200013F074FABDF89802401CADF89802BDF835
:108B300098020628B0D30020EEE70000BCCF010861
:108B4000107C0020220A0020F0B50D46064600EBFE
:108B500046011C48002200EBC104ADF5257D608A6A
:108B6000A8422BD9694606E0A0686368805C9854E7
:108B70008854521C92B2208A401E9042F4DC208A13
:108B8000401E81B26846FFF768FF228A0DF1FF316F
:108B900000275054A089228A284481B2684600F0F8
:108BA0002FF929463046FFF763FF012807D06420DC
:108BB00013F02CFA7F1CBFB2062FEBD300200DF56B
:108BC000257DF0BDBCCF010838B50025ADF80050BB
:108BD0000FF038F90A4C207000F088F82178094825
:108BE000242907D0272908D0282902D1022180F87A
:108BF000E61138BD80F8E65138BD0121F7E70000E5
:108C0000220A0020A42200202DE9F0410646154644
:108C10000C46012080F31088254F0020B8800FF00B
:108C2000F1F8000609D4012013F0F0F9B888401CCF
:108C300080B2B880C828F2D335E0B888C82832D2CC
:108C40001C4F1021384601F0BCF90821384601F0CC
:108C5000BAF9E82000F030F8C4F3871000F02CF8DF
:108C6000A006000E00F028F8002000F025F80024EF
:108C7000002000F021F8641CA4B2042CF8D30024D6
:108C800005E0FF2000F018F83055641CA4B2AC4297
:108C9000F7D31021384601F096F9002080F31088B0
:108CA0000120BDE8F081002080F31088F9E7000082
:108CB000220A00200000024070B50B4C054602213C
:108CC00020460FF0B9F90028F9D0294620460FF0C8
:108CD000BCF9012120460FF0AFF90028F9D0204659
:108CE0000FF0B1F9C0B270BD0030014010B50120E5
:108CF00080F310881A4C0020A0800FF083F8000643
:108D000009D4012013F082F9A088401C80B2A08011
:108D1000C828F2D320E0A088C8281DD2114C102109
:108D2000204601F04EF90821204601F04CF93D2083
:108D3000FFF7C2FF2A20FFF7BFFF8020FFF7BCFF2D
:108D4000A720FFF7B9FF1021204601F03CF90020D1
:108D500080F31088012010BD002080F3108810BD22
:108D6000220A0020000002402DE9F04106460D468F
:108D7000012080F31088204C0020A0800FF042F8E2
:108D8000000609D4012013F041F9A088401C82B2EA
:108D9000A280C82AF2D32AE0A088C82827D2174F79
:108DA0001021384601F00DF90821384601F00BF981
:108DB0008420FFF781FF0020FFF77EFF0020FFF7F0
:108DC0007BFF0020FFF778FF002404E0305DFFF711
:108DD00073FF641CA4B2AC42F8D31021384601F0F2
:108DE000F2F8002080F310880120BDE8F081002017
:108DF00080F31088F9E70000220A002000000240FA
:108E000070B50D46012181F310881146FFF7ACFFC4
:108E1000002832D01B4C0020A0800EF0F3FF00068B
:108E200009D4012013F0F2F8A088401C80B2A08081
:108E3000C828F2D322E0A088C8281FD2124C1021E3
:108E4000204601F0BEF80821204601F0BCF883203E
:108E5000FFF732FFC5F38710FFF72EFFA806000EBD
:108E6000FFF72AFF0020FFF727FF1021204601F01F
:108E7000AAF8002080F31088012070BD002080F344
:108E8000108870BD220A00200000024010B50023A7
:108E90001A4604E010F8014B6340521CD2B28A42D9
:108EA000F8D3184610BD000010B50446392013F061
:108EB000ADFAE0B213F0CAFAC4F3072013F0C6FA11
:108EC000C4F3074013F0C2FA200E13F0BFFA4FF4B8
:108ED0008051034801F077F8BDE8104011F096BCCE
:108EE000000402402DE9F041054614460E463A20A2
:108EF00013F08CFAF0B213F0A9FA300A13F0A6FAC4
:108F0000104F4FF480563146384601F05CF8B046B9
:108F10003E4611F07BFC1D2811D1284600F0A4F834
:108F200007463B2013F072FA4146304601F04BF8F9
:108F30003D44002CEDD0208838442080E9E7BDE88E
:108F4000F0810000000402402DE9F041054614467E
:108F50000E463C2013F05AFAF0B213F077FA300ABA
:108F600013F074FA114F4FF480563146384601F031
:108F70002AF80CB100202080B0463E4611F046FC95
:108F80001E2811D1284600F017F907463D2013F09E
:108F90003DFA4146304601F016F83D44002CEDD034
:108FA000208838442080E9E7BDE8F08100040240D1
:108FB00010B50EF06FFE08B100F028F8BDE81040C3
:108FC000302000F09FB80146362000F089B810B577
:108FD00008B100F0A5F8BDE81040342000F092B8C8
:108FE00010B5044600F09CF820785C2801D02F28AA
:108FF00003D10021642000F0FBF8BDE810403220CE
:1090000000F080B8682000F04BB8000010B52220B6
:1090100013F0FCF913F0F0F904464FF480510248C4
:1090200000F0D1FF204610BD000402402DE9F041C0
:1090300013F0E2F9064613F0DFF9054613F0DCF908
:10904000044613F0D9F907464FF48051054800F063
:10905000BAFF46EA052040EA044040EA0760BDE85E
:10906000F08100000004024070B50546272013F08F
:10907000CDF913F0C1F90446260007D013F0BCF96E
:10908000641E05F8010B14F0FF04F7D14FF4805172
:10909000024800F098FF304670BD00000004024016
:1090A00010B504460C2013F0B1F9204613F0CEF9A8
:1090B000BDE81040FFF7BABF10B504460A2013F010
:1090C000A5F9204613F0C2F913F096F904464FF4BF
:1090D0008051024800F077FF204610BD0004024096
:1090E00010B50C4613F092F9204613F0AFF94FF487
:1090F0008051034800F067FFBDE8104011F086BBC7
:109100000004024010B513F081F94FF48051034878
:1091100000F059FFBDE8104011F078BB0004024098
:1091200070B50546012013F071F913F065F9432875
:1091300028D22B20FFF7C0FF102823D22F2013F0B6
:1091400065F9002013F082F93220FFF7DBFF1428C5
:1091500018D1CF20FFF7B0FF040013D04C20FFF749
:109160009FFF00EB04214C2000F042F85020FFF755
:1091700097FF00EB0421502000F03AF80021702006
:1091800000F036F82F2013F041F92C7806E015F89E
:10919000014F5C2C01D02F2C00D10024204613F06D
:1091A00055F9002CF3D1BDE870404FF480510148CF
:1091B00000F009BF0004024070B505462D2013F0F1
:1091C00025F913F019F90446260007D0287813F082
:1091D0003DF9641E6D1C14F0FF04F7D14FF480516B
:1091E000024800F0F0FE304670BD0000000402406E
:1091F00070B505460C460D2013F008F9284613F00B
:1092000025F9E0B213F022F9C4F3072013F01EF998
:10921000C4F3074013F01AF9200E13F017F9BDE854
:1092200070404FF48051014800F0CDBE0004024070
:1092300070B5094DFF22134605F5807605E010F85C
:10924000014B54402A5D5A40335D491E89B2F6D223
:1092500042EA032070BD000049CD010870B500222C
:109260001346154605E010F8014BA2186B41491E44
:1092700089B20029F7D1100C40EA034092B280185D
:1092800045EB13414FEA014242EA104108186FEAE8
:10929000000080B270BD08F0A1BD08F03FBD08F02D
:1092A0000DBD08F06BBD0AF005B80EF065B9000001
:1092B000074A904201D2074801E005481038064AA3
:1092C0008B0001EA020101D5C160704781607047DF
:1092D00010640240006002407D0F7D0F002901688C
:1092E00002D041F0010101E021F00101016070476D
:1092F0002DE9F043016821F00101016000210160C6
:1093000041608160C1600161212141613C493C4A69
:109310003D251039904202D18D60BDE8F083384A76
:109320004FF474661832904201D18E60F5E7344AEA
:109330004FF474173032904201D18F60EDE7304A1C
:109340004FF0746C4832904202D1C1F808C0E4E793
:109350002B4B2C4A6033984201D1CA60DDE7284C80
:10936000294B7834A04201D1CB60D6E7DFF890805A
:10937000264C08F19008404501D1CC60CDE7DFF8DC
:1093800080804FF03D5908F1A808404502D1C1F84E
:109390000C90C2E71E49DFF878800839404501D1BA
:1093A0000D60BAE71A4D1835A84201D10E60B4E736
:1093B000174D3035A84201D10F60AEE7144D483546
:1093C000A84202D1C1F800C0A7E7114D104960358D
:1093D000091FA84201D10A609FE70D4A78329042E6
:1093E00001D10B6099E70A4A9032904201D10C609A
:1093F00093E7074AA83290428FD1C1F800908CE7DA
:10940000106002403D000020400F002000003D2081
:10941000106402400B0607D5436912B143F0800384
:1094200001E023F080034361802908D0002A02680C
:1094300001F01E0101D00A4300E08A430260704738
:1094400030B50368124ACC6813400A682243D1E958
:1094500005452C432243CC6922430C6A22434C6AC3
:1094600022438C6A22434C6B22438C6B22431A4367
:109470000260426922F00703D1E90B2422431A4318
:1094800042610A6942604A6882608968C16030BD91
:109490003F801CF02DE9FC41012120200EF002FC50
:1094A00001268DF8046000258DF8065003208DF804
:1094B00005001B4C302700978DF807506946204661
:1094C00000F02CFD3021204600F07DFD154C84F885
:1094D000705684F8725684F8716684F873664FF497
:1094E000FA70C4F8780600F01FF894F8E9038028B1
:1094F00014D1A4F580508565232084F8EE0305205F
:1095000084F8ED0384F8EC73142084F8EB03202036
:1095100084F8EA0384F8E95300F042F8BDE8FC81DE
:1095200000140240A42200207CB512F043FED0209B
:1095300012F010FE12F072FE002012F00BFE12F07C
:109540006DFE12F037FED12012F004FE12F066FE1E
:1095500000246D4601E0062C01D2012000E000202D
:1095600012F0C8FD2855641CE4B2072CF3D312F0A6
:109570003BFE0A489DF8061041719DF805100171E7
:109580009DF80410C1709DF8021081709DF80110C3
:1095900041709DF8001001707CBD00008D260020F8
:1095A0007CB51848002401788DF8001041788DF8BA
:1095B000011081788DF8021001218DF80310C17817
:1095C0008DF8041001798DF8051040798DF80600AA
:1095D00012F0F0FDD02012F0BDFD12F01FFE0020B1
:1095E00012F0B8FD12F01AFE6D46285D12F0B2FDC1
:1095F00012F014FE641CE4B2072CF6D312F0F4FD52
:109600007CBD00008D26002070B5094D0022134658
:1096100005F5807605E010F8014B54402A5D5A406C
:10962000335D491E89B2F6D242EA032070BD0000C4
:1096300049CD0108072A00D9072240EA002021B1BC
:10964000012901D1D040C0B270479040C0F307203B
:1096500070477047072A00D9072240EA002029B145
:10966000012902D19040C0F307207047D040C0B21A
:109670007047000070B5ADF5327D00260D46ADF89F
:10968000BC62ADF8C06200EB4001324800EBC1049F
:10969000608AA8425CD9ADF8C06255E0012264211D
:1096A0002D4800F0BFF92C4800788DF800003828CC
:1096B00042D1228AE06802FB0501274800F0B2F996
:1096C000ADF8BC626A46208A0BE0BDF8BC32616826
:1096D000C95CBDF8BC32D154BDF8BC12491CADF810
:1096E000BC12BDF8BC128842EFD8401E81B21046B1
:1096F00000F05AFA228A0DF1FF31515C81421BD1F0
:10970000ADF8BC620EE0BDF8BC226168895CA2685D
:1097100000FB0520BDF8BC221154BDF8BC02401C62
:10972000ADF8BC02208ABDF8BC12401E8842EADCBB
:1097300001200DF5327D70BD642012F067FCBDF88C
:10974000C002401CADF8C002BDF8C0020628A5D377
:109750000020EEE710C9010834570020F0B50E468E
:10976000074600EB47012648ADF5317D002500EBAB
:10977000C1048DF8BC52608AB0423DD90021084630
:10978000FFF778FF012837D1694609E0A268401E3B
:1097900000FB06206268285C505548556D1CADB230
:1097A000208AA842F2D80025208AE16800FB061131
:1097B000401E82B2134800F0B3F9208A401E81B2E5
:1097C000684600F0F1F98DF8BC02208AE1680122B8
:1097D00001447043401E0144AFA800F0A1F9314696
:1097E0003846FFF747FF012807D0642012F00EFC2F
:1097F0006D1CADB2062DD7D300200DF5317DF0BD27
:1098000010C90108345700202DE9F041ADF5307D35
:10981000354D4FF000088DF8BC82344EA5F800801D
:1098200000243FE000206F4607E056F832204968E8
:10983000125C0A543A54401C80B2298801EB410260
:1098400006EBC2010B8A5B1E8342EEDC288800EB2C
:10985000400006EBC000008A401E81B2384600F08E
:10986000A3F98DF8BC02288800EB400006EBC0008D
:10987000C168008A00FB0411401E82B21C4800F03F
:109880004FF92888012200EB400006EBC000C168B8
:10989000008A01446043401E0144AFA800F040F933
:1098A000641CA4B2288800EB400006EBC000408A8C
:1098B000A042B7D82888401C80B228800B28AFD39C
:1098C0000C48017821F001010170017841F0060196
:1098D0000170A0F8028000210120FFF73FFF0DF585
:1098E000307DBDE8F08100001000002010C90108A3
:1098F00034570020802400207CB5012108460EF05A
:10990000D1F901208DF8040002258DF805500024BE
:109910008DF806408DF807001820154E0090694616
:10992000304600F0FBFA05221146304600F032FBCB
:1099300005220621304600F02DFB05220721304686
:1099400000F028FBA02000908DF8045003208DF833
:1099500005008DF806408DF807406946304600F056
:10996000DDFA402000906946304600F0D7FA7CBD11
:1099700000000240F8B5002634460096FFF7BCFF11
:1099800000F0A0F82248641C8442FCD3214C08213A
:10999000204600F016FB1021204600F014FB0620A4
:1099A00000F076F80821204600F00DFB0821204643
:1099B00000F007FB1021204600F005FB012000F01D
:1099C00067F8002000F064F80821204600F0FBFA58
:1099D0001148D0F81C0208B9FFF716FF0F4D2E8072
:1099E0000F4E002405E0C0B22146FFF743FE641C81
:1099F000A4B2288800EB400106EBC101498AA142CC
:109A0000F1D880B2401C80B228800B28E9D3F8BD81
:109A1000FFFF0F0000000240000043421000002042
:109A200010C901082DE9F0410546002416460F46ED
:109A3000012080F31088DFF854800821404600F0B0
:109A4000C0FA1021404600F0BEFA032000F020F8D2
:109A5000C7F3074000F01CF8C7F3072000F018F820
:109A6000F8B200F015F806E0002000F011F8641CD0
:109A700005F8010BA4B2B442F6D30821404600F029
:109A8000A2FA002080F31088BDE8F08100000240B7
:109A900070B50B4C0546022120460EF0CDFA002889
:109AA000F9D0294620460EF0D0FA012120460EF0CA
:109AB000C3FA0028F9D020460EF0C5FAC0B270BD36
:109AC0000030014010B5012186B008030EF026F9E0
:109AD000124C20460EF086FA0021ADF808106015F1
:109AE000ADF80A003820ADF80C000720ADF80010E2
:109AF000ADF81000ADF804104FF48270ADF8061008
:109B0000ADF80E10ADF80200694620460EF09FFA3F
:109B1000012120460EF05CFA06B010BD0030014075
:109B20002DE9F0410546002416460F46012080F33A
:109B30001088DFF870800821404600F042FA1021BA
:109B4000404600F040FA0620FFF7A2FF08214046F9
:109B500000F039FA0821404600F033FA102140465F
:109B600000F031FA0220FFF793FFC7F30740FFF739
:109B70008FFFC7F30720FFF78BFFF8B2FFF788FFCF
:109B800005E02878FFF784FF641CA4B26D1CB44282
:109B9000F7D30821404600F016FA002080F3108821
:109BA000BDE8F08100000240027803E010F8013BBC
:109BB0001A44D2B2491E89B2F8D21046704700004A
:109BC00070B51E4A907B012825D1002595731C494C
:109BD0001C480F244E780123F6B14D70D0F828525E
:109BE000D0F8346245EAC605D0F83062D0F82C02CD
:109BF000B60046EA40000543AC43CC708878CC7888
:109C0000A04208D108710C78A04204D010720870EC
:109C1000002800D0D37170BD4B70D0F82852D0F816
:109C2000346245EAC605D0F83062D0F82C02B6009E
:109C300046EA40000543AC438C70DFE7A4120020E5
:109C4000C90A0020000042422DE9F041ADF57C7DBB
:109C500000273D46ADF8E873FFF7AAF9142808D0AD
:109C6000664880F8E85312F00DFB0DF57C7DBDE8E9
:109C7000F0816348FFF7B4F9614C103C1428207060
:109C800006D0422879D00120FFF79DF92570ECE736
:109C9000FFF7B8F9C4E90205A046BDF8E803FFF7ED
:109CA00003F9FAAA4FF4FA716846FFF71BF955A1B8
:109CB000684612F04BFBA080544C6E46F0B1E1199F
:109CC00001F5805181F83F577F1CBFB2282FF6D392
:109CD000474630444EA112F039FB78800021001F26
:109CE0000AE0BA880A443244D378621802F58052F6
:109CF00082F83F37491C89B28142F2DB45A16846B0
:109D000012F024FB4746A8F80400F0B100216218C5
:109D100002F5805282F86757491C89B22829F6D388
:109D200030443BA112F012FB7880002109380AE090
:109D3000BA880A443244137A621802F5805282F8D3
:109D40006737491C89B28142F2DB35A1684612F0BF
:109D5000FDFAB880F8B10021621802F5805282F84D
:109D60008F57491C89B21429F6D3304428A112F028
:109D7000EDFA788000210D380BE03AE0BA880A4409
:109D80003244137B621802F5805282F88F37491CE7
:109D900089B28142F2DB26A1684612F0D7FAB88078
:109DA000F0B10021621802F5805282F8F956491C80
:109DB00089B23229F6D3304415A112F0C7FA78805F
:109DC0000021C01F0AE0BA880A443244937962181D
:109DD00002F5805282F8F936491C89B28142F2DBE1
:109DE00000210320FFF7BAFC0120FFF7ECF8012067
:109DF0003BE70348FFF7EBF837E70000A422002019
:109E0000380A002041504E3D00000000A4120020FE
:109E10003B000000574946494E414D453D0000007A
:109E20005749464950415353574F52443D00000053
:109E30005345525645523D002F4910B5884206D130
:109E4000012108460DF03AFF002101204FE02B4987
:109E5000884206D1012102200DF030FF00210220AE
:109E600045E02749884206D1012104200DF026FF54
:109E7000002104203BE02349884206D1012108202B
:109E80000DF01CFF0021082031E01F49884206D157
:109E9000012110200DF012FF0021102027E01B49A6
:109EA000884206D1012120200DF008FF002120204A
:109EB0001DE01749884206D1012140200DF0FEFE29
:109EC0000021402013E01349884206D1012180205F
:109ED0000DF0F4FE0021802009E00F4988420AD1EC
:109EE0008415012120460DF0E9FE00212046BDE841
:109EF00010400DF0E3BE10BD00000240000402401F
:109F000000080240000C0240001002400014024011
:109F100000180240001C024000200240F0B5002260
:109F200001274FF0030C0B6807FA02F52B40AB42F8
:109F30002CD1066853000CFA03F4A64306600E7990
:109F4000D0F800E09E4046EA0E0606600E79012E2B
:109F500001D0022E12D18668A64386604E79D0F8D1
:109F600008E09E4046EA0E0686604668AE434660BC
:109F700045688E799640B6B235434560C568A543BD
:109F8000C560CC799C40C3681C43C460521C102A35
:109F9000C9D3F0BD4B07DB0E9A40C90810B500EBE2
:109FA0008100016A0F249C40A1430162016A1143B0
:109FB000016210BD0246002012690A4200D0012051
:109FC0007047418370470183704700000249087A57
:109FD00000220A7270470000A412002002480068A4
:109FE000C00700D000BEFEE7F0ED00E002494AF6EF
:109FF000AA200860704700000030004010B512F041
:10A0000041F9BDE81040642012F000B82DE9F04F8E
:10A0100083466AA0ADF57D7D002500689A460F460F
:10A02000A946FB90ADF8E853042A25D8644C94F86F
:10A03000ED03302101EB101302EBC20000EB021222
:10A0400060481618337194F8ED0300F00F003030BB
:10A05000707194F8EC0301EB1010B07194F8EC03FC
:10A0600000F00F003030F071FEF7A2FF142807D087
:10A0700084F8E89312F006F90DF57D7DBDE8F08FC8
:10A08000DFF84081A8F1240898F8000014280ED0C9
:10A090003046FEF7A5FF88F80000142807D04228B4
:10A0A0007ED00120FEF78FFF88F80090E4E74FF4A0
:10A0B0007A70874200D90746FEF7A4FFC8E9020973
:10A0C0004E46FEF7F1FE94F8EC13302000EB111130
:10A0D0008DF8001094F8EC1301F00F0130318DF879
:10A0E000011094F8EB1300EB11118DF8021094F8A5
:10A0F000EB1301F00F0130318DF8031094F8EA13DF
:10A1000000EB11118DF8041094F8EA1301F00F011F
:10A1100030318DF8051094F8E91300EB11108DF82B
:10A12000060094F8E90300F00F0030308DF80700C6
:10A13000BAF1000F03D0BAF1010F02D004E05420AD
:10A1400000E052208DF808003A208DF809000A231B
:10A150006C4617E00BEB550108780009B0FBF3F2F1
:10A16000C2EBC2021044621930309072087800F0DD
:10A170000F00B0FBF3F1C1EBC10108443030AD1C5E
:10A18000D072ADB2B5EB470FE4D303EB470081B219
:10A19000FAAA2046FEF7D8FEFAAA0221FBA800E0A0
:10A1A00007E0FEF7D1FE0120FEF70DFF88F8006002
:10A1B00062E73046FEF70BFF5EE700000D0A000085
:10A1C000A42200204C0A00202DE9F04F4FF0000B94
:10A1D0002DED028BA1B08DF824B08DF828B08DF84C
:10A1E0002CB0CDE912BBCDE900BB8DF808B08DF8DD
:10A1F0000CB08DF820B08DF814B0ADF818B09FED0C
:10A20000FE0AFE4C8DED0D0A04F12900079004F5BD
:10A210009C5004F5804A41F686554FF0010904F53B
:10A220008054049099E094F82A0B20B384F82ABB58
:10A23000BAF83C04F24ED6F88C10C1F57A71884217
:10A2400019D156F88C0FC0F57A70AAF83404EC4F87
:10A25000002188373846FFF741F8EA493846FFF7CA
:10A2600027F8E94981F800904FF47A7030600121B5
:10A270003846FFF733F894F8360B10B384F836BB42
:10A28000BAF83E04DE4E716CC1F57A71884218D17D
:10A29000706CC0F57A70AAF83604D94F00214037A7
:10A2A0003846FFF71BF8D9493846FFF701F8D64979
:10A2B00081F801904FF47A70706401213846FFF7FD
:10A2C0000DF894F8420B10B384F842BBBAF840047E
:10A2D000CB4E7169C1F57A71884218D17069C0F5A9
:10A2E0007A70AAF83804C64F002110373846FEF7B6
:10A2F000F5FFC7493846FEF7DBFFC34981F80290F6
:10A300004FF47A70706101213846FEF7E7FF94F848
:10A310004E0B10B384F84EBBBAF84204B84EF16A43
:10A32000C1F57A71884218D1F06AC0F57A70AAF83E
:10A330003A04B34F002128373846FEF7CFFFB5491E
:10A340003846FEF7B5FFB04981F803904FF47A70B4
:10A35000F06201213846FEF7C1FF94F82A0B94F809
:10A36000361B94F8422B014494F84E0B1044C14222
:10A370007FF459AF05F0BEBF017821B180F800B07D
:10A380008DF808B012E0417819B180F801B0484664
:10A390000AE0817819B180F802B0022004E0C178A7
:10A3A00021B180F803B003208DF808009DF8080063
:10A3B00000EB400101EB0011904800EB011000F5AB
:10A3C000805090F85A1D9DF8080000EB4002C2EB47
:10A3D000C012914810F83200C1280BD19DF8080036
:10A3E00000EB4002C2EBC0128B4800EBC200807849
:10A3F00008280CD0082985F04A87DFE811F0581F9B
:10A400002700F10A92145A1DFF1E7E226F268AF839
:10A410008C949DF8080030B1012807D002280FD095
:10A42000032808D10FE04FF4804101E04FF40051C0
:10A430007A48FFF7C6FD7A49C1F888B205F027BF10
:10A440004FF48051F4E74FF40061F1E79DF8080004
:10A45000DFF8C48100EB4001C1EBC01108EBC10083
:10A4600040785E46002107F05BFB8DF820008DF8F8
:10A470002C60624F1BE09DF8080000EB400101EBEF
:10A4800000109DF82C1007EB001000EB011000F5F8
:10A49000805090F8850D9DF8201088429DF82C0082
:10A4A00002D18DF8200012E0401C8DF82C009DF8A0
:10A4B000080000EB400101EB001007EB001000F575
:10A4C000805090F85B0D9DF82C108842D3D89DF8F1
:10A4D000080000EB4001C1EBC01008EBC000807821
:10A4E0000A21B1EB101F9DF8080000EB4001C1EB01
:10A4F000C01008EBC000807801D100F00F008DF88B
:10A500000C009DF80C0010B910208DF80C009DF87F
:10A51000080000EB4001C1EBC0109DF80C1008EBE7
:10A52000C00008444078ADF818009DF8080000EB22
:10A530004001C1EBC0109DF80C1008EBC000491C95
:10A5400007F0CFFE8DF828009DF8080000EB4001D1
:10A55000C1EBC0109DF80C1008EBC00008448078D7
:10A560009DF82810884245F092869DF8080000EB7F
:10A570004001C1EBC01008EBC0004078002805F096
:10A5800086869DF8080000EB4001C1EBC01008EB87
:10A59000C0019DF80C000844C1789DF8080000EB4C
:10A5A000001202EB002007EBC0029DF8200000EB38
:10A5B000001002EBC00000F5005080F858129DF822
:10A5C000080007EB00119DF82000084400F58050BA
:10A5D00080F8886B387E012837D19DF8080000EBA1
:10A5E000400101EB001007EB00119DF8200001EB8A
:10A5F00000102844017815E000000000A41200209B
:10A60000006002400088002012000020008020101E
:10A610002080001000880010806400200018024094
:10A620000000424241F080010170BDF81800B628D8
:10A6300005D0C52803D0D52801D0D92803D19DF84D
:10A640000C00032801D2ADF81860BDF81800CE2820
:10A6500013D013DCB9287DD009DC5A288FD0B2285A
:10A6600079D0B528F7D0B62845F01186FEE3C32887
:10A6700072D0C52871D0CA28F6D1F8E3E128FCD001
:10A6800006DCD52809D0D728E8D0D928ECD1E8E2D3
:10A69000E5287CD0E728E7D1EAE39DF8080000EB45
:10A6A0004001C1EBC01008EBC000C07884F8E201A3
:10A6B0009DF8080000EB001101EB002007EBC00142
:10A6C0009DF8200000EB001001EBC00000F50050E9
:10A6D00090F81C0201289DF8080000EB400101EBF6
:10A6E00000107DD09DF82020B846394607EB0010B9
:10A6F00000EB021094F8E2312844A9EBD31302785E
:10A7000063F3000202709DF8080000EB400202EBC8
:10A7100000109DF8202007EB001000EB021094F8C9
:10A72000E22128445309027863F3410202709DF844
:10A73000080000EB400202EB00109DF8202001EB26
:10A74000001000EB021000F5805090F8860DC0F369
:10A75000400203E0FEE3FEE3FEE3FEE39DF80800B3
:10A7600000EB001303EB002008EBC0019DF8200074
:10A7700000EB001001EBC00000F5005090F834022F
:10A78000C0F34000824254D09DF8080000E0E5E3A9
:10A7900000EB001101EB002008EBC0029DF8200047
:10A7A000414600EB001002EBC00042F234220244AA
:10A7B0009DF8080000EB400303EB00109DF82030EB
:10A7C00008EB001000EB031000F5805090F8860DA8
:10A7D0004308107863F3410010709DF8080000E012
:10A7E00028E000EB400202EB00109DF8202001EB76
:10A7F000001000EB021000F5805090F8860D8007E5
:10A8000048D59DF80800D92200EB001303EB002087
:10A8100008EBC0019DF8200000EB001001EBC00028
:10A8200000F5005080F821229DF808100220FEF764
:10A8300095FF78E09DF8201007EB001000EB011069
:10A8400094F8E2212844A9EBD212017862F30001C6
:10A8500001709DF8080000EB001101EB002007EBF0
:10A86000C00000F5005080F817629DF80800022132
:10A8700000EB001202EB002007EBC0029DF8200065
:10A8800000EB001002EBC00000F5005080F81C1235
:10A89000B6218AE39DF808004A4600EB001303EB5B
:10A8A000002001EBC0079DF8200000EB001007EB33
:10A8B000C00000F5005080F829929DF80800D927C3
:10A8C00000EB001303EB002001EBC00C9DF820000F
:10A8D00000EB00100CEBC00000F5005080F8217276
:10A8E0009DF8080000EB400303EB00109DF82030BA
:10A8F00001EB001000EB03102844037823F020073D
:10A9000007709DF8080000EB001303EB002008EB34
:10A91000C0019DF8200000EB001001EBC00000F525
:10A92000005080F85A229DF808009DF8202000EB86
:10A93000400101EB001008EB001000EB021000F5E5
:10A94000805090F8860D00F001029DF8080000EBA1
:10A95000001303EB002008EBC0019DF8200000EB82
:10A96000001001EBC00000F5005090F8340200F038
:10A970000100824270D09DF80800474600EB0011AC
:10A9800001EB002008EBC0019DF8200000EB001057
:10A9900001EBC00042F2342101449DF8080000EBB5
:10A9A000400202EB00109DF8202008EB001000EBA5
:10A9B000021000F5805090F8860D0A7860F30002CE
:10A9C0000A709DF8080000EB400101EB00109DF8B3
:10A9D000201007EB001000EB011000F5805090F8FC
:10A9E000860DC0079DF8080037D000EB001101EB81
:10A9F000002007EBC0019DF8200000EB001001EBE8
:10AA0000C00000F5005090F85A02E0B39DF808002D
:10AA100000EB001101EB002007EBC0029DF82000C5
:10AA200000EB001002EBC00000F5005080F8596206
:10AA30009DF8080000EB400101EB00109DF820108C
:10AA400007EB001000EB01102844017821F001020F
:10AA5000027094F8A407B8B3EDE000EB400101EBFD
:10AA600000109DF8201007EB001000EB01102844A7
:10AA7000017821F0200202709DF8080000EB00111F
:10AA800001EB002000E00CE008EBC0029DF8200084
:10AA900000EB001002EBC00000F5005080F8596296
:10AAA000C9E09DF8080000EB001202EB002007EB64
:10AAB000C0029DF8200000EB001002EBC00000F582
:10AAC000005080F85992C4E7FFE7787E012868D1EA
:10AAD000B86D798B884264D29DF8080000EB0011B4
:10AAE00001EB002007EBC0019DF8200000EB0010F7
:10AAF00001EBC00000F5005090F85902012850D138
:10AB00009DF8080000EB001101EB002007EBC001ED
:10AB10009DF8200000EB001001EBC00000F5005094
:10AB200090F89302E8BB9DF8080000EB400101EBB0
:10AB3000001007EB00119DF8200001EB001000F55C
:10AB4000805090F8841D9DF8080000EB001202EB85
:10AB5000002007EBC00000F5005080F815129DF8AA
:10AB60000800C32100EB001202EB002007EBC0023B
:10AB70009DF8200000EB001002EBC00000F5005033
:10AB800080F821129DF8080000EB400101EB001055
:10AB900007EB00119DF8200001EB001000F580503C
:10ABA00000E048E0C0F8886D9DF808100220FEF72C
:10ABB000D5FD8DF8246019E09DF8080000EB001128
:10ABC00001EB002007EBC0019DF8200000EB001016
:10ABD00001EBC0009DF82410084400F5005080F8F7
:10ABE0005B629DF82400401C8DF824009DF8240031
:10ABF0001428E1D38DF8246019E09DF8080000EBDB
:10AC0000001101EB002007EBC0019DF8200000EBD4
:10AC1000001001EBC0009DF82410084400F500501E
:10AC200080F877629DF82400401C8DF824009DF880
:10AC300024000A28E1D39DF808009DF8202000EBAD
:10AC4000400101EB001008EB001000EB021000F5D2
:10AC5000805090F8860D800745F11983D92204F0C1
:10AC600028BF9DF8080000EB400101EB001007EB46
:10AC7000001000F5805090F8600D00289DF80C0041
:10AC800003D00A2845F0038382E00828FAD18DF822
:10AC9000246024E09DF8080000EB4001C1EBC010E7
:10ACA0009DF8241008EBC0000844C07800F00F00A5
:10ACB000092818D89DF8080000EB4001C1EBC0102E
:10ACC0009DF8241008EBC0000844C07800F0F000A4
:10ACD000902808D89DF82400401C8DF824009DF889
:10ACE00024000628D6D39DF824000628C5F0CF827C
:10ACF0009DF8080000EB4001C1EBC01008EBC0005C
:10AD0000C07801049DF8080000EB4002C2EBC010BF
:10AD100008EBC000007941EA00219DF8080000EB33
:10AD20004002C2EBC01008EBC000407901439DF81F
:10AD3000080000EB001202EB002007EBC0029DF8B8
:10AD4000200000EB001002EBC00000F50050C0F83E
:10AD500035129DF8080000EB4001C1EBC01008EB74
:10AD6000C000807901049DF8080000EB4002C2EBAE
:10AD7000C01008EBC000C07941EA00219DF808002E
:10AD800000EB4002C2EBC01008EBC000007A99E073
:10AD90008DF8246024E09DF8080000EB4001C1EB31
:10ADA000C0109DF8241008EBC0000844C07800F0E3
:10ADB0000F00092818D89DF8080000EB4001C1EBEE
:10ADC000C0109DF8241008EBC0000844C07800F0C3
:10ADD000F000902808D89DF82400401C8DF824002D
:10ADE0009DF824000828D6D39DF824000828C5F033
:10ADF0004E829DF8080000EB4001C1EBC01008EB4B
:10AE0000C00081799DF8080000EB4002C2EBC01041
:10AE100008EBC000C07841EA00619DF8080000EB33
:10AE20004002C2EBC01008EBC000007902049DF89C
:10AE3000080000EB4003C3EBC01008EBC0004079F2
:10AE400042EA002001439DF8080000EB001202EBEB
:10AE5000002007EBC0029DF8200000EB001002EB81
:10AE6000C00000F50050C0F8351202E0EAE0DAE078
:10AE7000FDE39DF8080000EB4001C1EBC01008EBBA
:10AE8000C000817A9DF8080000EB4002C2EBC010C0
:10AE900008EBC000C07941EA00619DF8080000EBB2
:10AEA0004002C2EBC01008EBC000007A02049DF81B
:10AEB000080000EB4003C3EBC01008EBC000407A71
:10AEC00042EA002001439DF8080000EB001202EB6B
:10AED000002007EBC0029DF8200000EB001002EB01
:10AEE000C00000F50050C0F839129DF8080000EBD2
:10AEF000001101EB002007EBC0019DF8200000EBE2
:10AF0000001001EBC00000F5005090F81C0203286F
:10AF10009DF808002BD000EB400101EB00109DF8DC
:10AF2000201007EB001000EB011000F5805090F8A6
:10AF3000860D800777D49DF8080000EB001101EB27
:10AF4000002007EBC0019DF8200000EB001001EB92
:10AF5000C00004E068E016E13CE03FE1FDE300F5FD
:10AF6000005090F82A02012820D005F090B900EB9B
:10AF7000001101EB002007EBC00000F5005080F845
:10AF800017629DF80800042100EB001202EB00207C
:10AF900007EBC0029DF8200000EB001002EBC000A0
:10AFA00000F5005080F81C12C521FDE39DF8080053
:10AFB00000EB001101EB002007EBC0019DF8200021
:10AFC00000EB001001EBC00000F5005080F82A6291
:10AFD000B6218BE09DF80800D52100EB001202EBB2
:10AFE000002007EBC0029DF8200000EB001002EBF0
:10AFF000C00000F5005080F821129DF8080000EB19
:10B00000001202EB002007EBC00000F5005080F8B2
:10B0100017929DF8080000EB400101EB001007EBD0
:10B02000001004F077BDFCE39DF8080000EB001170
:10B0300001EB002007EBC00000F5005080F817621C
:10B04000C321B1E39DF8080000EB400101EB0010C3
:10B0500007EB001000F5805090F8600D00289DF877
:10B06000080000EB4001C1EBC01008EBC0005CD051
:10B07000C07801049DF8080000EB4002C2EBC0104C
:10B0800008EBC000007941EA00219DF8080000EBC0
:10B090004002C2EBC01008EBC000407901439DF8AC
:10B0A000080000EB001202EB002007EBC0029DF845
:10B0B000200000EB001002EBC00000F50050C0F8CB
:10B0C00050129DF8080000EB001101EB002007EB87
:10B0D000C0019DF8200000EB001001EBC00000F55E
:10B0E000005090F81C0202282CD0C5219DF80800C1
:10B0F00000EB001202EB002007EBC0029DF82000DD
:10B1000000EB001002EBC00000F5005080F82112A7
:10B110009DF8080000EB001101EB002007EBC000D8
:10B1200000F5005080F817621FE701799DF80800CC
:10B1300000EB4002C2EBC01008EBC000C07841EA4F
:10B140000021ACE79DF8080000EB001101EB0020A6
:10B1500007EBC00000F5005080F817629DF808006A
:10B16000032100EB001202EB002007EBC0029DF868
:10B17000200000EB001002EBC00000F5005080F84A
:10B180001C12D921E4E39DF8080000EB001202EB49
:10B19000002007EBC00000F5005080F817929DF8E2
:10B1A0000800D52100EB001202EB002007EBC002E3
:10B1B0009DF8200000EB001002EBC00000F50050ED
:10B1C00080F821129DF8080000EB400101EB00100F
:10B1D00007EB001004F0DFBC0170C6E69DF8080024
:10B1E000BE4600EB400101EB001107EB011000F53A
:10B1F000805090F8600D00289DF80C0002D00E28B9
:10B2000092D19FE00C288FD18DF8246024E09DF826
:10B21000081001EB4100C0EBC1109DF8241008EBB1
:10B22000C0000844C07800F00F00092818D89DF825
:10B23000081001EB4100C0EBC1109DF8241008EB91
:10B24000C0000844C07800F0F000902808D89DF8AD
:10B250002410491C8DF824109DF824000A28D6D308
:10B260009DF824000A28B8D30020CDE9000030461C
:10B270008DF824601FE0DDE90012120242EA11623B
:10B280000902CDE900129DF8081001EB4102C2EB62
:10B29000C1119DF8242008EBC1011144CA78DDE9F1
:10B2A00000371A4340EA0701CDE900219DF8241038
:10B2B000491C8DF824109DF824100529DBD3DDE905
:10B2C00000239DF8081001EB011707EB01210EEB9D
:10B2D000C10C9DF82010774601EB01110CEBC10168
:10B2E00001F5005CCCF83D226146C1F841320022F4
:10B2F000CDE900228DF824001FE0DDE900121202E2
:10B3000042EA11620902CDE900129DF8081001EB32
:10B310004102C2EBC1119DF8242008EBC101114488
:10B32000097ADDE90023114340EA0302CDE9001266
:10B330009DF82410491C8DF824109DF8241005292F
:10B34000DBD39DE08DF8246024E09DF8081001EB2C
:10B350004100C0EBC1109DF8241008EBC000084468
:10B36000C07800F00F00092818D89DF8081001EBEC
:10B370004100C0EBC1109DF8241008EBC000084448
:10B38000C07800F0F000902808D89DF82410491CDF
:10B390008DF824109DF824000C28D6D39DF82400A5
:10B3A0000C28C4F074870020CDE9000030468DF8E9
:10B3B00024601FE0DDE90012130243EA1163090271
:10B3C000CDE900139DF8081001EB4102C2EBC11159
:10B3D0009DF8242008EBC1011144C978DDE9003251
:10B3E000194340EA0203CDE900139DF82410491CDB
:10B3F0008DF824109DF824100629DBD3DDE9002305
:10B400009DF8081001EB011707EB01210EEBC10CB1
:10B410009DF82010774601EB01110CEBC10101F5FD
:10B42000005CCCF83D226146C1F841320022CDE9F2
:10B4300000228DF824001FE0DDE90012120242EA2A
:10B4400011620902CDE900129DF8081001EB4102DA
:10B45000C2EBC1119DF8242008EBC1011144497AC7
:10B46000DDE90023114340EA0302CDE900129DF813
:10B470002410491C8DF824109DF824100629DBD3D4
:10B48000DDE900129DF8080000EB001303EB00203B
:10B4900007EBC0039DF8200000EB001003EBC00099
:10B4A00000F50053C3F845121846C0F849229DF82C
:10B4B0000800F04600EB001101EB00200EEBC0028B
:10B4C0009DF8200000EB001002EBC00000F50050DA
:10B4D00090F81C229DF8080000EB001303EB0020FD
:10B4E0000EEBC00000F5005090F8180282427DD1AA
:10B4F00094F8A40780B19DF8080000EB400101EB2F
:10B50000001108EB01109DF8201000EB01102844F9
:10B51000017841F0080194E04746C8F839609DF889
:10B52000080000EB001101EB002008EBC0019DF8C2
:10B530002000102200EB001001EBC00142F23D2080
:10B5400001440798FCF781FE9DF8080000EB00110C
:10B5500001EB002007EBC0019DF8200000EB00107C
:10B5600001EBC00000F2352000F500500168C7F87B
:10B570001D104068C7F821009DF8080000EB40014D
:10B5800001EB001007EB00119DF8200001EB00100B
:10B5900000F5805090F8840D3877049850F8691FB2
:10B5A000C7F83D108088A7F841009DF8080000EB1F
:10B5B000001101EB002007EBC0019DF8200000EB1B
:10B5C000001001EBC00000F50050D0F85002C7F8A1
:10B5D00025009DF8080000EB400101EB001007EB8F
:10B5E00000119DF8200001EB001000E0B9E000F52B
:10B5F0008050D0F8880DC7F84300B86D81B20220A2
:10B60000FDF7A2FA00210620FEF7A8F8B86D798BA5
:10B61000884202D2B86D401CB86500210520FEF7B3
:10B620009DF89DF8080000EB400101EB00109DF82B
:10B63000201007EB001000EB01102844017821F0E6
:10B64000080101709DF808100220FEF787F89DF8A8
:10B6500020009DF80810474600EB0110C117CDE906
:10B66000000100EB8001C1EB8010384400E0B4E140
:10B67000C0F87D609DF8081001EB011202EB01217A
:10B6800008EBC1029DF820106D3001EB011102EBB7
:10B69000C10242F23D2111441022FCF7D6FD9DF873
:10B6A000080000EB001101EB002007EBC0019DF842
:10B6B000200000EB001001EBC001009801F23521E1
:10B6C00000EB800201F50051C2EB80100A6838449B
:10B6D00040F8612F496841609DF8081001EB410274
:10B6E00002EB01119DF8202007EB011101EB021183
:10B6F00001F5805191F8841D00F8011C049951F85E
:10B70000692F0262898881849DF8081001EB01127B
:10B7100002EB012107EBC1029DF8201001EB0111A2
:10B7200002EBC10101F50051D1F8501281609DF882
:10B73000081001EB410202EB01119DF8202007EBFC
:10B74000011101EB021101F58051D1F8881DC0F8FB
:10B750002610009881B2082000E0B0E0FDF7FEFF5F
:10B7600010E09DF8080000EB400101EB001108EB30
:10B7700001109DF8201000EB01102844017841F0E1
:10B78000040101709DF8080000EB001101EB00209E
:10B7900008EBC0029DF82000414600EB001002EBD0
:10B7A000C00000F5005000E0D2E080F85A629DF839
:10B7B0000800D52200EB001303EB002008EBC003C8
:10B7C0009DF8200000EB001003EBC00000F50050D6
:10B7D00080F821229DF8080000EB001202EB002007
:10B7E00001EBC0029DF8200000EB001002EBC0004E
:10B7F00000F5005090F81C02042844F048859DF89C
:10B80000080000EB400202EB00109DF8202001EB45
:10B81000001000EB02102844027842F0800202700F
:10B8200000E04AE09DF8080000EB001303EB002065
:10B8300001EBC00000F5005080F817929DF8080059
:10B84000052200EB001303EB002001EBC0039DF881
:10B85000200000EB001003EBC00000F5005080F862
:10B860001C22FCE39DF8080000EB400202EB0010F4
:10B870009DF8202001EB001000EB02102844027814
:10B8800022F0020303709DF8080000EB400202EB77
:10B8900000109DF8202001EB001000EB021028445E
:10B8A000027822F0200303709DF8080000EB4002AC
:10B8B00002EB001008EB0010FDE3D52148E04946FB
:10B8C00084F8E0969DF8080000EB001202EB0020DF
:10B8D00007EBC0029DF8200000EB001002EBC00057
:10B8E00000F5005090F81C0200289DF8080012D0C6
:10B8F00000EB001101EB002007EBC0019DF82000D8
:10B9000000EB001001EBC00000F5005090F81E02A3
:10B91000B22830D008E400EB001202EB002007EB65
:10B92000C00000F5005080F817629DF8080000EB99
:10B93000001202EB002007EBC0029DF8200000EB94
:10B94000001002EBC00000F5005080F81C12B4E7B4
:10B950009DF8080000EB001202EB002007EBC0028C
:10B960009DF8200000EB001002EBC00000F5005035
:10B9700080F8211231E49DF8080000EB001101EB82
:10B98000002007EBC00000F5005080F817629DF81A
:10B990000800B22100EB001202EB002007EBC0020E
:10B9A0009DF8200000EB001002EBC00000F50050F5
:10B9B00080F821129DF8080000EB001101EB002037
:10B9C00007EBC0019DF8200000EB001001EBC00068
:10B9D00000F5005080F81E629CE784F8E0666CE792
:10B9E0009DF8080000EB4001C1EBC010FE4911F8C2
:10B9F0003000042809D09DF8080000EB4002C2EB9B
:10BA0000C01011F83000152801D1ADF818009DF8CC
:10BA10000800F54900EB4002C2EBC01001EBC0008A
:10BA200042789DF8080000EB4003C3EBC01011F80A
:10BA3000300042EA0020A0F58051303922D09DF834
:10BA4000080000EB4001C1EBC010E74901EBC0006A
:10BA500042789DF8080000EB4003C3EBC01011F8DA
:10BA6000300042EA0020A0F58052313A0CD09DF817
:10BA7000080000EB4002C2EBC01011F830000228B1
:10BA800004D019E0A62015E0A72013E09DF80800D7
:10BA900000EB4002C2EBC01001EBC00002799DF840
:10BAA000080000EB4003C3EBC01001EBC000C078FE
:10BAB00042EA0020ADF818009DF80800DFF82C835A
:10BAC00000EB001101EB002108EBC10101F5005171
:10BAD00091F816128DF820109DF808105F4608EBBB
:10BAE00001129DF82010114401F5805181F888BBA6
:10BAF00098F81800012810D19DF8080000EB4001CB
:10BB000001EB001108EB01109DF8201000EB011073
:10BB10002844017841F080010170BDF8180043F21B
:10BB20003002811A904272D009DC042870D01528A6
:10BB30006FD0A6280DD0A72844F0A98301E1B1F564
:10BB4000C06F67D0A1F5C06101397AD00429F3D163
:10BB5000FDE39DF8080000EB001101EB002008EB6D
:10BB6000C00000F50050414680F817729DF80800AB
:10BB700000EB001202EB002008EBC0029DF8200051
:10BB800000EB001002EBC00000F5005090F81C0222
:10BB9000032840D09DF8080000EB001202EB0020C3
:10BBA00001EBC0029DF8200000EB001002EBC0008A
:10BBB00000F5005090F81C02082843D09DF80800BA
:10BBC00000EB001202EB002001EBC0029DF8200008
:10BBD00000EB001002EBC00000F5005090F81C02D2
:10BBE0000D2844D09DF8080000EB001202EB002065
:10BBF00001EBC0029DF8200000EB001002EBC0003A
:10BC000000F5005090F82102A52845D055E028E124
:10BC100075E158E37DE39DF80800042200EB001372
:10BC200003EB002001EBC0039DF8200000EB0010A7
:10BC300003EBC00000F5005080F81C22A82203F09E
:10BC400038BFA9E39DF80800092200EB001303EBBD
:10BC5000002001EBC0039DF8200000EB001003EB77
:10BC6000C00000F5005080F81C22A922E7E79DF8EB
:10BC700008000E2200EB001303EB002001EBC003D1
:10BC80009DF8200000EB001003EBC00000F5005011
:10BC900080F81C22A222D2E79DF8080000EB4002A7
:10BCA00002EB00109DF8202001EB001000EB0210C9
:10BCB0002844027842F0040202709DF8080000EB6C
:10BCC000001202EB002001EBC0029DF8200000EB07
:10BCD000001002EBC00000F5005090F81E02A128F1
:10BCE00004F0D5829DF8080000EB001202EB002062
:10BCF00001EBC0029DF8200000EB001002EBC00039
:10BD000000F5005090F81E229DF8080000EB00138B
:10BD100003EB002001EBC0039DF8200000EB0010B6
:10BD200003EBC00000F5005080F821229DF80800C8
:10BD3000A12200EB001303EB002008EBC00102F08E
:10BD4000B2B99DF8080000EB001101EB002008EBF0
:10BD5000C00000F50050414680F817729DF80800B9
:10BD600000EB001202EB002008EBC0029DF820005F
:10BD700000EB001002EBC00000F5005090F81C0230
:10BD800005289DF8080000EB001202EB00200ED001
:10BD900001EBC0029DF8200000EB001002EBC00098
:10BDA00000F5005090F81C02092808D01AE001EBB9
:10BDB000C00000F5005080F81772062200E00A2249
:10BDC0009DF8080000EB001303EB002001EBC0031B
:10BDD0009DF8200000EB001003EBC00000F50050C0
:10BDE00080F81C2204E0000080640020A4120020DF
:10BDF0009DF8080000EB001202EB002001EBC002EE
:10BE00009DF8200000EB001002EBC00000F5005090
:10BE100090F82102A42822D19DF8080000EB4002EE
:10BE200002EB00109DF8202001EB001000EB021047
:10BE30002844027842F0200202709DF8080000EBCE
:10BE4000001202EB002001EBC0029DF8200000EB85
:10BE5000001002EBC00000F5005080F85972A122DA
:10BE6000EDE68DF8247014AAFE4913E09DF8080051
:10BE700000EB4003C3EBC0109DF8243001EBC00081
:10BE80001844C0789DF82430D0549DF82400401CFC
:10BE90008DF824009DF824000628E7D306211046DB
:10BEA00010F0CAF8CDE912071299000A401847EBC2
:10BEB00007014FF480720023FCF784F99DF8080015
:10BEC00000EB001101EB002008EBC0039DF82000FF
:10BED000414600EB001003EBC00000F5005080F875
:10BEE00020229DF8080000EB001202EB002008EB76
:10BEF000C00000F5005080F817724A462DE29DF808
:10BF0000080000EB001101EB002008EBC0029DF8D7
:10BF10002000414600EB001002EBC00000F500508D
:10BF200090F81C02062831D19DF8080000EB0012A1
:10BF300002EB002001EBC00000F5005080F8177202
:10BF40009DF80800072200EB001303EB002001EB33
:10BF5000C0039DF8200000EB001003EBC00000F5CB
:10BF6000005080F81C229DF80800A72200EB001367
:10BF700003EB002001EBC0039DF8200000EB001054
:10BF800003EBC00000F5005080F821229DF8080066
:10BF900000EB001202EB002001EBC0029DF8200034
:10BFA00000EB001002EBC00000F5005090F81C02FE
:10BFB00001289DF8080000EB001202EB002060D081
:10BFC00001EBC0029DF8200000EB001002EBC00066
:10BFD00000F5005090F81C0207289DF8080000EBBF
:10BFE000001202EB002054D001EBC0029DF82000AB
:10BFF00000EB001002EBC00000F5005090F81C02AE
:10C000000B289DF8080000EB001202EB00205DD029
:10C0100001EBC0029DF8200000EB001002EBC00015
:10C0200000F5005090F81C020C289DF8080000EB69
:10C03000001202EB002063D001EBC0029DF820004B
:10C0400000EB001002EBC00000F5005090F81C025D
:10C050000E285DD09DF8080000EB001200E0B3E070
:10C0600002EB002001EBC0029DF8200000EB001065
:10C0700002EBC00000F5005090F81C020F287CD0A5
:10C0800048E401EBC00000F5005080F8177202226E
:10C0900006E001EBC00000F5005080F8177208229E
:10C0A0009DF8080000EB001303EB002001EBC00338
:10C0B0009DF8200000E0FCE300EB001003EBC00063
:10C0C00000F5005080F81C22A322B8E501EBC00067
:10C0D00000F5005080F817729DF808000C2200EB64
:10C0E000001303EB002001EBC0039DF8200000EBE0
:10C0F000001003EBC00000F5005080F81C22AEE6F3
:10C1000001EBC00000F5005080F817720D22C7E760
:10C110009DF808000F2200EB001303EB002001EB59
:10C12000C0069DF8200000EB001006EBC00000F5F3
:10C13000005080F81C229DF80800A12200EB00139B
:10C1400003EB002001EBC0069DF8200000EB00107F
:10C1500006EBC00000F5005080F821229DF8080091
:10C1600000EB001303EB002001EBC0069DF820005C
:10C1700000EB001006EBC00000E039E000F50050D5
:10C1800080F81E229DF8080000EB400202EB001030
:10C190009DF8202001EB001000EB021028440278EB
:10C1A00042F0800202709DF8080000EB400202EBB2
:10C1B00000109DF8202001EB001000EB0210284435
:10C1C000027842F0040202709DF8080000EB400281
:10C1D00002EB00109DF8202001EB001000EB021094
:10C1E00000F5805090F8860D80073FF53BAB47E7A0
:10C1F0009DF8080000EB001202EB002001EBC002EA
:10C200009DF8200000EB001002EBC00000F500508C
:10C2100090F81E02A12836D09DF80800A32200EB5A
:10C22000001303EB002001EBC0039DF8200000EB9E
:10C23000001003EBC00000F5005080F821229DF8AB
:10C24000080000EB001202EB002001EBC0029DF899
:10C25000200000EB001002EBC00000F5005090F849
:10C260001E0201E080640020A228C0D09DF80800D2
:10C2700000EB001202EB002008EBC00000F50050BC
:10C2800080F81772FCE69DF80800A12200EB00136D
:10C2900003EB002001EBC0039DF8200000EB001031
:10C2A00003EBC00000F5005080F821229DF8080043
:10C2B00000EB001303EB002008EBC00000F500507A
:10C2C00080F81792DCE69DF80800A12200EB00112F
:10C2D00001EB002008EBC0039DF8200000EB0010EC
:10C2E00003EBC00000F5005080F81E229DF8080006
:10C2F00000EB001303EB002008EBC0039DF82000C7
:10C3000000EB001003EBC00000F5005080F8212284
:10C31000ACE79DF8080000EB001101EB002008EBF2
:10C32000C0029DF82000414600EB001002EBC00067
:10C3300000F5005090F81C020628A3D19DF80800D3
:10C3400000EB001202EB002001EBC00000E050E324
:10C3500000F5005080F8177207229DF8080000EBE6
:10C36000001303EB002001EBC0039DF8200000EB5D
:10C37000001003EBC00000F5005080F81C22A7223B
:10C380005DE49DF8200000EB001001EBC00000F51B
:10C39000005080F8212273E69DF80800464600EB25
:10C3A000001101EB002008EBC00000F5005080F800
:10C3B00017729DF80800A72100EB001202EB002085
:10C3C00008EBC0029DF8200000EB001002EBC0005B
:10C3D00000F5005080F821129DF80800DFF8688C05
:10C3E00000EB4001C1EBC01108EBC10040793028DF
:10C3F0009DF8080000EB400146D0C1EBC01008EBEF
:10C40000C0004146407931289DF808007DD000EBFE
:10C410004002C2EBC01001EBC000407933289DF808
:10C42000080073D000EB4002C2EBC01008EBC00064
:10C43000407934289DF8080000EB400101EB001022
:10C440009DF8201006EB001000EB01102844017845
:10C4500073D021F0010202709DF8080000EB40014A
:10C4600001EB00109DF8201006EB001000EB01100E
:10C470002844017821F0020202700020CDE900007A
:10C480008DF82470414617E201EB00109DF8201052
:10C4900006EB001000EB01102844017821F00101A7
:10C4A00001709DF8080000EB400101EB001006EB65
:10C4B00000119DF8200001EB00104119087820F0D0
:10C4C00002020A709DF8080000EB001101EB002049
:10C4D00006EBC0019DF8200000EB001001EBC0004E
:10C4E00000F5005090F81F023128C6D19DF80800D1
:10C4F00000EB400101EB00109DF8201006EB00104E
:10C5000000EB01102844017801E017E03DE121F043
:10C51000200101709DF8080000EB001101EB0020E4
:10C5200006EBC0019DF8200000EB001001EBC000FD
:10C5300000F5005080F859729FE771E100EB00119F
:10C5400001EB002006EBC0019DF8200000EB00107D
:10C5500001EBC00000F5005090F85A02F0B39DF8CE
:10C56000080000EB001101EB002006EBC0029DF873
:10C57000200000EB001002EBC00000F5005080F836
:10C5800059729DF8080000EB400101EB00109DF886
:10C59000201006EB001000EB01102844017821F078
:10C5A000010202709DF8080000EB400101EB001051
:10C5B0009DF8201006EB001000EB011028440178D4
:10C5C00021F00201017094F8A4070028B4D1707E14
:10C5D0000128B1D1B06D718B884200E0B1E0ABD2DF
:10C5E0009DF8080000EB001101EB002006EBC001F4
:10C5F0009DF8200000EB001001EBC00000F500509A
:10C6000090F85902012897D19DF8080000EB00111D
:10C6100001EB002006EBC0019DF8200000EB0010AC
:10C6200001EBC00000F5005090F893020028CDD136
:10C630009DF808004FF0104100EB001202EB0020C3
:10C6400006EBC0029DF8200000EB001002EBC000DA
:10C6500000F50050C0F824129DF8080000EB4001DE
:10C6600001EB001006EB00119DF8200001EB00101B
:10C6700000F5805090F8841D9DF8080000EB001232
:10C6800002EB002006EBC00000F5005080F8151208
:10C690009DF8080000EB001101EB002006EBC00143
:10C6A0009DF8200000EB001001EBC00000F50050E9
:10C6B00090F81C129DF8080000EB001202EB00201D
:10C6C00006EBC00000F5005090F8180281429AD1A4
:10C6D0009DF8080000EB001101EB002006EBC00103
:10C6E0009DF8200000EB001001EBC00000F50050A9
:10C6F00080F822729DF80800A42100EB001202EBE2
:10C70000002006EBC0029DF8200000EB001002EBB9
:10C71000C00000F5005080F81E129DF80800A3210B
:10C7200000EB001202EB002006EBC0029DF8200097
:10C7300000EB001002EBC00000F5005080F8211261
:10C740009BE69DF8080000EB001202EB002006EBD0
:10C75000C0039DF8200000EB001003EBC00000F5C3
:10C76000005080F859929DF8080000EB400101EB61
:10C7700000109DF8201006EB001000EB011028447B
:10C78000017841F0010101700CE700EB400101EB81
:10C7900000109DF8201006EB001000EB011028445B
:10C7A000017841F0010101709DF8080000EB4001A3
:10C7B00001EB00109DF8201006EB001000EB0110BB
:10C7C00000F5805090F8860D800715D49DF808007C
:10C7D00000EB400101EB001006EB00119DF820007A
:10C7E00001EB00102844017841F0020101709DF82E
:10C7F00008100220FCF7B2FF9DF80800A22100EB10
:10C80000001202EB002006EBC0029DF8200000EBB6
:10C81000001002EBC00000F5005080F81E122CE65C
:10C8200021F0200202709DF8080000EB400101EBAE
:10C8300000109DF8201006EB001000EB01102844BA
:10C84000017821F0020202709DF80800A92200EB95
:10C85000001101EB002006EBC0039DF8200000EB67
:10C86000001003EBC00000F5005080F81E2204E623
:10C87000DDE90002120142EA10720001CDE9000276
:10C880009DF8080000EB4002C2EBC0109DF8242088
:10C8900001EBC00010448079DDE9003C3038C2175C
:10C8A000184342EA0C02CDE900029DF82400401C26
:10C8B00000E0F8E38DF824009DF824000628D7D383
:10C8C0009DF80800009A00EB001303EB002006EB34
:10C8D000C0039DF8200000EB001003EBC00000F542
:10C8E0000050C0F835220023CDE900331A468DF8F8
:10C8F000247020E00098120142EA10720001CDE994
:10C9000000029DF8080000EB4002C2EBC0109DF849
:10C91000242001EBC0001044407BDDE9003C3038AE
:10C92000C217184342EA0C02CDE900029DF8240028
:10C93000401C8DF824009DF824000428DAD39DF8CB
:10C940000800009A00EB001303EB002006EBC00C7C
:10C950009DF8200000EB00100CEBC00000F500502B
:10C96000C0F850220020CDE900008DF8247020E0AE
:10C97000DDE90002120142EA10720001CDE9000275
:10C980009DF8080000EB4002C2EBC0109DF8242087
:10C9900001EBC0001044407CDDE900373038C2179D
:10C9A00018433A43CDE900029DF82400401C8DF85D
:10C9B00024009DF824000628DAD39DF80800009A88
:10C9C00000EB001303EB002006EBC0039DF82000F2
:10C9D00000EB001003EBC00000F50050C0F8392256
:10C9E0009DF8080000EB4002C2EBC01001EBC00054
:10C9F000F9E39DF80800464600EB001101EB00202A
:10CA000008EBC00000F5005080F817729DF8080090
:10CA100000EB001101EB002008EBC0019DF82000A5
:10CA200000EB001001EBC00000F5005090F81C0274
:10CA30000A2833D09DF8080000EB001101EB00201C
:10CA400006EBC0019DF8200000EB001001EBC000D8
:10CA500000F5005090F81C129DF8080000EB001241
:10CA600002EB002006EBC00000F5005090F8180221
:10CA7000814226D194F8A40720B39DF8080000EB6A
:10CA8000400101EB00109DF8201006EB001000EBB8
:10CA900001102844017841F0080193E09DF8080056
:10CAA0000B2100EB001202EB002006EBC0029DF808
:10CAB000200000EB001002EBC00000F5005080F8F1
:10CAC0001C1285E0C6F839709DF8080000EB0011D3
:10CAD00001EB002006EBC0019DF82000102200EBC6
:10CAE000001001EBC00142F23D2001440798FBF722
:10CAF000ACFB9DF8080000EB001101EB002006EBF9
:10CB0000C0019DF8200000EB001001EBC00000F216
:10CB1000352000F500500168C6F81D104068C6F8C1
:10CB200021009DF8080000EB400101EB001006EB2E
:10CB300000119DF8200001EB001000F5805090F8E6
:10CB4000840D30779DF8080000EB001101EB002008
:10CB500006EBC0019DF8200000EB001001EBC000C7
:10CB600000F50050D0F85002C6F82500049850F89F
:10CB7000691FC6F83D108088A6F84100B06D81B2EB
:10CB80000220FBF7E1FF00210620FCF7E7FDB06D76
:10CB9000718B884202D2B06D401CB0650021052027
:10CBA000FCF7DCFD9DF8080000EB400101EB0010F4
:10CBB0009DF8201006EB001000EB011028440178CE
:10CBC00021F0080101709DF808100220FCF7C6FD55
:10CBD0009DF80800A72200EB001101EB002006EBF6
:10CBE000C0039DF8200000EB001003EBC00000F52F
:10CBF000005080F821229DF80800A22200EB0011CD
:10CC000001EB002006EBC0039DF8200000EB0010B4
:10CC100003EBC00000F5005080F81E229DF80800CC
:10CC200000EB001101EB002006EBC0029DF8200094
:10CC300000EB001002EBC00000F5005080F85A72C3
:10CC40000020CDE9000002468DF82470FE4920E066
:10CC50000098120142EA10720001CDE900029DF82D
:10CC6000080000EB4002C2EBC0109DF8242001EB4D
:10CC7000C0001044C07ADDE9003C3038C2171843C8
:10CC800042EA0C02CDE900029DF82400401C8DF818
:10CC900024009DF824000A28DAD3DDE900239DF85A
:10CCA000080000EB001C0CEB002006EBC0089DF810
:10CCB000200000EB001008EBC00000F5005CCCF891
:10CCC0003D226046C0F841320020CDE90000024616
:10CCD0008DF824701FE00098120142EA10720001E2
:10CCE000CDE900029DF8080000EB4002C2EBC01045
:10CCF0009DF8242001EBC0001044407DDDE90037A1
:10CD00003038C21718433A43CDE900029DF8240099
:10CD1000401C8DF824009DF824000A28DBD30099DC
:10CD2000FEE39DF8080000EB4001C1EBC010C649CE
:10CD300011F83000042809D09DF8080000EB4002EB
:10CD4000C2EBC01011F83000152801D1ADF8180061
:10CD50009DF808000F4600EB4002C2EBC01001EB4B
:10CD6000C00042789DF8080000EB4003C3EBC01000
:10CD700011F8300042EA0020A0F58051303922D06D
:10CD80009DF8080000EB4001C1EBC01007EBC000AC
:10CD9000394642789DF8080000EB4003C3EBC01011
:10CDA00017F8300042EA0020A0F58052313A0CD04A
:10CDB0009DF8080000EB4002C2EBC01011F83000F3
:10CDC000022804D019E0A62015E0A72013E09DF862
:10CDD000080000EB4002C2EBC01001EBC00002797A
:10CDE0009DF8080000EB4003C3EBC01007EBC00048
:10CDF000C07842EA0020ADF818009DF80800934E74
:10CE000000EB001101EB002006EBC00000F5005024
:10CE100090F816028DF820009DF8081058469DF8ED
:10CE2000202006EB0111114401F5805181F888BBE7
:10CE3000317E012910D19DF8081001EB410202EB6F
:10CE400001119DF8202006EB011101EB021129448C
:10CE50000A7842F080020A70BDF81810A7297DD028
:10CE600007DC04297BD015297AD0A62943F00F824C
:10CE70003DE001F51D61B1F5804104D0112970D06C
:10CE80001229F3D1FEE39DF8081001EB011202EB29
:10CE9000012106EBC1029DF8201001EB011102EB0C
:10CEA000C10101F5005191F81C120029DED19DF855
:10CEB000081001EB011202EB012106EBC10101F5A3
:10CEC000005181F817029DF8080000EB001202EBF8
:10CED000002006EBC0029DF8200000EB001002EBE2
:10CEE000C00000F5005080F81C92A72120E19DF8B9
:10CEF000081001EB011202EB012106EBC10101F563
:10CF0000005181F817029DF8080000EB001101EBB9
:10CF1000002006EBC0019DF8200000EB001001EBA3
:10CF2000C00000F5005090F81C0202282DD09DF89A
:10CF3000080000EB001101EB002006EBC0019DF89A
:10CF4000200000EB001001EBC00000F5005090F84D
:10CF50001C0205282ED09DF8080003E0A4E0F1E0B3
:10CF600069E28EE200EB001101EB002006EBC0014C
:10CF70009DF8200000EB001001EBC00000F5005010
:10CF800090F82102A5282AD03AE09DF80800032154
:10CF900000EB001202EB002006EBC0029DF820001F
:10CFA00000EB001002EBC00000F5005080F81C12EE
:10CFB000A921BDE09DF80800062100EB001202EB5C
:10CFC000002006EBC0029DF8200000EB001002EBF1
:10CFD000C00000F5005080F81C12A221A8E09DF8C6
:10CFE000080000EB400101EB00109DF8201006EB5B
:10CFF000001000EB01102844017841F00401017099
:10D000009DF8080000EB001101EB002006EBC001C9
:10D010009DF8200000EB001001EBC00000F500506F
:10D0200090F81E02A12803F032819DF8080000EB61
:10D03000001101EB002006EBC0019DF8200000EB81
:10D04000001001EBC00003E080640020A412002067
:10D0500000F5005090F81E129DF8080000EB001239
:10D0600002EB002006EBC0029DF8200000EB001050
:10D0700002EBC00000F5005080F821129DF8080076
:10D08000A12100EB001202EB002006EBC0029DF88C
:10D09000200000EB001002EBC00000F5005080F80B
:10D0A0001E1203F0F4B84FE19DF8081001EB0112D5
:10D0B00002EB012106EBC1029DF8201001EB0111EA
:10D0C00002EBC10101F5005191F82112A42922D1EE
:10D0D0009DF8081001EB410202EB01119DF82020A0
:10D0E00006EB011101EB021129440A7842F02002FB
:10D0F0000A709DF8081001EB011202EB012106EB0A
:10D10000C1029DF8201001EB011102EBC10101F5F4
:10D11000005181F859029DF8081001EB011202EB51
:10D12000012106EBC10101F5005181F81702A1218F
:10D130009DF8080000EB001202EB002006EBC00295
:10D14000FEF70EBC9DF8081001EB011202EB012165
:10D1500006EBC1029DF8201001EB011102EBC101A9
:10D1600001F5005191F81C1201299DF8081001EBFE
:10D17000011202EB012137D006EBC1029DF820100D
:10D1800001EB011102EBC10101F5005191F81C12F4
:10D1900004299DF8081001EB011202EB01212BD0AC
:10D1A00006EBC1029DF8201001EB011102EBC10159
:10D1B00001F5005191F81C1206299DF8081001EBA9
:10D1C000011202EB012132D006EBC1029DF82010C2
:10D1D00001EB011102EBC10101F5005191F81C12A4
:10D1E00007297DD05DE7FCE306EBC10101F50051A5
:10D1F00081F81702022106E006EBC10101F500519A
:10D2000081F8170205219DF8080000EB001202EBDF
:10D21000002006EBC0029DF8200000EB001002EB9E
:10D22000C00000F5005080F81C12A32180E706EB37
:10D23000C10101F5005181F817029DF8080007228D
:10D2400000EB001101EB002006EBC0039DF820006D
:10D2500000EB001003EBC00000F5005080F81C222A
:10D260009DF80800A12200EB001101EB002006EB65
:10D27000C0039DF8200000EB001003EBC00000F598
:10D28000005080F821229DF8080000EB400101EBDE
:10D2900000109DF8201006EB001000EB0110284450
:10D2A000017841F0800202709DF8080000EB400117
:10D2B00001EB00109DF8201006EB001000EB0110B0
:10D2C0002844017841F0040202709DF8080000EB48
:10D2D000400101EB001006EB00109DF8201000E06B
:10D2E00041E000EB011000F5805090F8860D8007BA
:10D2F00042F1CD879DF8080000EB400101EB0010E2
:10D300009DF8201006EB001000EB01102844017876
:10D3100021F0020202709DF8080000EB400101EBD1
:10D3200000109DF8201006EB001000EB01102844BF
:10D33000017821F0200101709DF8080000EB400108
:10D3400001EB001006EB00109DF8201000EB01101F
:10D350002844017841F0080101709DF8081002206E
:10D36000FCF7FCF99DE69DF8081001EB011202EBB9
:10D37000012106EBC1029DF8201001EB011102EB27
:10D38000C10101F5005191F81E12A12933D09DF879
:10D390000810A32201EB011303EB012106EBC103EB
:10D3A0009DF8201001EB011103EBC10101F50051C3
:10D3B00081F821229DF8081001EB011202EB0121F6
:10D3C00006EBC1029DF8201001EB011102EBC10137
:10D3D00001F5005191F81E12A229C3D09DF8081042
:10D3E00001EB011202EB012106EBC10101F5005135
:10D3F00081F8170255E69DF80800A12100EB001204
:10D4000002EB002006EBC0029DF8200000EB0010AC
:10D4100002EBC00000F5005080F821129DF80800D2
:10D4200000EB001202EB002006EBC00000F50050FC
:10D4300080F8179235E69DF80810A12201EB011340
:10D4400003EB012106EBC1039DF8201001EB011154
:10D4500003EBC10101F5005181F821229DF808106C
:10D4600001EB011303EB012106EBC1039DF8201032
:10D4700001EB011103EBC10101F5005181F81E22FE
:10D48000ACE7804601469DF8080000EB001202EB75
:10D49000002006EBC00000F5005080F817129DF840
:10D4A0000800A72100EB001202EB002006EBC002EF
:10D4B0009DF8200000EB001002EBC00000F50050CA
:10D4C00080F821129DF8080000EB4001C1EBC0106C
:10D4D00007EBC000407930289DF8080000EB4001C0
:10D4E00053D0C1EBC01007EBC000407931289DF844
:10D4F00008007DD000EB4001C1EBC01007EBC0007D
:10D50000407933289DF8080000EB400171D0C1EB51
:10D51000C01007EBC000407934289DF8080000E0F7
:10D52000FEE300EB400165D0C1EBC01007EBC0008B
:10D530004079352871D09DF8080000EB400101EBDF
:10D5400000109DF8201006EB001000EB011028449D
:10D55000017821F0010202709DF8080000EB400103
:10D5600001EB00109DF8201006EB001000EB0110FD
:10D570002844017821F0020202700020CDE9000069
:10D58000014643468DF824800EE201EB00109DF821
:10D59000201006EB001000EB01102844017821F068
:10D5A000010101709DF8080000EB400101EB001043
:10D5B00006EB00119DF8200001EB001041190878DE
:10D5C00020F002020A709DF8080000EB001101EB48
:10D5D000002006EBC0019DF8200000EB001001EBDD
:10D5E000C00000F5005090F81F023128C5D102E0BC
:10D5F00014E03BE171E19DF8080000EB400101EB14
:10D6000000109DF8201006EB001000EB01102844DC
:10D61000017821F020010170AFE790E100EB0011EB
:10D6200001EB002006EBC0019DF8200000EB00108C
:10D6300001EBC00000F5005090F85A02F0B39DF8DD
:10D64000080000EB001202EB002006EBC0039DF87F
:10D65000200000EB001003EBC00000F5005080F844
:10D6600059829DF8080000EB400101EB00109DF885
:10D67000201006EB001000EB01102844017821F087
:10D68000010100E063E201709DF8080000EB400139
:10D6900001EB00109DF8201006EB001000EB0110CC
:10D6A0002844017821F00201017094F8A4070028B1
:10D6B000B2D1707E0128AFD1B06D00E0B3E0718BC4
:10D6C0008842A9D29DF8080000EB001101EB002070
:10D6D00006EBC0019DF8200000EB001001EBC0003C
:10D6E00000F5005090F85902012895D19DF80800E6
:10D6F00000EB001101EB002006EBC0019DF82000BB
:10D7000000EB001001EBC00000F5005090F8930210
:10D710000028CDD19DF808004FF0104100EB001219
:10D7200002EB002006EBC0029DF8200000EB001089
:10D7300002EBC00000F50050C0F824129DF808006C
:10D7400000EB400101EB001006EB00119DF82000FA
:10D7500001EB001000F5805090F8841D9DF8080042
:10D7600000EB001202EB002006EBC00000F50050B9
:10D7700080F815129DF8080000EB001101EB002065
:10D7800006EBC0019DF8200000EB001001EBC0008B
:10D7900000F5005090F81C129DF8080000EB0012F4
:10D7A00002EB002006EBC00000F5005090F81802D4
:10D7B00081429AD19DF8080000EB001202EB002094
:10D7C00006EBC0029DF8200000EB001002EBC00049
:10D7D00000F5005080F822829DF80800A42100EB9B
:10D7E000001202EB002006EBC0029DF8200000EBC7
:10D7F000001002EBC00000F5005080F81E129DF8EA
:10D800000800A32100EB001202EB002006EBC0028F
:10D810009DF8200000EB001002EBC00000F5005066
:10D8200080F82112A9E69DF8080000EB001202EB37
:10D83000002006EBC0039DF8200000EB001003EB76
:10D84000C00000F5005080F859929DF8080000EBE8
:10D85000400101EB00109DF8201006EB001000EBDA
:10D8600001102844017841F001010AE701EB0010A2
:10D870009DF8201006EB001000EB01102844017801
:10D8800041F0010101709DF8080000EB400101EB3F
:10D8900000109DF8201006EB001000EB011000F5C1
:10D8A000805090F8860D800715D49DF8080000EB95
:10D8B000400101EB00109DF8201006EB001000EB7A
:10D8C00001102844017841F0020101709DF8081010
:10D8D0000220FBF743FFA22132E001EB00109DF88C
:10D8E000201006EB001000EB01102844017821F015
:10D8F000200202709DF8080000EB400101EB0010CF
:10D900009DF8201006EB001000EB01102844017870
:10D9100021F0020202709DF80800A92200EB00111C
:10D9200001EB002006EBC0039DF8200000EB001087
:10D9300003EBC00000F5005080F81E221DE6A12177
:10D940009DF8080000EB001202EB002006EBC0027D
:10D950009DF8200000EB001002EBC00000F5005025
:10D9600080F81E1209E60098090141EA10710001D1
:10D97000CDE900019DF8080000EB4001C1EBC010AB
:10D980009DF8241007EBC00008448079DDE9002CE5
:10D990003038C117104341EA0C01CDE900019DF870
:10D9A0002400401C8DF824009DF824000828DAD3B8
:10D9B0009DF80800009900EB001202EB002006EB36
:10D9C000C00C9DF8200000EB00100CEBC00000F52F
:10D9D0000050C0F835120020CDE900008DF8243049
:10D9E00022E07EE0DDE90001090141EA1071000159
:10D9F000CDE900019DF8080000EB4001C1EBC0102B
:10DA00009DF8241007EBC0000844C07BDDE9002C22
:10DA10003038C117104341EA0C01CDE900019DF8EF
:10DA20002400401C8DF824009DF824000628D9D33A
:10DA30009DF80800009900EB001202EB002006EBB5
:10DA4000C00C9DF8200000EB00100CEBC00000F5AE
:10DA50000050C0F850120020CDE900008DF82430AD
:10DA600020E0DDE90001090141EA10710001CDE982
:10DA700000019DF8080000EB4001C1EBC0109DF8CB
:10DA8000241007EBC0000844407DDDE90023303856
:10DA9000C11710431943CDE900019DF82400401C33
:10DAA0008DF824009DF824000828DAD39DF808009A
:10DAB000009900EB001202EB002006EBC0029DF87B
:10DAC000200000EB001002EBC00000F50050C0F891
:10DAD00039129DF8080000EB4001C1EBC01007EBC4
:10DAE000C00041799DF8080000EB001202EB002015
:10DAF00006EBC0029DF8200000EB001002EBC00016
:10DB000000F5005080F81F129DF8080000EB40015E
:10DB100001EB001006EB00119DF8200001EB001056
:10DB200000F5805090F8861D9DF8080000EB00126B
:10DB300002EB002006EBC0029DF8200000EB001075
:10DB400002EBC00000F5005080F834120AE4804671
:10DB500001469DF8080000EB001202EB002006EBE6
:10DB6000C00000F5005080F817129DF8080000EB87
:10DB7000001101EB002006EBC0019DF8200000EB36
:10DB8000001001EBC00000F5005090F81C020328C3
:10DB900033D09DF8080000EB001101EB002006EBEC
:10DBA000C0019DF8200000EB001001EBC00000F563
:10DBB000005090F81C129DF8080000EB001202EBD8
:10DBC000002006EBC00000F5005090F818028142DA
:10DBD00026D194F8A40720B39DF8080000EB40017B
:10DBE00001EB00109DF8201006EB001000EB011077
:10DBF0002844017841F0080195E09DF808000421CF
:10DC000000EB001202EB002006EBC0029DF82000A2
:10DC100000EB001002EBC00000F5005080F81C1271
:10DC200087E0C6F839809DF8080000EB001101EB91
:10DC3000002006EBC0019DF82000102200EB001030
:10DC400001EBC00142F23D2001440798FAF7FDFACA
:10DC50009DF8080000EB001101EB002006EBC0016D
:10DC60009DF8200000EB001001EBC00000F2352011
:10DC700000F500500168C6F81D104068C6F8210084
:10DC80009DF8080000EB400101EB001006EB0011CD
:10DC90009DF8200001EB001000F5805090F8840DF5
:10DCA00030779DF8080000EB001101EB002006EB37
:10DCB000C0019DF8200000EB001001EBC00000F552
:10DCC0000050D0F85002C6F82500049850F8691F9B
:10DCD000C6F83D108088A6F84100B06D81B20220E0
:10DCE000FAF732FF00210620FBF738FDB06D718B8B
:10DCF000884202D2B06D401CB06500210520FBF7C0
:10DD00002DFD9DF8080000EB400101EB00109DF88F
:10DD1000201006EB001000EB01102844017800E011
:10DD2000B1E021F0080101709DF808100220FBF716
:10DD300015FD9DF80800424600EB001101EB0020A4
:10DD400006EBC0019DF8200000EB001001EBC000C5
:10DD500000F5005080F85A829DF80800A72100EBDA
:10DD6000001303EB002006EBC0039DF8200000EB3E
:10DD7000001003EBC00000F5005080F821129DF860
:10DD80000800A22100EB001303EB002006EBC00308
:10DD90009DF8200000EB001003EBC00000F50050E0
:10DDA00080F81E120021CDE900118DF8242039469B
:10DDB00021E0DDE900031B0143EA10730001CDE916
:10DDC00000039DF8080000EB4003C3EBC0109DF872
:10DDD000243001EBC0001844C07ADDE9007C303803
:10DDE000C317384343EA0C03CDE900039DF8240030
:10DDF000401C8DF824009DF824000C28D9D3DDE9BF
:10DE000000379DF8080000EB001C0CEB002006EB2F
:10DE1000C0089DF8200000EB001008EBC00000F5E2
:10DE2000005CCCF83D326046C0F841720020CDE97C
:10DE300000008DF8242020E0DDE90002120142EA12
:10DE400010720001CDE900029DF8080000EB4002CD
:10DE5000C2EBC0109DF8242001EBC0001044C07D2F
:10DE6000DDE900373038C21718433A43CDE90002E4
:10DE70009DF82400401C8DF824009DF824000C28F7
:10DE8000DAD3DDE900129DF8080000EB001303EB84
:10DE9000002006EBC0039DF8200000EB001003EB10
:10DEA000C00000F50053C3F845121846C0F84922D7
:10DEB0004CE6FF499DF808005A469DF8203001EBDA
:10DEC0000010184400F5805080F888BB9DF80800C9
:10DED00000EB4003C3EBC010F64B03EBC0004078EF
:10DEE00070280AD19DF8080000EB4006C6EBC01070
:10DEF00003EBC0008078FA2858D09DF8080000EBAA
:10DF00004006C6EBC01003EBC00040780C26B6EB11
:10DF1000101F0AD19DF8080000EB4006C6EBC010A8
:10DF200003EBC0008078FA2842D09DF8080000EB8F
:10DF30004006C6EBC01013F830600520B0EB161F8A
:10DF400017D19DF8080000EB4006C6EBC01003EBAC
:10DF5000C00046780320B0EB161F0AD19DF80800D8
:10DF600000EB4006C6EBC01003EBC0008078ADF8B4
:10DF700018009DF8080000EB001606EB002001EBEE
:10DF8000C00000F5005090F816628DF820609DF8F2
:10DF9000080001EB00169DF82000304400F5805089
:10DFA00080F8882B087E012804D014E0B120DEE739
:10DFB000B620DCE79DF8080000EB400606EB0010F9
:10DFC0009DF8206001EB001000EB06102844067855
:10DFD00046F080060670BDF81800012803D06528B9
:10DFE00042F055816AE09DF8080000EB4006C6EB60
:10DFF000C01003EBC0000079012802F0488102281C
:10E00000FBD00328F9D00528EAD19DF8080000EBE1
:10E01000001303EB002001EBC0039DF8200000EB90
:10E02000001003EBC00000F5005090F81C0200281F
:10E03000D6D19DF8080000EB001303EB002001EBA4
:10E04000C00000F5005080F817229DF8080000EB92
:10E05000001303EB002001EBC0039DF8200000EB50
:10E06000001003EBC00000F5005080F81C929DF8F2
:10E070000800B62200EB001303EB002001EBC00305
:10E080009DF8200000EB001003EBC00000F50050ED
:10E0900080F821229DF80800B22200EB001303EB68
:10E0A000002001EBC0019DF8200000EB001001EB07
:10E0B000C00000F5005080F81E2247E59DF80800DA
:10E0C00000EB4006C6EBC01003EBC000007900096E
:10E0D00012D0B920ADF818009DF8080000EB4006FA
:10E0E000C6EBC01003EBC000007900F00F008DF804
:10E0F00014008DF8242021E0B820EBE79DF80800FB
:10E1000000EB400606EB00109DF8246001EB0010C8
:10E1100000EB061000F5805090F8856D9DF8080022
:10E1200000EB4007C7EBC01013F8300050388642B0
:10E1300014D09DF82400401C8DF824009DF80800A0
:10E1400000EB400606EB001001EB001000F58050DC
:10E1500090F85B0D9DF82460B042CFD89DF8240064
:10E160009DF8143018448DF820009DF8080000EB4D
:10E17000001303EB002001EBC0039DF8200000EB2F
:10E18000001003EBC00000F5005090F81C020128BD
:10E1900013D09DF8080000EB001303EB002001EB07
:10E1A000C0039DF8200000EB001003EBC00000F559
:10E1B000005090F81C02012879D19DF8080000EB6E
:10E1C000001303EB002001EBC00000F5005080F8C5
:10E1D00017229DF80800022200EB001303EB002039
:10E1E00001EBC0039DF8200000EB001003EBC00022
:10E1F00000F5005080F81C22B922EFE39DF80800DA
:10E2000000EB400101EB0011294800EB011000F583
:10E21000805090F8600D20B101286FD00228CBD13A
:10E2200083E2234E9DF8080006EB400000F5804095
:10E23000B0F83404801F81B29DF80800DFF87480C4
:10E2400000EB4002C2EBC01208EBC200401CFBF71F
:10E2500005F8CDE9120B9DF808005F4606EB40007B
:10E2600000F58040B0F834149DF80800414400EBFC
:10E270004002C2EBC0106FF0040202EBC000084481
:10E28000042109F0F3FFDDE91223C117CDE90001F4
:10E290005040594008438FD19DF8080006EB00100C
:10E2A00000F5805080F8887B9DF8080004E0E8E2E3
:10E2B000A41200208064002000EB4001C1EBC011DB
:10E2C00008EBC1000079ADF81800BDF8180031283E
:10E2D000A5D19DF8080006EB400000F58040B0F89D
:10E2E00034044121183890FBF1F0C117CDE9000149
:10E2F00084F884058DF82470BB46C6E0CFE09DF815
:10E300000800474600EB4001C1EBC01008EBC0011C
:10E310009DF8240000EB80100844017D9DF8240046
:10E32000304400F5805080F885159DF8080000EB1A
:10E330004001C1EBC01008EBC0019DF8240000EBC8
:10E340008010084408211A3009F05CFF8DED0D0A99
:10E3500010EE100A9DF8241006EB011101F5805112
:10E36000C1F895059DF8080000EB4001C1EBC01015
:10E3700007EBC0019DF8240000EB80100844082141
:10E38000323009F03FFF8DED0D0A10EE100A9DF8B6
:10E39000241006EB011101F58051C1F891059DF89B
:10E3A000080000EB4001C1EBC01007EBC0019DF875
:10E3B000240000EB8010084408213A3009F022FFC5
:10E3C0008DED0D0A10EE100A9DF8241006EB0111D8
:10E3D00001F58051C1F899059DF8080000EB400156
:10E3E000C1EBC01007EBC0019DF8240000EB8010CA
:10E3F00008440821423009F005FF8DED0D0A10EEAA
:10E40000101A9DF8240006EB001000F58050C0F8AB
:10E410009D159DF8080000EB400101EB00109DF8F0
:10E42000241006EB001000EB01102844017841F0A5
:10E43000800101709DF8080006EB400000F5804067
:10E44000B0F83404C1199DF8080000EB4002C2EB9B
:10E45000C0104FF0FF3202EBC000095C9DF80800CD
:10E4600000EB001202EB002006EBC0039DF8200039
:10E4700000EB001003EBC00000F5005080F85812CC
:10E480009DF82400401C8DF824009DF82410DDE93F
:10E490000023891A7BEB0300FFF631AF08E59DF8F6
:10E4A000080000EB4001C1EBC010FE4E06EBC000BF
:10E4B000417D9DF8080000EB4002C2EBC01006EB66
:10E4C000C000807D41EA0020C117CDE900019DF820
:10E4D000080000EB4001C1EBC01006EBC0001521A5
:10E4E000FAF7A6FECDE9120BDDE90001129F5A46AC
:10E4F000784051400843D1D19DF8080000EB40011D
:10E50000C1EBC01016F83010491E8DF82010DFF84E
:10E5100098839DF80800414608EB00139DF8200001
:10E52000184400F5805080F8882B9DF82000404466
:10E5300000F5805080F885259DF8200008EB00103C
:10E5400000F58050C0F895259DF8080000EB4002CA
:10E55000C2EBC01006EBC00082799DF8080000EB0A
:10E560004003C3EBC01006EBC000407942EA002034
:10E5700000EE100AF8EE400A9FEDCC0A9DF8080064
:10E5800080EE801A00EB4002C2EBC01006EBC00028
:10E5900002799DF8080000EB4003C3EBC01006EBC6
:10E5A000C000C07842EA002000EE900A9DF82000EA
:10E5B000F8EE600A71EE200A10EE902A01EB0010CE
:10E5C00000F58050C0F891259DF8080000EB40024E
:10E5D000C2EBC01006EBC000827A9DF8080000EB89
:10E5E0004003C3EBC01006EBC000407A42EA0020B3
:10E5F00000EE900A9DF80800B8EE601AC1EE000A1D
:10E6000000EB4002C2EBC01006EBC000027A9DF89E
:10E61000080000EB4003C3EBC01006EBC000C0795C
:10E6200042EA002000EE100A9DF82000B8EE400AF1
:10E6300030EE800A10EE102A01EB001000F5805039
:10E64000C0F899259DF8080000EB4001C1EBC0100F
:10E6500006EBC000C07A00069DF8080000EB400100
:10E66000C1EBC01006EBC000017B9DF8080000EB79
:10E670004002C2EBC01006EBC000C07A41EA0020A5
:10E680000AD400EE100AB8EE400ADFED890A20EE47
:10E69000200A10EE100A0BE0404280B2F9F7A2FF08
:10E6A0009FED841B53EC112BF9F7AAFEF9F7FFFF3E
:10E6B0009DF8202008EB021101F58051C1F89D055D
:10E6C0009DF808009DF8202000EB400101EB0010B0
:10E6D00008EB001000EB02102844027842F08002A0
:10E6E00002709DF8080000EB4002C2EBC01006EB80
:10E6F000C000C27D9DF8080000EB001303EB002072
:10E7000008EBC0039DF8200000EB001003EBC000F5
:10E7100000F5005080F858229DF8080000EB4002F8
:10E7200002EB001008EB0010E0E09DF80800DFF8B5
:10E73000748100EB4001C1EBC01008EBC000C3794D
:10E740009DF8080000EB4002C2EBC01008EBC000CF
:10E75000007A43EA0020C317CDE900039DF80800C2
:10E76000072100EB4002C2EBC01008EBC000FAF733
:10E770005FFDCDE9120BDDE90001129B5E465840BA
:10E78000714008437DD19DF8080000EB4001C1EBCA
:10E79000C01118F83100401E8DF82000424F9DF83E
:10E7A000081007EB011000F5805080F8886B9DF889
:10E7B0002010781800F5805080F885659DF80800D5
:10E7C00000EB4001C1EBC01108EBC1008079F9F703
:10E7D00009FF41EC110B9FED390B0CF0D1FA9DF8BC
:10E7E0000800B0EE408AF0EE608A00EB4001C1EB19
:10E7F000C01108EBC10002799DF8080000EB400150
:10E80000C1EBC01108EBC100C07842EA0020F9F763
:10E81000E9FE53EC182BF9F765FEF9F748FF9DF870
:10E82000201007EB011101F58051C1F895059DF805
:10E83000201007EB011000F58050C0F891659DF89D
:10E84000201007EB011000F58050C0F899659DF885
:10E85000201007EB011000F58050C0F89D659DF871
:10E86000080000EB400101EB001107EB01109DF8DF
:10E87000201000EB01102844017841F08002027062
:10E8800000E097E29DF8080000EB4001C1EBC011E9
:10E8900008EBC100427A9DF8080000EB001101EB83
:10E8A00000210FE080640020A412002000FF7F47B9
:10E8B0000000803D000000000000B0BF000000002C
:10E8C000000024409DF8200007EBC10300EB00107E
:10E8D00003EBC00000F5005080F858229DF80800B6
:10E8E00000EB400101EB001107EB011000F5805037
:10E8F00090F85B0D84F88405D0E59DF80800FD4E86
:10E9000000EB4001C1EBC01006EBC000C1789DF8E0
:10E91000080000EB4002C2EBC01006EBC00080789C
:10E9200041EA00208DF80C009DF8080000EB400142
:10E93000C1EBC0109DF80C1006EBC00008444178F4
:10E940009DF8080000EB4002C2EBC0109DF80C20BF
:10E9500006EBC000805C41EA0020C117CDE9000150
:10E960009DF8080000EB4001C1EBC01006EBC000B1
:10E970009DF80C10FAF75CFCCDE9120BDDE9000103
:10E98000129F5A46784051400843B5D19DF808007F
:10E9900000EB4001C1EBC01006EBC00040788DF8E1
:10E9A00020008DF82420D4491CE09DF8080000EBDD
:10E9B000400303EB00109DF8243001EB001000EB46
:10E9C000031000F5805090F8850D9DF82030984296
:10E9D0009DF8240003D18DF8200013E07FE1401C56
:10E9E0008DF824009DF8080000EB400303EB0010B5
:10E9F00001EB001000F5805090F85B0D9DF824307D
:10EA00009842D2D89DF8080000EB400303EB0010B9
:10EA100001EB00139DF8200003EB00104319187858
:10EA200040F080071F709DF8080000EB4003C3EB27
:10EA3000C01006EBC0000379ADF818309DF808004F
:10EA400001EB00139DF82000184400F5805080F879
:10EA5000882BBDF81800F32806D006DC05287DD0E9
:10EA6000F12807D0F22890D14DE2F42877D0F6288B
:10EA70008BD14AE29DF8080000EB001303EB002065
:10EA800001EBC0039DF8200000EB001003EBC00079
:10EA900000F5005090F81C0230B39DF8080000EB20
:10EAA000400303EB00109DF8203001EB001000EB59
:10EAB000031000F5805090F88D0DC00713D09DF81D
:10EAC000080000EB001303EB00239DF8200001EB8E
:10EAD000C30300EB001003EBC00000F5005090F8FA
:10EAE000A202C00726D0BAE09DF8080000EB00178C
:10EAF00007EB002001EBC0079DF8200000EB0010A1
:10EB000007EBC00000F5005080F81C929DF808004B
:10EB1000F42300EB001707EB002001EBC0079DF882
:10EB2000200000EB001007EBC00000F5005080F85B
:10EB3000213294E09DF8080000EB001303EB002065
:10EB400001EBC0039DF8200000EB001003EBC000B8
:10EB500000F5005090F89402C0B301E04FE2E8E104
:10EB60008DF824202AE09DF8080000EB001303EB49
:10EB7000002001EBC0039DF8200000EB001003EB28
:10EB8000C0039DF82400184400F5005090F8953219
:10EB90009DF8080000EB400707EB001001EB0017A1
:10EBA0009DF82400384400F5805090F8620D8342AF
:10EBB00008D19DF82400401C8DF824009DF8240005
:10EBC0000428D0D39DF82400042829D047E09DF8DC
:10EBD000080000EB001303EB002001EBC0039DF8DD
:10EBE000200000EB001003EBC0039DF82400184444
:10EBF00000F5005090F895329DF8080000EB4007B2
:10EC000007EB001001EB00179DF82400384400F5D5
:10EC1000805090F8620D834208D19DF82400401C7A
:10EC20008DF824009DF824000A28D0D39DF82400F4
:10EC30000A2814D09DF8080000EB001303EB002015
:10EC400001EBC0079DF8200042F2A22300EB001068
:10EC500007EBC0001844037843F0010707709DF8E4
:10EC60000C0011284AD09DF80C0014289DF80800CB
:10EC700000EB400303EB00107ED001EB00139DF886
:10EC8000200003EB00102844037823F004030370F2
:10EC90009DF8080000EB001303EB002001EBC0031C
:10ECA0009DF8200000EB001003EBC00000F50050C1
:10ECB00090F8A202C0077DD09DF8080000EB001379
:10ECC00003EB002001EBC0039DF8200000EB0010D7
:10ECD00003EBC00000F50050A0F8A02205229DF82B
:10ECE000080000EB001303EB002001EBC001FDF76F
:10ECF00048BB000080640020A41200209DF808009A
:10ED000000EB400303EB00109DF8203001EB0010F6
:10ED100000EB03102844037843F0040303708DF8DC
:10ED2000242025E09DF8080000EB4003C3EBC01051
:10ED30009DF8243006EBC000184443799DF8080084
:10ED400000EB001707EB002001EBC0079DF8200047
:10ED500000EB001007EBC0009DF82470384400F56C
:10ED6000005080F85B329DF82400401C8DF8240090
:10ED70009DF824000A2800E030E0D3D38DF8242049
:10ED800027E09DF8080000EB4002C2EBC0109DF8A0
:10ED9000242006EBC0001044C27B9DF8080000EB65
:10EDA000001303EB002001EBC0039DF8200000EBF3
:10EDB000001000E084E203EBC0009DF8243018440A
:10EDC00000F5005080F874229DF82400401C8DF856
:10EDD00024009DF824000228D3D38DE59DF820302F
:10EDE00001EB001000EB03102844037843F0040308
:10EDF00003708DF8242025E09DF8080000EB400307
:10EE0000C3EBC0109DF8243006EBC00018444379D2
:10EE10009DF8080000EB001707EB002001EBC0078E
:10EE20009DF8200000EB001007EBC0009DF8247057
:10EE3000384400F5005080F85B329DF82400401CF7
:10EE40008DF824009DF824000A28D5D38DF82420BD
:10EE50001AE0C27B9DF8080000EB001303EB0020D2
:10EE600001EBC0039DF8200000EB001003EBC00095
:10EE70009DF82430184400F5005080F874229DF865
:10EE80002400401C8DF824009DF8240002289DF8E1
:10EE9000080000EB4002C2EBC0109DF8242006EBF6
:10EEA000C0001044D5D3407C02049DF8080000EB5C
:10EEB0004003C3EBC0109DF8243006EBC00018449B
:10EEC000807C42EA00229DF8080000EB4003C3EB7F
:10EED000C0109DF8243006EBC0001844C07C0243EB
:10EEE0009DF8080000EB001303EB002001EBC001CC
:10EEF0009DF8200000EB001001EBC00000F5005071
:10EF0000C0F88822DCE1F122E9E69DF8080003223E
:10EF100000EB001303EB002001EBC0039DF8200081
:10EF200000EB001003EBC00000F5005080F81C223D
:10EF3000E9E79DF80800022300EB001707EB00202B
:10EF400001EBC0079DF8200000EB001007EBC000AC
:10EF500000F5005080F81C329DF80800F62300EB05
:10EF6000001707EB002001EBC0079DF8200000EB25
:10EF7000001007EBC00000F5005080F821329DF82A
:10EF8000080000EB001707EB002001EBC0079DF81D
:10EF9000200000EB001007EBC00000F5005080F8E7
:10EFA00094928DF8242025E09DF8080000EB4002A3
:10EFB000C2EBC0109DF8242006EBC000104442793B
:10EFC0009DF8080000EB001303EB002001EBC003E9
:10EFD0009DF8200000EB001003EBC0009DF82430EA
:10EFE000184400F5005080F895229DF82400401C3C
:10EFF0008DF824009DF824000A28D5D360E19DF8FF
:10F00000080000EB4002C2EBC01006EBC0008279A2
:10F010009DF8080000EB4003C3EBC01006EBC000F6
:10F02000407942EA00229DF8080000EB001303EB50
:10F03000002001EBC0039DF8200000EB001003EB63
:10F04000C00000F50050A0F8A0229DF8080000EBD9
:10F05000001202EB002001EBC0029DF8200000EB43
:10F06000001002EBC00000F50050B0F8A0229DF89F
:10F07000080000EB400303EB001001EB001000F56B
:10F080008050B0F86E0D8242B8D39DF80800F1228E
:10F0900000EB001303EB002001EBC0039DF8200000
:10F0A00000EB001003EBC00000F5005080F82122B7
:10F0B0009DF8080000EB001202EB002001EBC001FC
:10F0C0009DF8200000EB001001EBC00042F2A221ED
:10F0D0000844017821F00101FCF77EB89DF8080092
:10F0E00000EB4001C1EBC010FE4F07EBC000007900
:10F0F0008DF820008DF82CB0FB4E1BE09DF8080029
:10F1000000EB400101EB00109DF82C1006EB001005
:10F1100000EB011000F5805090F8850D9DF820104F
:10F1200088429DF82C0002D18DF8200012E0401C8E
:10F130008DF82C009DF8080000EB400101EB001059
:10F1400006EB001000F5805090F85B0D9DF82C1038
:10F150008842D3D89DF8080000EB4001C1EBC010F5
:10F1600007EBC000C078ADF81800BDF818001728EC
:10F170000FD2DFE800F00E6B6B0E6F6F6F696B0ED6
:10F180000E0E0E0E0E6D6F6F0E0E717173008DF8F8
:10F190000C009DF80C00001FC1B29DF8080000EBA8
:10F1A0004002C2EBC01007EBC000C01CF9F76EFEB6
:10F1B0008DF828009DF8080000EB4001C1EBC0105D
:10F1C0009DF80C1007EBC000084410F8010C9DF8E6
:10F1D0002810884274D19DF8080000EB4001C1EB73
:10F1E000C01007EBC0004078002869D09DF80800E7
:10F1F00000EB4001C1EBC011BA4800EBC1019DF822
:10F200000C000A5C9DF80800B04600EB001101EB11
:10F21000002006EBC0039DF8200000EB001003EB7C
:10F22000C00000F5005080F858229DF8080006EB59
:10F2300000139DF82000184400F5805080F888BB2A
:10F24000307E01280CD01CE01220A0E707209EE7AA
:10F2500009209CE706209AE70B2098E72A2096E7EA
:10F260009DF8080000EB400101EB001108EB0110D4
:10F270009DF8201000EB01102844017841F0800136
:10F280000170BDF8180007287ED007DC072817D2C8
:10F29000DFE800F016FDFC16FBFAF900103807282D
:10F2A000F5D2DFE800F0F2F20D0D0404F500BDF830
:10F2B0001800142805D0BDF81800152865D01FE1E6
:10F2C000C2E39DF8080000EB4001C1EBC010854986
:10F2D00001EBC000027A9DF8080000EB4003C3EB8D
:10F2E000C01001EBC000407942EA00629DF80800BE
:10F2F00000EB4003C3EBC01001EBC00080790304B6
:10F300009DF8080000EB4006C6EBC01001EBC00002
:10F31000C07943EA002002439DF8080000EB001189
:10F3200001EB00219DF8200008EBC10100EB00106B
:10F3300001EBC00000F50050C0F835229DF8080030
:10F3400000EB001101EB00219DF8200008EBC1014A
:10F3500000EB001001EBC00000F50050D0F83502C2
:10F36000002102F0DDFBCDE900019DF8080000EB73
:10F37000400101EB001108EB011000F5805090F8FE
:10F38000700D00F0030101E0FEE36BE09DF8080062
:10F3900000EB400202EB001208EB021000F5805077
:10F3A00090F8700DC0F3011001449DF8080000EBC7
:10F3B000400202EB001208EB021000F5805090F8BA
:10F3C000700DC0F38100081AF9F7FBF841EC110B3E
:10F3D0009FED460B0BF0D4FC51EC100BF9F742F902
:10F3E000CDE912019DF8080000EB001101EB0021AE
:10F3F0009DF8200008EBC10100EB001001EBC000FC
:10F4000000F50050D0F85002002102F089FBDDE940
:10F410000023A0FB026701FB027100FB0317DDE97B
:10F42000120102220023F8F7CDFEDDE91223301885
:10F430007941F8F7C7FECDE9000103F021F89DF806
:10F44000081001EB011202EB01229DF8201008EBDD
:10F45000C20201EB011102EBC10101F50051C1F83B
:10F4600039024DE09DF8080000EB4001C1EBC010EF
:10F470001C4901EBC000027A9DF8080000EB400334
:10F48000C3EBC01005E0FDE31DE3FCE35AE34BE3EF
:10F490008AE301EBC000407942EA00629DF808006F
:10F4A00000EB4003C3EBC01001EBC0008079030404
:10F4B0009DF8080000EB4006C6EBC01001EBC00051
:10F4C000C07943EA002002439DF8080000EB0011D8
:10F4D00001EB00219DF8200008EBC10100EB0010BA
:10F4E00008E0000080640020A4120020000000005A
:10F4F0000000244001EBC00000F50050C0F83922A4
:10F500009DF8080000EB4001C1EBC011FE4800EB84
:10F51000C100407A84F8E3019DF80800464600EBFC
:10F52000400101EB00109DF8201008EB001000EBEB
:10F53000011094F8E3112844CA09017862F300012C
:10F54000017094F8E30100F0030001287CD094F8E6
:10F55000E301C043800777D09DF8080000EB40012D
:10F5600001EB00109DF8201006EB001000EB0110DD
:10F570002844017821F0020101709DF8080000EB99
:10F58000400101EB00109DF8201006EB001000EB8D
:10F59000011000F5805090F8860DC0F340019DF8F1
:10F5A000080000EB001202EB002006EBC0029DF801
:10F5B000200000EB001002EBC00000F5005090F8B6
:10F5C0003402C0F34000814272D09DF8080000EB85
:10F5D000001101EB002006EBC0019DF8200000EBBC
:10F5E000001001EBC00042F2342101449DF80800F4
:10F5F00000EB400202EB00109DF8202006EB00100B
:10F6000000EB021000F5805090F8860D4208087853
:10F6100062F3410008709DF8080000EB400101EB27
:10F62000001006EB00119DF8200001EB001000F522
:10F63000805090F8860D800717D59DF8081002209D
:10F64000FAF78CF834E0FFE79DF8080000EB400182
:10F6500001EB00109DF8201006EB001000EB0110EC
:10F660002844017841F0020186E79DF808009DF8E2
:10F67000202000EB400101EB001008EB001000EB34
:10F6800002102844027822F0200202709DF808003F
:10F6900000EB001303EB002006EBC0019DF82000F7
:10F6A00000EB001001EBC00000F5005080F85A920A
:10F6B0009DF808009DF8202000EB400101EB0010B0
:10F6C000B04606EB001000EB021000F5805090F8F9
:10F6D000860D00F001029DF8080000EB001303EB1B
:10F6E000002006EBC0019DF8200000EB001001EBAC
:10F6F000C00000F5005090F8340200F00100824292
:10F7000070D09DF80800464600EB001101EB002088
:10F7100008EBC0019DF8200000EB001001EBC000D9
:10F7200042F2342101449DF8080000EB400202EB54
:10F7300000109DF8202008EB001000EB021000F5EF
:10F74000805090F8860D0A7860F300020A709DF8E8
:10F75000080000EB400101EB00109DF8201006EBC3
:10F76000001000EB011000F5805090F8860DC007E6
:10F770009DF8080037D000EB001101EB002006EBEC
:10F78000C0019DF8200000EB001001EBC00000F567
:10F79000005090F85A02E0B39DF8080000EB001208
:10F7A00002EB002006EBC0029DF8200000EB0010E9
:10F7B00002EBC00000F5005080F859B29DF8080037
:10F7C00000EB400101EB00109DF8201006EB00104B
:10F7D00000EB01102844017821F00101017094F838
:10F7E000A407B8B3F0E000EB400101EB00109DF876
:10F7F000201006EB001000EB01102844017821F0E6
:10F80000200101709DF8080000EB001202EB0020BF
:10F8100000E00CE008EBC0029DF8200000EB0010B7
:10F8200002EBC00000F5005080F859B2CCE09DF822
:10F83000080000EB001202EB002006EBC0029DF86E
:10F84000200000EB001002EBC00000F5005080F833
:10F850005992C4E7FFE7707E012854D1B06D718BD7
:10F86000884250D29DF8080000EB001101EB002007
:10F8700006EBC0019DF8200000EB001001EBC0007A
:10F8800000F5005090F8590201283CD19DF808007D
:10F8900000EB001101EB002006EBC0019DF82000F9
:10F8A00000EB001001EBC00000F5005090F893024F
:10F8B00048BB9DF8080000EB400101EB001006EB8F
:10F8C00000119DF8200001EB001000F5805090F829
:10F8D000841D9DF8080000EB001202EB002006EBEF
:10F8E000C00000F5005080F815129DF808000521B1
:10F8F00000EB001202EB002006EBC0029DF8200096
:10F9000000EB001002E05FE08064002002EBC0002A
:10F9100000F5005080F821129DF808005F4600EBCA
:10F92000400101EB001006EB00119DF8200001EBF7
:10F93000001000F58050C0F888BD9DF80810022026
:10F94000F9F70CFF8DF8247019E09DF8080000EB22
:10F95000001101EB002006EBC0019DF8200000EB38
:10F96000001001EBC0009DF82410084400F5005081
:10F9700080F85B729DF82400401C8DF824009DF8EF
:10F9800024001428E1D38DF8247019E09DF80800B4
:10F9900000EB001101EB002006EBC0019DF82000F8
:10F9A00000EB001001EBC0009DF82410084400F5A6
:10F9B000005080F877729DF82400401C8DF82400D8
:10F9C0009DF824000A28E1D394F8E301800612D5BB
:10F9D0009DF80800162100EB001202EB00229DF8B2
:10F9E000200008EBC20200EB001002EBC00000F5A3
:10F9F000005080F821129DF8080000EB001101EB87
:10FA0000002008EBC0029DF82000414600EB0010EA
:10FA100002EBC00000F5005090F81C02012814D041
:10FA20009DF8080000EB001202EB002001EBC00281
:10FA30009DF8200000EB001002EBC00000F5005024
:10FA400090F81C02022814D0D1E39DF8080002228D
:10FA500000EB001303EB002008EBC0019DF8200031
:10FA600000EB001001EBC00000F5005080F81C22F4
:10FA7000BDE39DF8080000EB001303EB002001EB51
:10FA8000C00000F5005080F817B29DF8080003226E
:10FA900000EB001303EB002001EBC0039DF82000F6
:10FAA00000EB001003EBC00000F5005080F81C22B2
:10FAB00007229DF8080000EB001303EB002008EB81
:10FAC000C001FCF75EBC9DF80800142200EB001199
:10FAD00001EB002008EBC0039DF8200000EB0010B4
:10FAE00003EBC00000F5005080F821229DF80800CB
:10FAF00000EB001303EB002008EBC00000F5005002
:10FB000080F817929DF8080000EB400202EB00100D
:10FB100008EB00109DF8201000EB0110284401783C
:10FB200041F02001FBF758BB9DF8080000EB0011E5
:10FB300001EB002008EBC00000F5005080F817B280
:10FB40000522B6E79DF8080000EB001101EB00204C
:10FB500008EBC00000F5005080F817929DF80800EF
:10FB6000142200EB001303EB002008EBC0039DF808
:10FB7000200000EB001003EBC00000F5005080F8FF
:10FB800021229DF8080000E0D4E000EB400202EBE7
:10FB9000001008EB00109DF8201000EB0110284425
:10FBA000017841F00401BDE70020CDE900000146E5
:10FBB0005E468DF824B01EE0090241EA10610002A1
:10FBC000CDE900019DF8080000EB4001C1EBC01138
:10FBD000FE4800EBC1009DF8241008444079DDE99F
:10FBE0000012084346EA0201CDE900019DF8240015
:10FBF000401C8DF824009DF8240003280098DBD3D6
:10FC000002F03EFC9DF80810474601EB011202EBA2
:10FC1000012108EBC1029DF8201001EB011102EB5C
:10FC2000C10101F50051C1F839020020CDE9000001
:10FC300002468DF82460DFF894831DE0120242EA48
:10FC400010620002CDE900029DF8080000EB4001BF
:10FC5000C1EBC01108EBC1009DF824100844007AE4
:10FC6000DDE90021104346EA0102CDE900029DF8DA
:10FC70002400401C8DF824009DF8240003280098DF
:10FC8000DCD301E0B4E2F7E2114602F0F9FB9DF8A3
:10FC9000081001EB011202EB012107EBC1029DF8F4
:10FCA000201001EB011102EBC10101F50051C1F877
:10FCB00035020020CDE900008DF8246042461FE0A7
:10FCC000DDE90001090241EA10610002CDE900010D
:10FCD0009DF8080000EB4001C1EBC0109DF8241016
:10FCE00002EBC0000844C07CDDE90013084346EA8B
:10FCF0000301CDE900019DF82400401C8DF824008B
:10FD00009DF824000328DBD39DF80800009900EB40
:10FD1000001202EB002007EBC0029DF8200000EB70
:10FD2000001002EBC00000F50050C0F8501207218F
:10FD3000FBF70EBE0020CDE9000001465F468DF8BE
:10FD400024B01EE0090241EA10610002CDE9000181
:10FD50009DF8080000EB4001C1EBC0119B4800EB8F
:10FD6000C1009DF8241008444079DDE900120843E1
:10FD700047EA0201CDE900019DF82400401C8DF8FE
:10FD800024009DF8240004280098DBD302F078FBBF
:10FD90009DF80820464602EB021303EB022208EB13
:10FDA000C2039DF8202002EB021203EBC20202F50F
:10FDB0000053C3F845021A46C2F849120020CDE9A3
:10FDC000000001468DF82470B846804A1DE0090203
:10FDD00041EA10610002CDE900019DF8080000EB46
:10FDE0004001C1EBC0109DF8241002EBC000084494
:10FDF000407ADDE90037184348EA0701CDE9000100
:10FE00009DF82400401C8DF824009DF8240004284F
:10FE10000098DCD302F034FB9DF8082002EB0213BB
:10FE200003EB022206EBC2039DF8202002EB021234
:10FE300003EBC20202F50053C3F83D021A46C2F8B2
:10FE400041129DF8080000EB001101EB002006EBC9
:10FE5000C0019DF8200000EB001001EBC00000F590
:10FE6000005090F81C129DF8080000EB001202EB05
:10FE7000002006EBC00000F5005090F81802814207
:10FE80007ED194F8A40780B19DF8080000EB4001F2
:10FE900001EB00109DF8201006EB001000EB0110A4
:10FEA0002844017841F0080181E0C6F839809DF8C6
:10FEB000080000EB001101EB002006EBC0019DF8EB
:10FEC0002000102200EB001001EBC00142F23D20A7
:10FED00001440798F8F7B9F99DF8080000EB001104
:10FEE00001EB002006EBC0019DF8200000EB0010A4
:10FEF00001EBC00000F2352000F500500168C6F8A3
:10FF00001D104068C6F821009DF8080000EB400174
:10FF100001EB001006EB00119DF8200001EB001032
:10FF200000F5805090F8840D30779DF8080000EBC4
:10FF3000001101EB002006EBC0019DF8200000EB52
:10FF4000001001EBC00000F50050D0F85002C6F8D8
:10FF50002500049850F8691FC6F83D108088A6F85F
:10FF60004100B06D81B20220F8F7EEFD00210620BD
:10FF7000F9F7F4FBB06D718B884204D2B06D00E0EC
:10FF8000A4E0401CB06500210520F9F7E7FB9DF8CF
:10FF9000080000EB400101EB001106EB01109DF899
:10FFA000201000EB01102844017821F008010170B5
:10FFB0009DF808100220F9F7D1FB9DF820009DF86C
:10FFC000081000EB0110C11702E00000806400205F
:10FFD000CDE9000100EB8002C2EB80103044C0F894
:10FFE0007D809DF8081001EB011202EB012106EB68
:10FFF000C1029DF820106D3001EB011102EBC1022E
:020000040801F1
:1000000042F23D2111441022F8F71FF99DF8080033
:1000100000EB001101EB002006EBC0019DF8200071
:1000200000EB001001EBC001009801F2352100EB5C
:10003000800201F50051C2EB80100A68304440F89C
:10004000612F496841609DF8081001EB410202EB05
:1000500001119DF8202006EB011101EB021101F5C1
:10006000805191F8841D00F8011C049951F8692F02
:100070000262898881849DF8081001EB011202EB6D
:10008000012106EBC1029DF8201001EB011102EBEA
:10009000C10101F50051D1F8501281609DF808109E
:1000A00001EB410202EB01119DF8202006EB01114A
:1000B00001EB021101F58051D1F8881DC0F826101E
:1000C000009881B20820F9F749FB10E09DF808007C
:1000D00000EB400101EB001006EB00119DF8200041
:1000E00001EB00102844017841F0040101709DF8F3
:1000F000080000EB001202EB002006EBC0029DF8A6
:10010000200000EB001002EBC00000F5005080F86A
:100110005A829DF80800172100EB001202EB002024
:1001200006EBC0029DF8200000EB001002EBC000BF
:1001300000F5005080F821129DF8080000EB001136
:1001400001EB002006EBC0019DF8200000EB001041
:1001500001EBC00000F5005090F81C129DF808005B
:1001600000EB001202EB002006EBC00000F500508F
:1001700090F8180281423AD29DF8080000EB400145
:1001800001EB00109DF8201006EB001000EB0110B1
:100190002844017841F0800101709DF8080000EBCF
:1001A000001202EB002006EBC00000F5005080F8C2
:1001B00017929DF8080000EB001101EB002006EB00
:1001C000C00000F5005090F818129DF8080000EBF0
:1001D000001202EB002006EBC0039DF8200000EBAC
:1001E000001003EBC00000F5005080F81C124EE038
:1001F0004A4684F8E0969DF8080000EB001101EBF8
:10020000002008EBC0039DF82000414600EB0010E1
:1002100003EBC00000F5005090F81C329DF8080078
:1002200000EB001606EB002008EBC00000F50050C4
:1002300090F8180283422AD29DF8080000EB0016BD
:1002400006EB002001EBC00000F5005080F817B26B
:100250009DF8080000EB001303EB002001EBC00346
:100260009DF8200000EB001003EBC00000F50050EB
:1002700080F81C2214221CE49DF80800142100EBD5
:10028000001202EB002208EBC202FBF769BB94F8F4
:10029000E803B0B11F489DF8081000EB410000F5DD
:1002A0008040B0F834149DF80800012300EB4002B0
:1002B000C2EBC012184800EBC2009DF80820F9F705
:1002C000A5FE59468DF824B0134A0FE09DF80800AA
:1002D00000EB4003C3EBC0109DF8243002EBC000DC
:1002E000C1549DF82400401C8DF824009DF8240082
:1002F0001428EBD3094801784278114482781144DC
:10030000C278D1427AF438A821B0BDEC028BBDE8A6
:10031000F08F0000A4120020806400201200002052
:100320002DE9F74F92B000209146ADF80800ADF8E6
:100330000000ADF80000ADF814008DF818008DF83D
:100340001C008DF82000CDE90000CDE90000ADF8DB
:100350004400F7A1D1E90023F7A1CDE90323D1E9B6
:100360000023F749CDE9092308711298F54A00EBFB
:10037000400101EB001002EB001E0EF580500190D1
:1003800090F85A0D8DF818001298139902EB00108E
:100390000D90084400F58050824690F8883B1298F2
:1003A000042B00EB001101EB0020114601EBC00013
:1003B00013990F9001EB011100EBC106139906F59B
:1003C00000550EEB011000F5805B22D105208AF864
:1003D000880B002085F81C029BF8860D20F0800118
:1003E0008BF8861D019890F85A1DA120082910D27B
:1003F000DFE801F00F040D0D06080A0CE52006E009
:10040000B12004E0312002E0F12000E0062085F870
:100410002102CC48007E012876D09DF818801298E1
:10042000022200EB001404EB0020C64C412104EB37
:10043000C004129804F50054C34F0094C0EB0010A0
:10044000A9F1A1034FF0040C00EB8004B8F1080FF0
:100450007ED2DFE818F07D000800A5020A047F05BF
:100460007206E906A1089BF8850D4FF00008414689
:1004700002F006F88DF81C0095F81C12009890F810
:100480001802814203D10098012180F817129AF8CE
:10049000880B401C8AF8880BA221A6224846B9F195
:1004A000CE0F70D014DC4FF0A503B9286CD007DC58
:1004B000B2286AD0B5283AD0B9F1B60F48D117E1C1
:1004C000C3287CD0C5287BD0B9F1CA0FF6D104E18E
:1004D000E12876D007DCD5280BD0D72872D0B9F127
:1004E000D90FEBD111E0E5286DD0B9F1E70FE5D1D7
:1004F00040E2F52007F834009DF81C0007EBC40526
:100500006870A970D5200AE0F1E3F52007F83400FF
:100510009DF81C0007EBC4056870A970D920E8702D
:100520002846032101F0DDFE287105208DE3F5202A
:1005300007F834009DF81C0007EBC40670700198A2
:1005400090F8600D4FF0B5090028D5F8240200E0BE
:10055000AFE208D0B0F1104F36D34FF01040002179
:10056000CDE9000134E0B0F5100F05D34FF41000D1
:100570000021CDE9000103E0D5F82402CDE900080F
:10058000B370404612E04EE13CE0BCE0BDF808002C
:10059000C0F10200C200DDE90001F7F744FEBDF83A
:1005A00008103144C870BDF80800401CADF80800C0
:1005B000BDF808000328E9D386F80690F8E081E04A
:1005C00026E1FCE0E1E1CAE1D5F82402CDE900082A
:1005D000B27040460FE0BDF80800C0F10300C20051
:1005E000DDE90001F7F71FFEBDF808103144C870BF
:1005F000BDF80800401CADF80800BDF8080004284C
:10060000E9D35DE0F52007F834009DF81C0007EB06
:10061000C4067070019890F8600D4FF0B909002879
:10062000D5F8240209D0B0F1104F2DD0D5F824020E
:10063000CDE90008B27040463CE0B0F5100F06D09E
:10064000D5F82402CDE90008B370404615E04FF418
:1006500010000021CDE90001F6E7BDF80800C0F167
:100660000200C200DDE90001F7F7DDFDBDF808106A
:100670003144C870BDF80800401CADF80800BDF852
:1006800008000328E9D397E74FF010400021CDE997
:100690000001CFE7BDF80800C0F10300C200DDE9AA
:1006A0000001F7F7C0FDBDF808103144C870BDF86F
:1006B0000800401CADF80800BDF808000428E9D384
:1006C00048469DE0F52007F834009DF81C0007EB34
:1006D000C4056870A970C32021E7F52007F834002D
:1006E0009DF81C0007EBC4056870A970CA2016E7C6
:1006F000F52007F834009DF81C0007EBC40568706E
:10070000A970B6200BE7F52007F834009DF81C000F
:1007100007EBC4067070019890F8600DB22110B11B
:10072000B37040463DE0A420B07040461DE000009C
:1007300001693230313030000169323045303000EB
:1007400012000020A4120020205B0020D5F85002E7
:10075000BDF80820C2F10102D200D040BDF8082047
:100760003244D070BDF80800401CADF80800BDF858
:1007700008000228EAD371713046052101F0B1FD6D
:10078000B07178E1D5F85002BDF80820C2F102023C
:10079000D200D040BDF808203244D070BDF8080027
:1007A000401CADF80800BDF808000328EAD3B17179
:1007B0003046062101F095FDF0710820B6E6F520DF
:1007C00007F834009DF81C0007EBC4067070B27087
:1007D00040460EE0D5F85402BDF80810C1F10301FF
:1007E000C900C840BDF808103144C870BDF8080001
:1007F000401CADF80800BDF808000428EAD3E12049
:10080000F0713046072101F06CFD307209208DE651
:10081000F52007F834009DF81C0007EBC40568704C
:10082000A970C5207BE6F52007F834009DF81C0070
:1008300007EBC4056870019890F8600D4FF0CE0981
:1008400018B1AE20A87040465CE0AC20A8704046CD
:1008500015E006F50050D0F83D0206F50051D1F83C
:100860004112BDF80820C2F10402D200F7F7DBFC08
:10087000BDF808102944C870BDF80800401CADF848
:100880000800BDF808000528E3D3404615E006F54A
:100890000050D0F8450206F50051D1F84912BDF8D4
:1008A0000820C2F10402D200F7F7BDFCBDF8081021
:1008B00029440872BDF80800401CADF80800BDF8D6
:1008C00008000528E3D385F80D9028460D2101F096
:1008D00008FDA8730F2029E606F50050D0F83D0268
:1008E00006F50051D1F84112BDF80820C2F1050209
:1008F000D200F7F798FCBDF808102944C870BDF87D
:100900000800401CADF80800BDF808000628E3D335
:10091000404615E006F50050D0F8450206F50051B6
:10092000D1F84912BDF80820C2F10502D200F7F74C
:100930007AFCBDF8081029444872BDF80800401C34
:10094000ADF80800BDF808000628E3D385F80F903D
:1009500028460F2101F0C5FC28741120E6E5F5209A
:1009600007F834009DF81C0007EBC4056870A970F7
:10097000E520D4E5F52007F834009DF81C0007EBCE
:10098000C4056870A970E720C9E5F52007F83400B0
:100990009DF81C0007EBC4056870A970D720BEE560
:1009A0009BF8850D8DF81C0095F81C62009890F856
:1009B0001802864203D10098012680F817629AF83F
:1009C000880B401C8AF8880B9DF81C0020B19DF80C
:1009D0001C00401E8DF81C000A2B6AD2DFE803F0D1
:1009E00041FD5588EAFCFB05FA6A07F834209DF8BA
:1009F0001C0007EBC40640307070B1703020F070FE
:100A0000307195F820020009707170790A287079A8
:100A100001D2303000E03730707195F8200200F0DC
:100A20000F00B071B0790A28B07901D2303000E0FF
:100A30003730B0710320F071701C0721F8F726FAE7
:100A400030720920ADF8440095F81C02042802D148
:100A5000052085F81C020099002081F81702062065
:100A600025E007F834C09DF81C1007EBC4004031A6
:100A70004170512144E1072058E528710320687135
:100A8000681C0521F8F702FAFAE307F834C09DF86C
:100A90001C2007EBC4004032427081700521C170F8
:100AA000ADF844C095F81C02022802D1032085F855
:100AB0001C022AE107F834209DF81C0007EBC4054E
:100AC00040306870A9703120E8703220287103200E
:100AD0006871681C0521F8F7D9F9A8710720ADF8ED
:100AE00044009BF8860D20F020018BF8861DE0E77E
:100AF00007F834209DF81C0007EBC40640307070E6
:100B0000B1703121F17030203071D5F82422B2F566
:100B1000100F00D23220707195F82202012803D004
:100B200095F8220210B103E0B17101E03220B071FA
:100B30000021ADF8081013E0D5F82402BDF8082014
:100B4000C2F105029200D040BDF8082000F00F006D
:100B500032443030D071BDF80800401CADF80800B8
:100B6000BDF808000628E7D332207073ADF80810EE
:100B700013E0D5F85002BDF80810C1F10301890057
:100B8000C840BDF8081000F00F00314430308873C1
:100B9000BDF80800401CADF80800BDF808000428A6
:100BA000E7D30320B074701C1221F8F76FF9F074CA
:100BB0001420BBE407F834209DF81C0007EBC406A2
:100BC00040307070B1703220F0703121317170712D
:100BD000B07103E07EE03EE038E06EE00021ADF869
:100BE000081013E0D5F85002BDF80820C2F1030246
:100BF0009200D040BDF8082000F00F0032443030A1
:100C0000D071BDF80800401CADF80800BDF8080020
:100C10000428E7D3ADF80810302108E0BDF808003B
:100C20003044C172BDF80800401CADF80800BDF8A2
:100C300008001928F2D3032086F82400701C242110
:100C4000F8F724F986F82500262075E2102007F829
:100C50003400302003E0102007F83400312007EB87
:100C6000C4014870ADF844204FE09BF8850D8DF825
:100C70001C0095F81C62009890F81802864203D177
:100C80000098012680F817629AF8880B401C8AF8B1
:100C9000880B9DF81C0020B19DF81C00401E8DF8AB
:100CA0001C000A2BE0D2DFE803F00708234CF30610
:100CB00005301531CFE7C9E7D3E607F834209DF8B2
:100CC0001C0007EBC40540306870A9703120E87043
:100CD0003520D2E607F834209DF81C0007EBC40548
:100CE00040306870A9703220E8703020C5E6F8E323
:100CF00007F834C09DF81C2007EBC4004032427056
:100D000081700521C170ADF844C0FAE107F83420C4
:100D10009DF81C0007EBC40540306870A9703120B5
:100D2000E8703220287103206871681C0521F8F7EB
:100D3000ADF8A8719BF8860D20F020018BF8861D78
:100D400099E607F834209DF81C0007EBC4064030F4
:100D50007070B1703120F0703171D5F82412B1F19A
:100D6000104F09D03221717195F82212012905D056
:100D700095F8220238B102E03021F4E7B071002288
:100D8000ADF8082015E03220F8E7D5F82402BDF8C8
:100D90000810C1F107018900C840BDF8081000F033
:100DA0000F0031443030C871BDF80800401CADF868
:100DB0000800BDF808000828E7D33220F073ADF82A
:100DC000082013E0D5F85002BDF80810C1F1050164
:100DD0008900C840BDF8081000F00F0031443030E1
:100DE0000874BDF80800401CADF80800BDF8080004
:100DF0000628E7D33020B075ADF8082008E0BDF82C
:100E000008103144C875BDF80810491CADF8081029
:100E1000BDF808100629F2D37077ADF8082008E075
:100E2000BDF8081031448877BDF80810491CADF8AA
:100E30000810BDF808100629F2D386F82400ADF892
:100E4000082009E0BDF80810314481F82500BDF8FC
:100E50000810491CADF80810BDF808100629F1D398
:100E600086F82B00ADF8082009E0BDF808103144E1
:100E700081F82C00BDF80810491CADF80810BDF829
:100E800008100629F1D386F83200ADF808200AE0F0
:100E900018E0BDF80810314481F83300BDF808109F
:100EA000491CADF80810BDF808100629F1D303203D
:100EB00086F83900701C3921F7F7E8FF86F83A0008
:100EC0003B2039E107F834209DF81C0007EBC406ED
:100ED00040307070B1703220F070312131713321A7
:100EE0007171B0710021ADF8081013E0D5F850020F
:100EF000BDF80820C2F105029200D040BDF80820DC
:100F000000F00F0032443030D071BDF80800401CB2
:100F1000ADF80800BDF808000628E7D3ADF80810C2
:100F2000302108E0BDF8080030444173BDF80800E6
:100F3000401CADF80800BDF808001928F2D30320C2
:100F400086F82600701C2621F7F7A0FF86F82700F8
:100F50002820F1E09BF8850D8DF81C00BDF80800F5
:100F60000F9900EB001001EBC00000F5005090F865
:100F70001C12009890F81802814203D100980121B8
:100F800080F817129AF8880B401C8AF8880B4FF0EB
:100F9000000840460EE0BDF808100EEB011000F509
:100FA000805090F8850D9DF81C1088420BD0BDF83C
:100FB0000800401CADF80800019890F85B0DBDF8E2
:100FC00008108842E7D8BDF808100EEB011000F5B4
:100FD000805090F8841D1398401A401C8DF8200012
:100FE0009DF81C0020B19DF81C00401E8DF81C00CF
:100FF00095F81D020F2803D295F81D02401C00E051
:10100000404685F81D02A9F1B1016520092978D271
:10101000DFE801F0050C56777778773042009DF8CD
:101020001C00503007F8340020217FE09DF81C00A0
:10103000503007F8340095F81D0207EBC40640F065
:10104000300070700120B070F07086F80480304677
:101050000521F8F7D9FACDE9000870710098000A67
:10106000B0710320F071FA2030720920ADF844000D
:10107000B120F0E29DF81C10503107F8341095F8BB
:101080001D1207EBC40541F030016970A870012002
:10109000E8709DF8200023E09DF81C10503107F8FF
:1010A000341095F81D1207EBC40541F0300169704A
:1010B000A8700120E8709DF8200040F010000FE0BB
:1010C0009DF81C00503007F8340095F81D0207EB1E
:1010D000C40540F0300068700120A870E870052059
:1010E000287128460521F8F78FFACDE900086871C4
:1010F0000098000AA8710320E871FA202872FFF70F
:1011000085BBA8E095F81E02B12806D095F81E020E
:1011100085F82102B12085F81E029DF81C00503090
:1011200007F8340095F81D0240F0C00107EBC40039
:101130004170FA218170032072E2BDF808100D9809
:10114000084441F6883108440178491C017001982F
:1011500090F8600D38B11399491CC9B2012837D0F5
:10116000022878D145E0B9F1310F03D0B9F1450F2C
:10117000F7D116E00020ADF8080003A90CE0BDF897
:101180000800BDF8083007EBC402085CD054BDF875
:101190000800401CADF80800BDF808000728EED391
:1011A00069E40020ADF8080009A90CE0BDF80800CA
:1011B000BDF8083007EBC402085CD054BDF8080045
:1011C000401CADF80800BDF808000728EED352E433
:1011D0008DF81C109DF81C0007F8340007EBC405BF
:1011E000032068700026AE70EA702E7109206871C5
:1011F0000EE08DF81C109DF81C0007F8340007EB7A
:10120000C405032068700026AE70EE702E716A71FE
:1012100028460621F8F70CF8CDE90006000AE87127
:101220000098A871FFF7C9BAFE499AF8880B401CCC
:101230008AF8880B9BF8850D8DF81C004846B9F19B
:10124000F30F74D008DC052872D0F1280AD0B9F168
:10125000F20F86D115E000E2F4286AD0B9F1F60F5A
:1012600086D1E7E0F52007F834009DF81C0007EB75
:10127000C40568700026AE700520E870F1200BE10F
:1012800014E1F52007F834009DF81C1007EBC400AA
:10129000804641704FF0000980F80290F221017100
:1012A00095F89212417195F89202012820D095F894
:1012B0009202202872D00620ADF84400BDF8440008
:1012C00088F803004046BDF84410F7F7B1FFCDE9B8
:1012D0000009BDF84420000A08F80200BDF84420C7
:1012E000009808EB02014870BDF84400801CB1E38F
:1012F0002520ADF844004946ADF8089010E0BDF84F
:101300000800304400F5005090F86522BDF8083020
:1013100008EB03008271BDF80800401CADF808001E
:10132000BDF808000F28EAD3ADF8081013E050E02C
:10133000BEE0A4E0BDF80800304400F5005090F88D
:101340007722BDF8083008EB03004275BDF80800AD
:10135000401CADF80800BDF808000A28EAD395F84B
:101360008C2288F81F20ADF8081011E0BDF80800A5
:10137000304400F5005090F88D12BDF8082008EBBD
:10138000020080F82010BDF80800401CADF80800ED
:10139000BDF808000528E9D390E7FFE70A20ADF87B
:1013A000440048460EE0BDF80800304400F5005007
:1013B00090F88D12BDF8082008EB02008171BDF88D
:1013C0000800401CADF80800BDF808000428EAD366
:1013D00074E7F52007F834009DF81C1007EBC400F3
:1013E000804641704FF0000980F80290F3220271AC
:1013F00095F8922242710C22ADF8442095F88C2287
:101400008271ADF8089010E0BDF80800304400F596
:10141000005090F88D12BDF8082008EB0200C17151
:10142000BDF80800401CADF80800BDF8080005280C
:10143000EAD343E70620ADF84400F52007F834006E
:101440009DF81C0007EBC40568700026AE70BDF85F
:101450004400E870F62028719BF88C0D68712846CE
:10146000BDF84410F7F7E4FECDE90006BDF84410DE
:10147000000A6854BDF844100098294433E7F52069
:1014800007F834009DF81C0007EBC40568700026BF
:10149000AE700520E870F420287128460521F7F782
:1014A000C7FECDE90006000A68710098A87147E4FC
:1014B00040F21320ADF84400F52007F834009DF801
:1014C0001C0007EBC4067070BDF84400000AB07041
:1014D000BDF84400F070052030714FF00008404620
:1014E0000FE00EE3BDF808200EEB020000F580507F
:1014F00090F8620DBDF8082032445071BDF8080024
:10150000401CADF80800BDF808000A28EAD301988D
:101510008946B0F86E0D000AF0730198B0F86E0DB0
:101520003074B5F8A002000A7074B5F8A002B07467
:10153000B5F8A012129801EB802081B20320F7F7D2
:1015400097FA4546ADF808804FF4007249460FE01F
:10155000BDF80800084400F5805090F8E701BDF898
:1015600008303344D874BDF80800401CADF80800BA
:10157000BDF808009042EBD33046BDF84410F7F7B1
:1015800057FECDE90005BDF84410000A7054BDF8BF
:10159000441000983144A6E69BF8850D4FF00008F2
:1015A000414600F06DFF8DF81C0095F81C12009864
:1015B00090F81802814203D10098012180F8171297
:1015C0009AF8880B401C8AF8880BB9F1070F15D0E0
:1015D0000ADCDFF854A0B9F1070F3ED2DFE809F0CA
:1015E0003D3EF23D0E0EF100A9F110000828F4D2A4
:1015F000DFE800F004E933330433041CFA2007F871
:10160000340007EBC4056870A87085F803909DF856
:101610001C002871E81C0221F7F738FC68710620CD
:1016200018E20000A412002000E1F505FA2007F8F6
:10163000340007EBC4067070B07086F803909DF814
:101640001C003071F01C0221F7F720FC707106209D
:10165000ADF84400142085F82102FDE1FA2007F8D6
:10166000340007EBC4067070B07086F803909DF8E4
:101670001C00307195F82202012803D095F822024F
:10168000E8B332E1D5F82402B0F1104F05D34FF49E
:1016900010000021CDE9000103E0D5F82402CDE9D6
:1016A000000840460FE0BDF80800C0F10200C2008B
:1016B000DDE90001F6F7B7FDBDF8081031444871C7
:1016C000BDF80800401CADF80800BDF8080003286C
:1016D000E9D30020CDE9000040460FE0BDF8080046
:1016E000C0F10300C200DDE90001F6F79CFDBDF882
:1016F000081031440872BDF80800401C00E05BE0AF
:10170000ADF80800BDF808000428E7D340460FE014
:10171000BDF80800C0F10200C200DDE90001F6F7E3
:1017200082FDBDF8081031440873BDF80800401C64
:10173000ADF80800BDF808000328E9D3D5F8501229
:10174000CDE9001840460FE0BDF80800C0F10200E6
:10175000C200DDE90001F6F766FDBDF8081031446E
:10176000C873BDF80800401CADF80800BDF80800BB
:101770000328E9D3D5F850124546BAFBF1F0CDE97C
:101780000008ADF8088011E0BDF80800C0F10300C2
:10179000C200DDE90001F6F746FDBDF8081031444E
:1017A0008874BDF80800401CADF80800BDF80800BA
:1017B0000428E9D3B57598E00020CDE90000404643
:1017C00012E010E1B5E020E1BDF80800C0F1020030
:1017D000C200DDE90001F6F726FDBDF8081031442E
:1017E0004871BDF80800401CADF80800BDF80800BD
:1017F0000328E9D3D5F82402B0F1104F05D34FF4F4
:1018000010000021CDE9000103E0D5F82402CDE964
:10181000000840460FE0BDF80800C0F10300C20018
:10182000DDE90001F6F7FFFCBDF80810314408724D
:10183000BDF80800401CADF80800BDF808000428F9
:10184000E9D340460FE0BDF80800C0F10200C20035
:10185000DDE90001F6F7E7FCBDF808103144087334
:10186000BDF80800401CADF80800BDF808000328CA
:10187000E9D3D5F85012CDE9001840460FE0BDF885
:101880000800C0F10200C200DDE90001F6F7CBFC60
:10189000BDF808103144C873BDF80800401CADF80D
:1018A0000800BDF808000328E9D3D5F850124046D7
:1018B000BAFBF1F1CDE900180FE0BDF80800C0F166
:1018C0000300C200DDE90001F6F7ADFCBDF8081029
:1018D00031448874BDF80800401CADF80800BDF81C
:1018E00008000428E9D30120B075DBF8881D4046C4
:1018F000491CCDE900180FE0BDF80800C0F1010057
:10190000C200DDE90001F6F78EFCBDF80810314495
:10191000C875BDF80800401CADF80800BDF8080007
:101920000228E9D3F01C1621F7F7B0FA70761A20D6
:1019300090E0FA2007F8340007EBC4067070B0702E
:1019400086F803909DF81C003071D5F85012CDE94F
:10195000001840460FE0BDF80800C0F10200C200C8
:10196000DDE90001F6F75FFCBDF80810314448716D
:10197000BDF80800401CADF80800BDF808000328B9
:10198000E9D3D5F850024546002100F0C9F80246D7
:101990000B4650460021F6F715FCCDE9000100F09A
:1019A0006FFDCDE90001ADF8085011E0BDF8080069
:1019B000C0F10300C200DDE90001F6F734FCBDF818
:1019C000081031440872BDF80800401CADF808004A
:1019D000BDF808000428E9D3F01C0921F7F756FAEE
:1019E00030730D2036E0FA2007F8340007EBC40509
:1019F0006870A87085F803909DF81C002871552028
:101A00006871E81C0321FFF73DB8FA2007F834009D
:101A100007EBC4056870A87085F803909DF81C005A
:101A20002871AA2068714046ADF8088008E0BDF82A
:101A3000081029448871BDF80810491CADF8081039
:101A4000BDF808100329F2D3E81C0621F7F71EFAA7
:101A500068720A20ADF844002D482E4D129931B11C
:101A6000012912D002291DD003293AD12AE0BDF85C
:101A70004410B1B38021F8F7A4FABDF84400C5F8CA
:101A8000A40024480121A03029E0BDF8441041B34E
:101A90000821F8F796FABDF8440068671D4801214F
:101AA00070301CE0BDF84400D8B14FF480711A4882
:101AB000F8F787FABDF84400C5F8BC0015480121C5
:101AC000B8300CE0BDF8441059B14FF48061F8F71C
:101AD00078FABDF84400E8650E4801215830F7F760
:101AE000FDFB0E4890F8E803002807D007EBC40080
:101AF0000023BDF84410129AF8F788FA15B0BDE833
:101B0000F08F9AF8880B401C8AF8880BF6E70000E3
:101B1000000C02400060024000000240A4220020AD
:101B20002DE9F04700242DED048B804689469FED7A
:101B30001E9B25462646E20040464946F6F773FBC3
:101B4000C7B22046F6F74EFD41EC110BB0EE490A44
:101B5000F0EE690A09F014F9380907F00F0100EBFB
:101B60008000B0EE408AF0EE608A01EB4000F6F7AC
:101B700039FD53EC182BF6F743FC41EC180B2846C3
:101B80003146F6F73CFD53EC182BF6F792FBF6F7CF
:101B900069FD641CE4B205460E46082CCBD3BDECAF
:101BA000048BBDE8F08700000000000000005940F1
:101BB00070B50E4D40F224442146284608F099FDA8
:101BC000012812D1298828462A1D1188214608F0AB
:101BD0002DFD0748012180F8291B0648D0F88C000C
:101BE0000549C0F57A70A1F83C0470BD004400407E
:101BF000A422002000600240A452002010B50B4C2B
:101C000040F22441204608F074FD01280DD12088BF
:101C1000201D00880648012180F8351B0548406CCE
:101C20000549C0F57A70A1F83E0410BD004C004093
:101C3000A422002000600240A452002010B50B4CEA
:101C400040F22441204608F054FD01280CD12088A0
:101C5000A0880748012180F8411B064840690649D1
:101C6000C0F57A70A1F8400410BD0000005000409B
:101C7000A422002000600240A452002010B50B4CAA
:101C800040F22441204608F034FD01280DD120887F
:101C9000201D00880648012180F84D1B0548C06AB8
:101CA0000549C0F57A70A1F8420410BD0048004013
:101CB000A422002000600240A452002010B5124C63
:101CC00010492046F7F7F4FA00212046F7F706FB03
:101CD0000E4C4021204608F005FD0028F9D0802157
:101CE0000B48F8F770F9084C0A49183C2046F7F7FA
:101CF000DFFA01212046F7F7F1FA074901200871C0
:101D000010BD000000802020A06002400044004080
:101D1000000C0240008800201200002010B5124C78
:101D200010492046F7F7C4FA00212046F7F7D6FA03
:101D30000E4C4021204608F0D5FC0028F9D008219F
:101D40000B48F8F740F9084C0A49303C2046F7F7B1
:101D5000AFFA01212046F7F7C1FA074901200871BF
:101D600010BD00002080002070600240004C004048
:101D7000000C0240008020101200002010B5124C10
:101D800010492046F7F794FA00212046F7F7A6FA03
:101D90000E4C4021204608F0A5FC0028F9D04FF455
:101DA00080710B48F8F70FF9074C0A49A83C204608
:101DB000F7F77EFA01212046F7F790FA064901204D
:101DC000087110BD00800028B8600240005000403B
:101DD00000000240208000101200002010B5124CBC
:101DE00010492046F7F764FA00212046F7F776FA03
:101DF0000E4C4021204608F075FC0028F9D04FF425
:101E000080610B48F8F7DFF8074C0A49303C204660
:101E1000F7F74EFA01212046F7F760FA064901204C
:101E2000087110BD00800018586002400048004052
:101E3000000C024000880010120000202DE9F0473D
:101E4000012190B0480505F02DFF8648F7F750FABC
:101E5000402738010024CDE90540C50107940894C6
:101E6000CDE9094546040C940D94DFF8FC917F48B8
:101E70000B94CDE90207CDE9006969460E947948D3
:101E8000F7F7DEFA012210217648F7F7C3FADFF8F8
:101E9000D4A1AAF1180A5046F7F72AFA4FF47A7833
:101EA000CDE90348E811CDE9054007940894CDE950
:101EB00009456F480B940C940D9400960E94CDE94F
:101EC000019069465046F7F7BBFA01215046F7F7F3
:101ED00005FADFF890A1AAF1300A5046F7F708FAA0
:101EE000E811CDE9054007940894CDE909450C9423
:101EF0000D94DFF8809160480B94CDE90207CDE99D
:101F0000006969460E945046F7F79AFA01221021AB
:101F10005046F7F77FFADFF84CA1AAF1600A504665
:101F2000F7F7E6F9CDE90348E811CDE90540079454
:101F30000894CDE9094551480B940C940D940096F2
:101F40000E94CDE9019069465046F7F779FA0121E0
:101F50005046F7F7C3F9DFF80CA10AF1180A50460A
:101F6000F7F7C6F9E811CDE9054007940894CDE9E3
:101F700009450C940D94DFF8089142480B94CDE983
:101F80000207CDE9006969460E945046F7F758FA02
:101F9000012210215046F7F73DFADFF8C8A0AAF158
:101FA000900A5046F7F7A4F9CDE90348E811CDE9C6
:101FB000054007940894CDE9094533480B940C94E7
:101FC0000D9400960E94CDE9019069465046F7F7BE
:101FD00037FA01215046F7F781F9DFF88890A9F127
:101FE00048094846F7F784F90397E811CDE9054019
:101FF00007940894CDE9094525480B940C940D9459
:10200000224F00960E94CDE9017069464846F7F7D5
:1020100017FA012210214846F7F7FCF9DFF844903F
:10202000A9F178094846F7F763F9CDE90348E811C3
:10203000CDE9054007940894CDE9094515480B946E
:102040000C940D9400960E94CDE9017069464846B3
:10205000F7F7F6F901214846F7F740F910B0BDE867
:10206000F0870000A060024004440040205B002094
:1020700080640020044C0040785D002068680020E7
:1020800004500040D05F0020506C00200448004005
:1020900028620020387000202DE9FC41012108460B
:1020A00005F000FE0121042005F0FCFD01210820BF
:1020B00005F0F8FD0121402005F0F4FDDFF8FC807B
:1020C000072205214046F7F765FF07220621404613
:1020D000F7F760FF072208214046F7F75BFF07226A
:1020E00009214046F7F756FF354F08220A213846A6
:1020F000F7F750FF08220B213846F7F74BFF08226D
:1021000002214046F7F746FF08220C213846F7F730
:1021100041FF02268DF8056000244FF459708DF8B8
:102120000640012500908DF807508DF8046069463F
:102130004046F7F7F3FE8DF805604FF4E0508DF858
:10214000064000908DF807508DF8046069463846C7
:10215000F7F7E4FE4FF4916000908DF806408DF89B
:10216000045069464046F7F7D9FE280200908DF8E2
:1021700006408DF8045069461248F7F7CFFE8DF8F7
:1021800006404FF4F040104C00908DF80450694622
:102190002046F7F7C3FEA9032046F7F712FF6903AD
:1021A0002046F7F70EFFA1142046F7F70AFFE114C7
:1021B0002046F7F706FFBDE8FC810000000C024056
:1021C00000080240000002400018024070B50024E0
:1021D000FFF762FFFFF732FE00F01EF80C48002107
:1021E0000170817041700121C1704FF47A7181607A
:1021F000084D042085F8240B04E0204600F062F925
:10220000641CE4B295F8240BA042F6D870BD00001F
:1022100024570020A4220020F8B511208DF80000DA
:1022200002258DF8015001248DF802408DF80340FD
:10223000684601F0C1F926208DF800008DF80140B4
:1022400000268DF802608DF80340684601F0B4F96D
:102250000E208DF800008DF801508DF802408DF8A9
:102260000340684601F0A8F927208DF800008DF89A
:1022700001408DF802608DF80340684601F09CF93A
:102280000F208DF800008DF801508DF802408DF878
:102290000340684601F090F934208DF800008DF875
:1022A00001408DF802608DF80340684601F084F922
:1022B0002F208DF800008DF801508DF802408DF828
:1022C0000340684601F078F935208DF800008DF85C
:1022D00001408DF802608DF80340684601F06CF90A
:1022E000F8BD01B9102110F8012B10F8013B491E6F
:1022F0005A400904090CF8D102F07F007047000031
:102300002DE9FF5F14460F464FF480564FF4806866
:102310004FF4C0694FF00C0A40F2244B002580B105
:10232000012830D0022851D0032871D1012188041E
:1023300005F0DCFC0097012C6DD0022C70D094B31A
:1023400077E00121480405F0D1FC0097012C03D06F
:10235000022C06D054B10DE0ADF80460ADF8088051
:1023600008E0ADF80460ADF8089003E0ADF8045063
:10237000ADF80850ADF80650ADF80C50ADF80AA015
:1023800069463B4C5DE00121C80405F0AFFC0097B5
:10239000012C03D0022C07D05CB10EE0ADF8046034
:1023A000ADF8088009E040E0ADF80460ADF80890B1
:1023B00003E0ADF80450ADF80850ADF80650ADF8A4
:1023C0000C50ADF80AA069462A4C3AE001210805F4
:1023D00005F08CFC0097012C03D0022C06D054B1E0
:1023E0000DE0ADF80460ADF8088008E0ADF80460D9
:1023F000ADF8089003E0ADF80450ADF80850ADF822
:102400000650ADF80C50ADF80AA069461A4C18E019
:102410002CE000E004E0ADF80460ADF8088008E0CE
:10242000ADF80460ADF8089003E0ADF80450ADF8E5
:102430000850124CADF80650ADF80C50ADF80AA09B
:102440006946204608F08CF90121204608F0F1F891
:1024500001225946204608F06BF91021204608F069
:10246000E5F80122C021204608F0EDF8BDE8FF9F05
:1024700000440040004C0040005000400048004034
:102480002DE9FC410024CDE900446F46642200237D
:10249000F5F798FE0E460546104619460A22002317
:1024A000F5F790FE010102F00F000818385504F10D
:1024B0000104E4B228463146082CE7D3DDE90001E7
:1024C000BDE8FC812DE9FC5F984E4FF0040982467F
:1024D000002586F8249B00EB400101EB0A10A6F5CD
:1024E000805707EB0014019404F5805494F8610DB3
:1024F000012803D10021504600F020F90AEB4A02DE
:10250000BB4607EB8207A7F59B6707F500574FF01F
:10251000000887F8008087F8028087F8018087F834
:1025200003800521B96087F8308087F83280012068
:1025300087F8310087F83300D4F85C0D00EB800099
:102540004000B86394F8592DD4F8541D5046A7F6AE
:102550002837FFF7D5FE94F85A1D0AEB0A1202EB52
:102560000A20734A082902EBC000009000F50050D1
:1025700013D2DFE801F01204060A1A0C181A05211A
:1025800000E00F2180F8181207E00721FAE7D4F8DD
:102590005C1D64225143C7F8601B9BF81810D94694
:1025A000012904D019E00321ECE74946EAE780F865
:1025B00018820120C7F8300B5E4F80213846F7F7AC
:1025C00002FD08213846F7F7FEFCB9155A48F7F71F
:1025D000FAFC39153846F7F7F6FC4FF0A10ECB465A
:1025E0007FE0009805EB051200EBC20000F50770D4
:1025F00000F5005000210173012282734173C17301
:10260000D4F85C2D94F85B7D7A4302EB8202920051
:102610004261019A02EB051202F5805292F8867D22
:1026200027F0800782F8867D017094F85A1DA0F586
:102630000770082953D2DFE801F0520408080A0C99
:102640000E44E52180F8211249E07146FAE7B121F4
:10265000F8E73121F6E7F12180F8211200212BE083
:1026600001EB011303EB01230BEBC30701EB410368
:1026700003EB01130BEB0313002003F5805915E066
:1026800003EB001C0CF5805C9CF884CD92F88C8DDB
:10269000C44509D192F884CD00EB001807EBC808B7
:1026A00008F5005888F893C2401CC0B299F85BCD79
:1026B0008445E5D8491CC9B296F8240B8842CFD886
:1026C0000DE0062180F8211205EB0A1101EB8102D1
:1026D000C2EB81115944D1F86910C0F850126D1C39
:1026E000EDB294F85B0D5B46A8423FF67AAF00204E
:1026F00086F8250B00EB400101EB001103EB011103
:1027000001F5805191F85A2D052A09D291F85A2DD8
:1027100032B196F8252B91F85B1D114486F8251BE4
:10272000401CC0B20428E5D3BDE8FC9FA4220020D1
:10273000A4120020000C0240000002402DE9F041EC
:10274000054663484FF4804253100668614884147C
:10275000C71439B1C5B1012D18D0022D18D0032DE1
:102760001BD117E035B1012D06D0022D06D0032D67
:1027700013D105E0114604E0194602E0214600E0CD
:102780003946F7F720FC08E0114604E0194602E05C
:10279000214600E03946F7F714FC642009F036FCC6
:1027A00000224FF416512846FFF7AAFD4A4905EBCF
:1027B000450001EB800000F58050002280F85A2B84
:1027C000C0F85C2B05EB450000EB051001EB001099
:1027D00000F58050D0F85C3D01F58041C1F88834A7
:1027E000012381F8813490F85A1D3C4C962305EB67
:1027F0008500204406290AD2DFE801F00903050517
:102800000733762102E0837001E06E218170C5EB11
:102810000511334B01EB8101C02403F8314003EB78
:10282000C10462700821A170E27006F00F0105EB8F
:10283000051211442171807860712020A071E1712E
:10284000802020724C2060725420A0722548264FB0
:102850000B2645B1012D0FD0022D25D0032D14D10B
:102860002DE06621D2E78021F7F7ABFBC7F8A46023
:102870001D480121A03006E00821F7F7A2FB7E6782
:10288000194801217030F6F729FD184890F8E8033F
:1028900028B1204600232A460B21F7F7B7FBBDE8F5
:1028A000F041642009F0B2BB4FF480711048F7F793
:1028B00088FBC7F8BC600C480121B830E3E74FF44F
:1028C0008061F7F77EFBFE65074801215830DAE7A3
:1028D000187AFF1F00180240A41200202074002064
:1028E000205B0020000C024000600240A422002077
:1028F000000002402DE9F04700252DED028B8EB03F
:102900008DF828508DF82C508DF83050CDE90855B1
:10291000CDE900558DF808508DF80C508DF8105009
:102920008DF81450ADF818509FEDFE0AFE4C079537
:102930008DED090A94F83A0D4FF0010908B384F8B7
:102940003A5DB4F8520DF94E3168C1F57A7188429A
:1029500017D13068C0F57A70A4F8500D371F0021E8
:102960003846F6F7BBFCF2493846F6F7A1FCF149C8
:1029700081F800904FF47A70306001213846F6F704
:10298000ADFC94F8DA0CEB4FBF1C02280AD00428E7
:1029900001D0052803D184F8469DC4F8485D8DF820
:1029A000285055E2E048603090F8D80BDFF8888373
:1029B00041F6865A08F1020606F5805600287DD0B9
:1029C00001287CD00228E6D1F879397A40EA012042
:1029D000C117CDE90001D7480721801CF6F728FC74
:1029E000CDE90805DDE90001089B6940584008432E
:1029F000D1D13878401E8DF8100086F82C5D9DF8F6
:102A000010004646404400F5805080F88555B8795E
:102A1000F5F7E8FD41EC110B9FEDC80B08F0B0F99C
:102A20003879B0EE408AF0EE608AF97840EA012009
:102A3000F5F7D8FD53EC182BF5F754FDF5F737FEF5
:102A40009DF8101006EB011101F58051C1F89505B4
:102A50009DF8100006EB001000F58050C0F891556D
:102A60009DF8100006EB001000F58050C0F8995555
:102A70009DF8100006EB001000F58050C0F89D5541
:102A80009DF8080000EB400101EB00109DF81010CC
:102A900006EB001000EB011101EB0A00017841F098
:102AA00080010170797A9DF8080000EB001202EBBA
:102AB000002006EBC0029DF8100001E017E00BE1DA
:102AC00000EB001002EBC00000F5005080F8581237
:102AD0009DF8080000EB400101EB001006EB001030
:102AE00000F5805090F85B0D84F8840553E79DF85D
:102AF000081008EB410000F58040B0F83414781C51
:102B0000891FF6F7ABFBC117CDE908019DF8081046
:102B100008EB410000F58040B0F834148548C01E31
:102B20000844042105F0A2FBC117CDE90001DDE94D
:102B3000083201460198594050400143D6D186F8E9
:102B40002C5D3879ADF81800BDF818003128CDD1CA
:102B50009DF80800464608EB400000F58040B0F8BC
:102B600034044121183890FBF1F0C117CDE9000180
:102B700084F884058DF82850A4E09DF8280000EB27
:102B800080103844017D9DF82800304400F58050C5
:102B900080F885159DF82800082100EB8010384446
:102BA0001A3005F02FFB00EE100AB8EEC00A8DEDCA
:102BB000090A10EE100A9DF8281006EB011101F524
:102BC0008051C1F895059DF82800082100EB801080
:102BD0003844323005F016FB00EE100AB8EEC00A99
:102BE0008DED090A10EE100A9DF8281006EB011170
:102BF00001F58051C1F891059DF82800082100EBEE
:102C0000801038443A3005F0FDFA00EE100AB8EEB4
:102C1000C00A8DED090A10EE100A9DF8281006EB87
:102C2000011101F58051C1F899059DF8280008218E
:102C300000EB80103844423005F0E4FA00EE100A50
:102C4000B8EEC00A8DED090A10EE100A9DF82810A2
:102C500006EB011101F58051C1F89D059DF80800B2
:102C600000EB400101EB00109DF8281006EB00106E
:102C700000EB011101EB0A00017841F080010170C5
:102C80009DF8080006EB400000F58040B0F83414D1
:102C90002848401C095C9DF8080000EB001202EB7C
:102CA000002006EBC0029DF8100000EB001002EBC4
:102CB000C00000F5005080F858129DF82800401C14
:102CC0008DF828009DF82810DDE90023891A75EB9E
:102CD0000300FFF652AF5EE6787DB97D40EA012041
:102CE000C117CDE9000113481521801CF6F7A0FAA1
:102CF000CDE90805DDE90010089B68405940014313
:102D0000E9D13878401E8DF8100086F82C5D9DF8CA
:102D100010004646404400F5805080F885559DF8E7
:102D200010000FE000000000A42200202C640240EC
:102D300000880010CE0A0020A4120020000000002D
:102D40000000244008EB001000F58050C0F89555B5
:102D5000B879797940EA012000EE100AF8EE400ACD
:102D60009FED400A387980EE801AF97840EA012018
:102D700000EE900A9DF81000F8EE600A71EE200A4D
:102D800010EE901A06EB001000F58050C0F8911577
:102D9000B87A797A40EA012000EE900A387AB8EEE3
:102DA000601AC1EE000AF97940EA012000EE100A2B
:102DB0009DF81010B8EE400A30EE800A10EE100AAE
:102DC00006EB011101F58051C1F89905F87A00066A
:102DD000387BF97A40EA01200AD400EE100ADFEDD0
:102DE000220AB8EE400A20EE200A10EE100A0BE08C
:102DF000404280B2F5F7F6FB9FED1C1B53EC112B04
:102E0000F5F7FEFAF5F753FC9DF8101006EB0111EB
:102E100001F58051C1F89D059DF8080000EB4001C7
:102E200001EB00109DF8101006EB001000EB0111F3
:102E300001EB0A00017841F080010170F97D32E672
:102E40009DF828003D549DF82800401C8DF828006E
:102E50009DF828001428F3D30EB0BDEC028BBDE81A
:102E6000F087000000FF7F470000803D0000000069
:102E70000000B0BF2DE9F34F8246F2A085B0D0E943
:102E80000010CDE90110F1A00026D0E90010CDE935
:102E90000310F04935463746B046B3464E70EE4A09
:102EA00002EB0A0000F5805090F82C1D042921D176
:102EB000052180F82C1D594680F8DEBC90F8BC3CFA
:102EC00023F0800380F8BC3C5046BAF1020F07D0D3
:102ED000042803D0BAF1050F0CD105E0DF4805E066
:102EE000DE483121801E01E0DC48401C00F5005026
:102EF00080F8E31CD8480AEB4A0100EB011000F50A
:102F00008050814690F8D22BD548D64C4FF4807132
:102F1000022A7DD0042A0FD0052A0AD194F82C0D5C
:102F2000401C84F82C0D99F8D11BD9F8CC0B00F07B
:102F3000FDFA07B0BDE8F08F94F8DC2C002AF8D039
:102F4000F7F73FF8C44E99F8D11BD9F8CC0B00F035
:102F5000EDFA94F8DC0C012802D0022841D11BE0E4
:102F600094F8DB1C01EB8100C0EB8110304490F839
:102F70006080B94A50F8617F02F64173C2F8217F40
:102F80004768C2F8257F8268C6F8292F026A1A604E
:102F9000808C98800F0924E096F8208F1DE007EBC5
:102FA000470101EB071106EB0112002002F58051E9
:102FB00009E002EB001303F5805393F884CDC44578
:102FC00005D0401C80B291F85B3D8342F1D891F866
:102FD0005B1D814205D87F1CBFB294F8240BB84218
:102FE000DDD840460021FFF74BFA02460B4606218A
:102FF0000020CDF800B004F0ABFD07EB470000EB7C
:10300000071006EB0017A7F5247707F5005700E037
:10301000ADE03878C0F381000090D6F8212F00236E
:103020000721184606F6297604F092FD387800F05C
:103030000300009056F8042C00230821184604F0E1
:1030400087FD3878C0F30110009032680023092111
:10305000184604F07DFD322004F8C70F3020607060
:10306000717F00EB1111A170717F01F00F01303100
:10307000E1702D212171327F00EB12126271327FDB
:1030800002F00F023032A271E171F17E00EB1111FA
:103090002172F17E01F00F0130316172B17E00EBDF
:1030A0001111E172B17E01F00F01303121733A212B
:1030B0006173727E00EB1212A273727E02F00F0235
:1030C0003032E2732174317E00EB11106074307E77
:1030D00000F00F003030A07400202021624F40F239
:1030E0008A22C73CA6F629763954401C80B2904209
:1030F000FAD34FF00A0C87F800C087F801C000210E
:10310000002006EB4112131893F85B3F202B03D1EC
:10311000401C80B22028F6D31F280DD2002013189F
:1031200093F85B3F00EB451807F80830401C80B26D
:103130002028F4D36D1CADB2491C89B21429DFD309
:1031400007EB451080F820C080F821C080F822C02D
:1031500080F823C080F824C080F825C0252000EB2B
:1031600045100004000C84F8DCBC55D1E1E60F46A4
:103170008046F6F728FF4FF400714046F6F723FF2C
:10318000354D99F8D11BD9F8CC0B00F0CFF994F854
:103190002C0D401C84F82C0D0AEB4A0101EB0A109F
:1031A00005EB001000F5805090F8600DE8B10225A5
:1031B0000124032601283AD00228D7D139464046B7
:1031C000F6F701FF284F3C707E7087F802B087F851
:1031D00003B087F804B07D7106212348F6F728F87C
:1031E000010AF971B871082016E0069831280AD052
:1031F0004528BBD11C4803A98A5D8255761CB6B20E
:10320000072EF9D307E0184801A98A5D8255761C7C
:10321000B6B2072EF9D307201449086013480121DC
:10322000001FF6F75BF80B4981F801B081E60E4FFD
:103230003C707E7087F802B0FD7087F804B00920FA
:103240007871C9E7016932303130300001693230BC
:1032500045303000CE0A0020A4120020A802002031
:1032600000080240A4220020B80E0020A4640240FE
:1032700070B50D4C40F224452946204607F039FA36
:10328000002810D02946204607F0D0F92088201DBC
:1032900000880648012180F8391D05490968C1F5F3
:1032A0007A71A0F8521D70BD00140140A4220020C4
:1032B0002C64024010B5124C10492046F5F7F8FF77
:1032C00000212046F6F70AF80E4C4021204607F070
:1032D00009FA0028F9D04FF400710B48F6F771FE97
:1032E000074C0A49783C2046F5F7E2FF01212046C9
:1032F000F5F7F4FF06490120487010BD008020203A
:10330000A064024000140140000802400088001040
:10331000CE0A00202DE9F04301218FB0880504F08A
:10332000C1FCDFF894904846F5F7E2FF4020050124
:1033300003900024CDE90545C60207940894CDE921
:1033400009464FF020681E480B940C940D941B4FB7
:10335000CDF800800E94CDE9017069464846F6F735
:103360006FF8012210214846F6F754F8DFF848902C
:10337000A9F178094846F5F7BBFF4FF47A70CDE91B
:103380000340CDE9054507940894CDE909460D4869
:103390000B940C940D94CDF800800E94CDE901703F
:1033A00069464846F6F74CF801214846F5F796FF7E
:1033B0000FB0BDE8F0830000A06402400414014097
:1033C000B80E0020D00A00207CB50121042004F0B2
:1033D00069FC184E082206213046F6F7DBFD08226C
:1033E00007213046F6F7D6FD02218DF8051000259D
:1033F0008DF806500124C0208DF8074000908DF80C
:10340000041069463046F6F789FD4FF4407000908D
:103410008DF804408DF8065003208DF805008DF8D6
:10342000074069463046F6F779FD61023046F6F707
:10343000C8FD7CBD000802402DE9F0410024FFF7E3
:10344000C3FF00214FF4E13000F070F8FFF762FF96
:1034500000F04EF824480023037083704370C3705B
:10346000022181600373837301264673C6734FF490
:103470007A7141611D4A04EB440102EB8100A0F521
:10348000447000F50050037083704670C67002EB04
:10349000011505F58055D5F8D41B01EB81014900D4
:1034A000816095F8D21BA0F54F60022909D004294C
:1034B00001D0052911D1101900F5805080F8E33CA6
:1034C0000BE03121171907F5805787F8E31CD5F871
:1034D000D41B64256943C0F8F81C641CE4B2052CB5
:1034E000C9D3BDE8F0810000DC2F0020A412002029
:1034F00038B545208DF8000002208DF80100012428
:103500008DF802408DF80340684600F055F84720DA
:103510008DF800008DF8014000208DF802008DF834
:103520000340684600F048F838BD00007FB50C46FF
:1035300005460121202004F0F1FB00204FF48051CA
:103540000095012C03D0022C06D064B10FE0ADF839
:1035500004104FF4806103E0ADF804104FF4C06133
:10356000ADF8081003E0ADF80400ADF80800ADF8C0
:103570000400ADF80600ADF80C000C200D4CADF8C1
:103580000A006946204607F0EBF80121204607F0C3
:1035900050F8012240F22441204607F0C9F81021DA
:1035A000204607F043F80122C021204607F04BF8DF
:1035B0007FBD00000014014030B50F23C2780178B0
:1035C0000125FAB1144A126801F1E02102F4E06227
:1035D000C2F5E062C2F30722C2F10404D34042788C
:1035E000A24084781C401443220181F80024007812
:1035F00000F01F018D404009800000F1E020C0F87C
:10360000005130BD01F01F0085404809800000F1E5
:10361000E020C0F8805130BD0CED00E0024A1140BE
:10362000014302480160704780FFFF1F08ED00E082
:1036300010B50021074B0A46002003EBC004401CD4
:10364000C0B262548028F8D3491CC9B20829F3D308
:1036500010BD0000237E00202DE9FE4F0026171A22
:103660008146701E3546A3EB010A8846002F02DD15
:103670004FF0010102E003D14FF00001019102E09F
:10368000C7F100070190BAF1000F02DD4FF0010011
:1036900002E003D14FF00000009002E0C7F1000A01
:1036A00000905046574501DD3C4600E00446601C52
:1036B0004FF0000B029016E008F0FF0109F0FF0048
:1036C0000C9A00F015F83E445544A64202DD0199DB
:1036D000361B8944A54202DD00992D1B88440BF15D
:1036E00001001FFA80FB02998B45E5DBBDE8FE8FE8
:1036F00030B5CC0801F0070301259D40EBB2064D23
:1037000005EBC005C808285C0AB1184302E063EA6B
:103710000000C043285530BD237E00202DE9FC4128
:1037200001210A2004F0BEFA01248DF8044000268D
:103730004FF4C0508DF80660032700908DF8057097
:103740008DF8074069464648F6F7E8FB8DF80440D7
:103750008DF806608DF80570A5028DF80740414C84
:10376000009569462046F6F7D9FBC82008F04EFCC4
:1037700029462046F6F725FCC82008F047FC2946D4
:103780002046F6F720FCC82008F040FC0021FD2070
:1037900000F054FA0021122000F050FA0021AE206F
:1037A00000F04CFA0021D52000F048FA0021A020BA
:1037B00000F044FA0021A82000F040FA00213F2048
:1037C00000F03CFA0021D32000F038FA002108462E
:1037D00000F034FA0021402000F030FA0021A0204F
:1037E00000F02CFA0021C02000F028FA0021DA2095
:1037F00000F024FA0021122000F020FA002181209C
:1038000000F01CFA00217F2000F018FA0021D920D6
:1038100000F014FA0021822000F010FA0021DB20D1
:1038200000F00CFA0021342000F008FA0021A42056
:1038300000F004FA0021A62000F000FA0021202068
:1038400000F0FCF90021084600F0F8F9FFF7F0FE5F
:103850000021AF2000F0F2F900F054F8BDE8FC813F
:10386000000C0240000402400346012000E05843DF
:10387000491EC9B2FBD270472DE9F84F82460A981B
:103880000D4650436421B0FBF1F0984600F0FF0B69
:103890004FF001090AEB02072B4600245046FAB20A
:1038A0001946CDF80090FFF7D7FE05EB0806F3B2F6
:1038B000FAB2F1B25046CDF80090FFF7CDFE524675
:1038C000F3B229461046CDF80090FFF7C5FEF3B2DB
:1038D000FAB2F8B22946CDF80090FFF7BDFE4F4688
:1038E0000AEB0B0609E02819C3B2C1B2F2B2504686
:1038F0000097FFF7B1FE641CE4B24445F3D3BDE882
:10390000F88F000070B50025B020294600F096F928
:103910000021084600F092F90021102000F08EF9F5
:10392000084E002406EBC4000121405D00F086F93A
:10393000641CE4B2802CF5D36D1CEDB2082DF0D3DD
:1039400070BD0000237E002070B50B4C054602219F
:10395000204604F071FB0028F9D02946204604F0E7
:1039600074FB0121204604F067FB0028F9D02046B3
:1039700004F069FBC0B270BD003800402DE9FC4F77
:103980001D46884681468B460090082B0ED068075E
:1039900000D0012000EBD500690810FB01F0C0B297
:1039A000203A02F0FF0A0026019046E00620F7E7E1
:1039B000082D10D00C2D14D0102D16D0182D3FD15D
:1039C00021490AEBCA0001EB80000027845DE00773
:1039D0000FD00B9A10E01D490AEB4A0001EB4000A2
:1039E000F3E70AEB4A001A49EDE71A4901EB0A101E
:1039F000EBE70B9830B3002241464846FFF778FECC
:103A00007F1C640808F10100FFB200F0FF08082FD6
:103A1000DDD309F1010000F0FF09082D0AD000995B
:103A2000A9EB0100B0EB550F04D10BF1080089465A
:103A300000F0FF0B761CD846F6B201988642B7D349
:103A4000BDE8FC8F0122D7E728DE01089CD10108E0
:103A5000C4D3010838D801082DE9FF4F81B04FF0D9
:103A60000005DDE90F7ADDF838B05FEA030980462A
:103A70002E4612D10398F4F7B5FD41EC100B07F078
:103A8000E7F89FED331B51EC100B53EC112BF4F7BF
:103A900010FCF4F7C8FD00F0FF09082F00D1022543
:103AA000D94510D8BBF1000F0DD03B463022CDF8E0
:103AB00000A040460299FFF761FF05EB570101EBBB
:103AC000080000F0FF08002431E0A9EB0B01A1423F
:103AD0000DD105EB570101FB0480C0B23B462E22FD
:103AE000CDF800A00299FFF749FF01261DE0001B59
:103AF000401EC1B20A20FFF7B7FE0399CDF800A01F
:103B0000B1FBF0F00A21B0FBF1F201FB120106EB70
:103B10000800A1B105EB570202FB04003031C0B22E
:103B2000CAB23B460299FFF729FF641CE4B209EBD5
:103B30000600A042C9D805B04846BDE8F08F05EBA5
:103B4000570101FB0400C0B23B463022EAE7000007
:103B5000000000000000F03F2DE9FF4F81B0064655
:103B600000900F464FF0000A8946580700D0012008
:103B700000EBD3000490002032E0002029E00E98F2
:103B8000002410F80A500AF101001FFA80FAE80731
:103B900001D00F9A02E00F9848B300223946304610
:103BA000FFF7A6FD7F1C641C6D08E4B2FFB2082C71
:103BB000EDD3761C0098F6B2311A0398814204D1F5
:103BC00009F10800009E00F0FF0908F101004F46CE
:103BD000C0B2039980468842D1D30BF10100C0B234
:103BE000049983468842C8D305B0BDE8F08F01220E
:103BF000D4E72DE9F8431D46DDE9087816468946E5
:103C000004460EE03B4649462046CDF80080FFF7CB
:103C1000B5FE082F0ED004EB5700C4B26D1EEDB2F6
:103C2000761C002D04D03278202A01D37E2AE9D9CF
:103C3000BDE8F883A41DE4B2F0E700002DE9F041EF
:103C4000114C06464FF4006500292946204602D053
:103C5000F6F7B9F901E0F6F7B4F94FF480573946B1
:103C60002046F6F7AEF939460848F6F7ACF9304683
:103C7000FFF76AFE39462046F6F7A5F929462046A1
:103C8000BDE8F041F6F79FB9000C02400004024085
:103C90002DE9F04F8BB04FF000094F46ADF8009082
:103CA000ADF80490ADF80890ADF80C90ADF8109018
:103CB000ADF81490F74C4D4694F8E206A4F5805AFE
:103CC0000106F54E0AF580404FF0010B069001F118
:103CD000B28701F0B8BF94F8A607022805D194F87E
:103CE000A50710B10720ADF81400BDF8140030444A
:103CF0008079BDF814103144C97840EA0160BDF8FC
:103D0000141031440979BDF8142009043244527961
:103D100041EA02210843E1494A6890424DD0486097
:103D2000BDF8140030448078BDF81410314449784F
:103D300040EA0125B4F86A16BDF814002844801C36
:103D400081423AD3B4F86A06BDF81410401B401AF9
:103D5000801EA4F86A06BDF8140029463044F5F721
:103D600067FABDF81410294431444978BDF814208D
:103D70002A44B25C41EA0221814241F0418794F831
:103D8000E80340B1A81C81B2BDF8140001233044FF
:103D90000422F6F73BF9BDF814003044007900F036
:103DA00001000890BDF81400304480790023C0F36E
:103DB0004200A5F10708079012E0A4F86A760BB05C
:103DC000BDE8F08F18443044C079DDE90721F5F7EC
:103DD00031FCBDF8141019443144C8715B1C9BB20E
:103DE000BDF814004345EDDB3044C07984F8A4B736
:103DF000C4F8A87684F8A676069981F87674C1F896
:103E0000787494F8A617032903D094F8A61701290B
:103E100002D1A34AC2F888B2ADF80C7012287DD046
:103E20000CDCA0F10B00072817D2DFE810F04B0BD9
:103E3000AD0BE90BE30BFA0D2100AD0CA2286FD0FE
:103E400007DC14286DD0152801F06286A12804D162
:103E50002EE3A32866D0A42865D00020BDF8141056
:103E600001447754401C80B20528F7D301F0C3BE4B
:103E7000ADF80070F5E1BDF80000D04600EB400160
:103E800001EB00100AEB001000F5805090F85A0D7D
:103E900008287DD2DFE800F07C040404047CA70439
:103EA000ADF804708CE0BDF81400BDF80C2010448F
:103EB0003044007A98B3012802D0022876D113E06A
:103EC000BDF80000BDF8041000EB400202EB00104A
:103ED00008EB001000EB011041F686510844017810
:103EE00021F00401017061E0BDF8000000EB400228
:103EF00002EB0010BDF8042001EB001000EB0210F3
:103F000041F686521044027822F008020270BDF891
:103F1000000000EB400202EB001005E0FDE345E08D
:103F2000FCE3FCE3FCE3FCE3BDF8041008EB001049
:103F300000EB011000F58050C0F8887DBDF800103E
:103F40000220F5F70BFC00204346BDF8001001EB02
:103F5000011202EB012103EBC102BDF8041001EBD9
:103F6000011102EBC101014401F5005181F85B72BE
:103F7000401C80B21428E8D30020BDF8001001EBEB
:103F8000011202EB012103EBC102BDF8041000E0B5
:103F900062E101EB011102EBC101014401F50051A5
:103FA00081F87772401C80B20A28E6D3BDF80C0075
:103FB000401CADF80C00BDF80400401CADF8040036
:103FC000BDF8000000EB400101EB001008EB001011
:103FD00000F58050414690F85B0DBDF804209042FA
:103FE0003FF661AF38E1ADF8047023E1BDF814008D
:103FF000BDF80C2010443044007A042805D005DCBC
:1040000058B101284ED002287ED132E108287CD058
:1040100010287BD0202877D1E7E1BDF8000000EB25
:10402000001202EB002001EBC002BDF8040000EB1F
:10403000001002EBC00000F5005090F8920210282A
:1040400024D1BDF8000000EB001202EB002001EBD0
:10405000C002BDF8040000EB001002EBC00000F548
:10406000005080F89272BDF80000F32200EB0013BC
:1040700003EB002008EBC001BDF8040000EB0010CA
:1040800001EBC00000F5005080F82122BDF80C00C3
:10409000401CC8E0A4220020347400201802002034
:1040A00000004042BDF80000F22200EB001303EBD9
:1040B000002001EBC003BDF8040000EB001003EB8F
:1040C000C00000F5005080F82122BDF8000000EB90
:1040D000400202EB0010BDF8042001EB001000EBE1
:1040E000021041F686521044027822F00402027057
:1040F000BDF81400BDF80C2010443044027ABDF81D
:10410000000000EB001302E08FE0B2E0F1E003EB0F
:10411000002001EBC003BDF8040000EB001003EB2E
:10412000C00000F5005080F892220020BDF8142055
:10413000BDF80C301A4402443244537ABDF80020D2
:1041400002EB021C0CEB022201EBC20CBDF80420B6
:1041500002EB02120CEBC202024402F5005282F89A
:104160006532401C80B20F28E0D30020BDF8142037
:10417000BDF80C301A4402443244137EBDF80020CE
:1041800002EB021C0CEB022201EBC20CBDF8042076
:1041900002EB02120CEBC202024402F5005282F85A
:1041A0007732401C80B20A28E0D3BDF81400BDF875
:1041B0000C201044304490F82200BDF8002002EB9F
:1041C000021303EB022201EBC203BDF8042002EB51
:1041D000021203EBC20202F5005282F88C020020A8
:1041E000BDF81420BDF80C301A440244324492F851
:1041F0002330BDF8002002EB021C0CEB022201EB85
:10420000C20CBDF8042002EB02120CEBC202024405
:1042100002F5005282F88D32401C80B20528DFD3AF
:10422000BDF80C002030ADF80C00BDF80400401CB7
:10423000ADF80400BDF8000000EB400101EB0010F8
:1042400008EB001000F58050414690F85B0DBDF87A
:10425000042090423FF6CAAEBDF80000401CADF805
:10426000000094F8240BBDF8001088423FF603AE1E
:10427000FCE5BDF80000F22200EB001303EB002088
:1042800001EBC003BDF8040000EB001003EBC0001D
:1042900000F5005080F82122BDF8000000EB40023C
:1042A00002EB0010BDF8042001EB001000EB02103F
:1042B00041F686521044027822F004020270BDF8E2
:1042C0001400BDF80C2010443044027ABDF8000000
:1042D00000EB001303EB002008EBC001BDF8040065
:1042E00000EB001001EBC00000F5005080F89222B6
:1042F000CCE6BDF80000F32200EB001303EB002036
:1043000001EBC003BDF8040000EB001003EBC0009C
:1043100000F5005080F82122BDF8000000EB4002BB
:1043200002EB0010BDF8042001EB001000EB0210BE
:1043300041F686521044027822F004020270BDF861
:104340001400BDF80C2010443044027ABDF800007F
:1043500000EB001303EB002001EBC003BDF80400E9
:1043600000EB001003EBC00000F5005080F8922233
:10437000BDF81400BDF80C2010443044427ABDF85A
:10438000000000EB001303EB002001EBC003BDF8BD
:10439000040000EB001003EBC00000F5005080F8B3
:1043A0008C220020BDF81420BDF80C301A440244C1
:1043B0003244937ABDF8002002EB021C0CEB02227F
:1043C00001EBC20CBDF8042002EB02120CEBC2029E
:1043D000024402F5005282F88D32401C80B205285A
:1043E000E0D3BDF80C00C01D1DE7BDF80000F222AF
:1043F00000EB001303EB002001EBC003BDF8040049
:1044000000EB001003EBC00000F5005080F8212203
:10441000BDF8000000EB400202EB0010BDF80420E4
:1044200001EB001000EB021041F6865210440278B6
:1044300022F004020270BDF81400BDF80C201044F4
:104440003044027ABDF8000000EB001303EB0020BB
:1044500001EBC003BDF8040000EB001003EBC0004B
:1044600000F5005080F892220020BDF81420BDF81D
:104470000C301A4402443244537ABDF8002002EB57
:10448000021C0CEB022201EBC20CBDF8042002EB73
:1044900002120CEBC202024402F5005282F88D3285
:1044A000401C80B20428E0D3BDF80C00401DBAE6E1
:1044B000A81E0D2190FBF1F0C0B20990ADF800707C
:1044C00009E2B846ADF80470DFE1BDF80000BDF8C0
:1044D000041000EB400202EB00120AEB021000EBAA
:1044E000011000F5805090F8860D80077ED409EB0E
:1044F000890101EBC900BDF8141008443044007A6A
:104500000021FDF70DFBBDF80020BDF804C002EB53
:10451000420303EB021352460AEB031303EB0C13A3
:1045200003F5805393F8843D434088EA0100034338
:104530005CD1BDF8000000EB001101EB002002EBA4
:10454000C001BDF8040000EB001001EBC00000F555
:10455000005090F8590201287ED1BDF81400304473
:10456000417ABDF8000000EB001303EB00200AEBDA
:10457000C002BDF8040000EB001002EBC00000F523
:10458000005080F82212BDF814003044407BBDF882
:1045900014103144897A40EA0161BDF814003044B6
:1045A000C07ABDF8142000043244127B40EA022095
:1045B0000143BDF8000000EB001202EB0022BDF841
:1045C00004000AEBC20200EB001002EBC00000F591
:1045D0000050C0F82412BDF814003044007DBDF82E
:1045E00014103144497C40EA016000E048E1BDF824
:1045F00014103144897CBDF8142009043244D27C63
:1046000041EA02210843BDF8001001EB410202EB30
:1046100001120AEB0211BDF8042001EB021101F5B1
:104620008051C1F8880DBDF8000000EB400101EB9E
:1046300000110AEB0110BDF8041000EB011041F667
:1046400086510844017841F020010170BDF8001046
:104650000220F5F783F800E089E0BDF8000000EBE8
:10466000400101EB00110AEB0110BDF8041000EB52
:10467000011000F5805090F8841DBDF8000000EB9B
:10468000001202EB00220AEBC20000F5005080F895
:104690001512BDF8000000EB400101EB00110AEB20
:1046A000011000F5805090F85A0D012806D002281C
:1046B00060D003285ED0072859D114E1BDF800006E
:1046C00000EB001101EB00200AEBC002BDF8040072
:1046D000514600EB001002EBC00000F5005090F8CE
:1046E000220210B1012842D142E0BDF8000000EBE7
:1046F000400202EB001001EB001000F5805090F832
:10470000600D0028BDF8000000EB001202EB002055
:1047100001EBC002BDF8040004E0FCE327E2FBE388
:10472000A0E30BE100EB001002EBC00000F500502D
:10473000D0F8240203D0B0F1104F03D104E0B0F55B
:10474000100F01D0B52200E0C322BDF8000000EB3D
:10475000001303EB00200AEBC001BDF8040000EBDE
:10476000001001EBC00000F5005080F8212280E02D
:10477000B922EAE7BDF80000524600EB001101EB58
:1047800000200AEBC001BDF8040000EB001001EBB3
:10479000C00000F5005090F81C12BDF8000000EBBE
:1047A000001303EB00200AEBC00000F5005090F866
:1047B000180281425DD1BDF814003044807BBDF801
:1047C000141000043144C97B40EA0121BDF81400F3
:1047D0003044007C0143BDF8000000EB001303EB04
:1047E000002002EBC003BDF8040000EB001003EB57
:1047F000C00000F50050C0F85012BDF8140030445D
:10480000417ABDF8000000EB001303EB002002EB3F
:10481000C003BDF8040000EB001003EBC00000F57E
:10482000005080F82212BDF80000A42100EB001314
:1048300003EB002002EBC003BDF8040000EB001006
:1048400003EBC00000F5005080F81E12BDF8000018
:10485000A32100EB001303EB00200AEBC002BDF81C
:10486000040000EB001002EBC00000F5005080F8DF
:10487000211209F10100099900F0FF09894515D2BB
:10488000BDF80400401CADF80400BDF8000000EBCA
:10489000400101EB00100AEB001000F5805090F889
:1048A0005B0DBDF8042090423FF60FAEBDF800004E
:1048B00000EB400101EB00110AEB011000F5805004
:1048C00090F85B0DBDF8041088427CD8BDF800005C
:1048D000401CADF8000094F8240BBDF8001088428D
:1048E0003FF6EFADC4E4BDF8000000EB400101EB82
:1048F00000100AEB001000F5805090F8600D0028C1
:10490000BDF8000000EB001202EB00200AEBC00231
:10491000BDF8040000EB001002EBC00000F50050F1
:10492000D0F8240203D0B0F1104F05D002E0B0F56A
:10493000100F01D05A4608E7052206E7ADF80070CF
:104940004BE0ADF80470B84620E0BDF814003044E8
:10495000007A0021FDF7E4F8BDF8002002EB4203E5
:1049600003EB02130AEB0312BDF8043002EB03124F
:1049700002F5805292F8842D424088EA01000243F9
:1049800032D0BDF80400401CADF80400BDF80000B2
:1049900000EB400101EB00110AEB011000F5805023
:1049A00090F85B0DBDF804108842CED8BDF8000029
:1049B00000EB400101EB00110AEB011000F5805003
:1049C00090F85B0D00E099E1BDF80410884289D8A9
:1049D000BDF80000401CADF8000094F8240BBDF8B1
:1049E00000108842ADD843E4BDF80000BDF80420B3
:1049F00000EB400101EB001051460AEB001000EB08
:104A0000021000F5805090F8842DBDF8000000EBF6
:104A1000001303EB00200AEBC00000F5005080F803
:104A20001522BDF8000000EB400202EB00100AEB7B
:104A3000001000F5805090F85A0D012806D0022889
:104A400006D0032839D00728B0D17CE0CA227BE009
:104A5000BDF8000000EB001202EB002001EBC002E9
:104A6000BDF8040000EB001002EBC00000F50050A0
:104A700090F81C22BDF8000000EB001303EB0020AF
:104A800001EBC00000F5005090F8180282428DD171
:104A9000BDF80000AA2200EB001303EB002001EB9D
:104AA000C003BDF8040000EB001003EBC00000F5EC
:104AB000005080F81E22A32246E0BDF8000000EB63
:104AC000001202EB002001EBC002BDF8040000EB75
:104AD000001002EBC00000F5005090F81C22BDF859
:104AE000000000EB001303EB002001EBC00000F519
:104AF000005090F81802824225D1BDF80000AA2289
:104B000000EB001303EB002001EBC003BDF8040031
:104B100000EB001003EBC00000F5005080F81E22EF
:104B2000BDF80000A32200EB001303EB002001EB13
:104B3000C003BDF8040000EB001003EBC00000F55B
:104B4000005080F821220422BDF8000000EB001381
:104B500003EB00200AEBC001BDF8040000EB0010DD
:104B600001EBC00000F5005080F821221EE7ADF8EF
:104B7000007049E0ADF80470B84620E0BDF81400BC
:104B80003044007A0021FCF7CBFFBDF8002002EB97
:104B9000420303EB02130AEB0312BDF8043002EBED
:104BA000031202F5805292F8842D424088EA0100F7
:104BB000024330D0BDF80400401CADF80400BDF83D
:104BC000000000EB400101EB00110AEB011000F5C1
:104BD000805090F85B0DBDF804108842CED8BDF827
:104BE000000000EB400101EB00110AEB011000F5A1
:104BF000805090F85B0DBDF8041088427ED8BDF857
:104C00000000401CADF8000094F8240BBDF8001023
:104C10008842AFD866E6BDF80000BDF8042000EB7E
:104C2000400101EB001051460AEB001000EB0210AE
:104C300000F5805090F8842DBDF8000000EB0013C3
:104C400003EB00200AEBC00000F5005080F81522AD
:104C5000BDF814003044407ABDF8142000043244FA
:104C6000927A40EA0222BDF814003044C07A02432E
:104C7000BDF8000000EB001303EB002001EBC003C4
:104C8000BDF8040000EB001003EBC00000F500507D
:104C9000C0F85022BDF8000000EB400202EB00100B
:104CA00001EB001000F5805090F85A0D082896D2BC
:104CB000DFE800F004053C3C830404B68FE7BDF850
:104CC000000000EB001202EB002001EBC002BDF877
:104CD000040000EB001002EBC00000F5005090F85B
:104CE0001C22BDF8000000EB001303EB002001EBD9
:104CF000C00000F5005090F8180200E01DE3824269
:104D0000DCD1BDF80000B22200EB001303EB002061
:104D100001EBC003BDF8040000EB001003EBC00082
:104D200000F5005080F81E22E52233E0BDF80000B7
:104D300000EB001202EB002001EBC002BDF8040002
:104D400000EB001002EBC00000F5005090F81C22B0
:104D5000BDF8000000EB001303EB002001EBC000E6
:104D600000F5005090F818028242A7D1BDF800006B
:104D7000A52200EB001303EB002001EBC003BDF8FC
:104D8000040000EB001003EBC00000F5005080F8B9
:104D90001E22A322BDF8000000EB001303EB00204D
:104DA0000AEBC001BDF8040000EB001001EBC000ED
:104DB00000F5005080F8212211E7BDF8000000EB5B
:104DC000001202EB002001EBC002BDF8040000EB72
:104DD000001002EBC00000F5005090F81C22BDF856
:104DE000000000EB001303EB002001EBC00000F516
:104DF000005090F81802824212D1BDF80000B5228E
:104E000000EB001303EB002001EBC003BDF804002E
:104E100000EB001003EBC00000F5005080F82122E9
:104E2000BDF8000000EB001202EB002001EBC00215
:104E3000BDF8040000EB001002EBC00000F50050CC
:104E400090F81C22BDF8000000EB001303EB0020DB
:104E500001EBC00000F5005090F818028242ABD17F
:104E6000022297E7BDF814003044007A0528BDF807
:104E700014003044007A7CD2401EADF800000020BF
:104E8000BDF8001001EB410202EB01110AEB011128
:104E900001EB001101F5805181F8847DBDF800100F
:104EA00001EB410303EB01110AEB011101EB0011CE
:104EB00001F5805181F8857DBDF8001001EB4103BB
:104EC00003EB01110AEB011101EB001101F5805117
:104ED00081F88C7D401C80B21028D1D3BDF814001D
:104EE0003044807B0021FCF71BFE08437ED0BDF8D8
:104EF00014003044407ABDF8141000043144897A1B
:104F000040EA0120BDF814103144C97A0843C117A2
:104F1000FCF706FE01E0FDE3FDE3BDF8001001EB48
:104F2000410202EB01120AEB021101F58051C1F8B6
:104F3000540DBDF814003044007BB8460021FCF746
:104F4000EFFDBDF8001001EB410202EB01120AEB8C
:104F5000021101F5805181F8580DBDF8140030445C
:104F6000407B0021FCF7DCFDBDF8001001EB4102A5
:104F700000E0E3E102EB01120AEB021101F58051BE
:104F800081F8590DBDF814003044807B0021FCF7F6
:104F9000C7FDBDF8001001EB410202EB01120AEB64
:104FA000021101F5805181F85A0DBDF8140030440A
:104FB000C07B0021FCF7B4FDBDF8001001EB4102FD
:104FC00002EB01120AEB021101F5805181F85B0D31
:104FD000BDF814003044007C0021FCF7A1FDBDF8B1
:104FE000001001EB410202EB011200E0E5E00AEBE8
:104FF000021101F58051C1F85C0DBDF81400304478
:10500000407C0021FCF78CFDBDF8001001EB410253
:1050100002EB01120AEB021101F5805181F8600DDB
:10502000BDF8000000EB400101EB00110AEB01109C
:1050300000F5805090F85A0DADF804800628D0464F
:105040005CD0A9E0BDF81400BDF804100844304459
:10505000807C0021FCF764FDBDF804200321B2FB35
:10506000F1F2BDF8001001EB410303EB011308EB73
:10507000031101EB021101F5805181F8840DBDF897
:105080001400BDF8041008443044C07C0021FCF733
:1050900047FDBDF804200321B2FBF1F2BDF800107A
:1050A00001EB410303EB011308EB031101EB0211C8
:1050B00001F5805181F8850DBDF81400BDF804108C
:1050C00008443044007D0021FCF72AFDBDF804208F
:1050D0000321B2FBF1F2BDF8001001EB410303EB39
:1050E000011308EB031101EB021101F5805181F866
:1050F0008C0DBDF80400C01CADF80400BDF8000024
:1051000000EB400101EB001108EB011000F58050AD
:1051100090F85B0DBDF8041000EB4000884291D878
:105120004BE0BDF81400BDF8041008443044807C06
:105130000021FCF7F5FCBDF8001001EB410202EB89
:10514000011208EB0211BDF80420520801EB021114
:1051500001F5805181F8840DBDF81400BDF80410EC
:1051600008443044C07C0021FCF7DAFCBDF8001094
:1051700001EB410202EB011208EB0211BDF8042021
:10518000520801EB021101F5805181F8850DBDF83F
:105190000400801CADF80400BDF8000000EB4001E5
:1051A00001EB001108EB011000F5805090F85B0D49
:1051B000BDF80410B1EB400FB3D3BDF804001230BA
:1051C00085427DD9BDF8000000EB400101EB0010E5
:1051D0000AEB001000F58050514690F85A0D012856
:1051E00037D0BDF8000000EB400202EB001001EBED
:1051F000001000F5805090F85A0D032829D0BDF812
:10520000000000EB400202EB001001EB001000F583
:10521000805090F85A0D02281BD0BDF8000000EB1A
:10522000400202EB001001EB001000F5805090F8F6
:105230005A0D07280DD0BDF8000000EB400202EB2C
:10524000001001EB001000F5805090F85A0D042872
:105250005FD1BDF814002844304410F8020C00F06F
:105260000F00042814D2BDF8000000EB400202EB4E
:10527000001001EB001241F670501044BDF81420EC
:105280002A44324412F8022C037862F301030370BB
:10529000BDF814002844304410F8012C0420B0EB71
:1052A000121F17D9BDF8000000EB400202EB0010FE
:1052B00001EB001241F670501044BDF8142000E0DC
:1052C00027E02A44324412F8012C1309027863F3D0
:1052D00083020270BDF814002844304410F8010C19
:1052E00000F00F00042814D2BDF8000000EB4002CB
:1052F00002EB00100AEB001141F670500844BDF8B3
:1053000014102944314411F8012C017862F305117D
:105310000170BDF800100220F4F720FABDF800007B
:10532000C0B2FDF7CFF8BDF8000000EB40020AEB79
:10533000820000F5805080F8B1B624E20528FCD147
:10534000BDF814000930ADF80C00BDF80C00305C5D
:1053500084F8C80BBDF80C00401CADF80C00ADF88B
:105360000070A1E0BDF80C00305C0021FCF7D8FB18
:10537000BDF8001001EB41020AEB021101F580516A
:1053800081F8D30BBDF80C00401CADF80C00BDF843
:105390000C00305C0021FCF7C3FBBDF8001001EBF2
:1053A00041020AEB021101F5805181F8D20BBDF8E0
:1053B0000C00401CADF80C00BDF80C00305CBDF8D2
:1053C0000C1000043144497840EA0120BDF80C106B
:1053D000314489780843C117FCF7A2FBBDF80010DF
:1053E00001EB41020AEB021101F58051C1F8CC0B2F
:1053F000BDF80C00C01CADF80C00BDF80C00305C12
:105400000021FCF78DFBBDF8001001EB41020AEB17
:10541000021101F5805181F8D00BBDF80C00401C41
:10542000ADF80C00BDF80C00305C0021FCF778FBF7
:10543000BDF8001001EB41020AEB021101F58051A9
:1054400081F8D10BBDF80C00401CADF80C00BDF884
:105450000C00305C0021FCF763FBBDF8001001EB91
:1054600041020AEB021101F58051C1F8D40BBDF8DD
:105470000C00401CADF80C00BDF80C003044407826
:10548000BDF80C10715C40EA0120BDF80C10891CBD
:10549000ADF80C10BDF80C100844ADF80C00BDF8C8
:1054A0000000401CADF8000094F8C80BBDF80010D7
:1054B00088423FF657AF00210A20F4F74FF9FDF775
:1054C000BBFF98E3BDF814003044007A84F8EE0383
:1054D000BDF814003044407A84F8ED03BDF81400A0
:1054E0003044807A84F8EC03BDF814003044C07A6C
:1054F00084F8EB03BDF814003044007B84F8EA0321
:10550000BDF814003044407B84F8E90304F2E93428
:10551000F4F746F8F4F708F82078A4F2E934FF2805
:1055200029D1F3F7B7FFBDF814003044007A84F8AE
:10553000EE03BDF814003044407A84F8ED03BDF862
:1055400014003044807A84F8EC03BDF81400304431
:10555000C07A84F8EB03BDF814003044007B84F873
:10556000EA03BDF814003044407B84F8E903F4F703
:1055700017F8F3F7D9FFDAF8580008B10F2000E068
:105580000E2084F8A80736E3102084F8A807BDF899
:1055900014003044007A84F8EE03BDF8140030445F
:1055A000407A84F8ED03BDF814003044807A84F822
:1055B000EC03BDF814003044C07A84F8EB03BDF866
:1055C00014003044007B84F8EA03BDF81400304432
:1055D000407B84F8E90304F2E934F3F7E1FF02F0D9
:1055E0000BFCC4F80700D4F80700D4F80700A4F2B5
:1055F000E93400E30E2084F8A80784F8E171FAE2A8
:10560000ADF8007050463EE0ADF8047016E0BDF80D
:10561000001001EB410202EB0111BDF8042000EB88
:10562000011101EB021101F5805191F8861DC907A6
:1056300014D1BDF80410491CADF80410BDF80010D9
:1056400001EB410202EB011100EB011101F5805168
:1056500091F85B1DBDF804209142D8D8BDF8001028
:1056600001EB410202EB011100EB011101F5805148
:1056700091F85B1DBDF80420914208D8BDF80010D8
:10568000491CADF80010BDF800100429BCD3BDF8CA
:10569000001004296ED3FE4B5F70FE4AC2F888B238
:1056A000C2F888B294F8E611002975D00D2184F86B
:1056B000A817BDF814103144497ABDF814203244BB
:1056C000127A41EA0221ADF80810BDF814103144F5
:1056D000C97ABDF814203244927A41EA02215980F5
:1056E00000214FF4007CD046BDF81400084430443B
:1056F000027B08EB010000F5805080F8E721491C8F
:1057000089B26145F0D3E248408800F2FF3081B2AF
:10571000012001E041E0A5E1F3F716FA00283BD0B3
:1057200084F8E171DA48418864225143BDF80820C9
:10573000B1FBF2F184F8E01188F807B04188491C08
:1057400041804088BDF80810884225D994F8DC01D2
:1057500040F0010084F8DC0194F8DC0120F0060040
:10576000801C84F8DC01BDF80800A4F8DE010021EB
:1057700001204EE1102084F8A80794F8DC0140F0E5
:10578000800084F8DC0136E2BDF814003044007A71
:1057900084F8E1011120F4E694E0ADF80070504681
:1057A0003EE0ADF8047016E0BDF8001001EB4102D8
:1057B00002EB0111BDF8042000EB011101EB021115
:1057C00001F5805191F8861DC90714D1BDF8041068
:1057D000491CADF80410BDF8001001EB410202EBCA
:1057E000011100EB011101F5805191F85B1DBDF82D
:1057F00004209142D8D8BDF8001001EB410202EB21
:10580000011100EB011101F5805191F85B1DBDF80C
:105810000420914208D8BDF80010491CADF80010D2
:10582000BDF800100429BCD3BDF800100429AAD388
:10583000DFF85C8288F80170964AC2F888B2C2F834
:1058400088B294F8E611E9B3122184F8A817BDF8DC
:1058500014103144097A84F8E11194F8E111491ED9
:10586000ADF800100021BDF814200A443244537AE8
:10587000BDF8002002EB420C0CEB021200EB02120E
:105880000A4402F5805282F8623D491C89B20A2915
:10589000E9D3BDF814103144097DBDF81420324419
:1058A000D27C41EA0221ADF80810BDF81410314451
:1058B000897DBDF814203244527D41EA0221A8F8C6
:1058C000021000E05CE000214FF40073BDF814000A
:1058D00008443044C27D0AEB010000F5805080F896
:1058E000E721491C89B29942F0D3B8F80200BDF80B
:1058F000001000EB8120401E81B20320F3F724F951
:10590000F0B3B8F80210404664225143BDF80820B5
:10591000B1FBF2F184F8E01152468AF807B0B8F80A
:105920000210491CA8F80210B8F80210BDF808309F
:10593000994243D9002041F68D5CBDF8001001EB7F
:10594000410303EB011102EB011101EB0011614472
:105950000B7843F001030B70401C80B21028ECD38D
:10596000BDF8000000EB400101EB001002EB00105D
:1059700041F66C510844037843F00103037000E0E2
:1059800049E0BDF8000000EB400303EB001002EB20
:1059900000100844017821F00601891C0170BDF84F
:1059A0000810BDF8000000EB400303EB00100AEB09
:1059B000001000F58050A0F86E1D27E040880128F7
:1059C00029D1002041F68D5CBDF8001001EB4103A8
:1059D00003EB011102EB011101EB001161440B78A3
:1059E00023F001030B70401C80B21028ECD3BDF8EB
:1059F000000000EB400101EB00100AEB001041F643
:105A00006C510844017821F001010170BDF80010CB
:105A10000220F3F7A3FE1F48C0F88872C0F888720E
:105A2000E9E0DAF858000A21B0FBF1F0BDF81410F3
:105A30003144097A884214D1BDF814003044007A08
:105A40000028504603D0816D0A39816503E08765DF
:105A5000102084F8A80700210520F3F77FFE8AF8BC
:105A600007B0C8E000212022D44600200CEB4113EF
:105A700003EB000888F85B2F401C80B22028F7D386
:105A8000491C89B21429F0D3142184F8A81703E023
:105A90001802002000004242BDF814003044007A91
:105AA000ADF80800BDF814003044407AADF810009D
:105AB000BDF80800142801D9ADF80810BDF8100091
:105AC000202801D9ADF81020002118E000200CEBAF
:105AD00041180EE0BDF81020BDF8143001FB026241
:105AE00003441A44927A08EB000383F85B2F401CAE
:105AF00080B2BDF810209042ECD3491C89B2BDF8A9
:105B000008008142E2D300210720F3F727FE72E06C
:105B1000152084F8A807BDF814003044017A5046D7
:105B20008AF8201FBDF814103144097BBDF81420F9
:105B30003244527A41EA0261BDF814203244927A2A
:105B4000BDF8143012043344DB7A42EA03221143D5
:105B5000C0F8251FBDF814103144097CBDF814208D
:105B60003244527B41EA0261BDF814203244927BF8
:105B7000BDF8143012043344DB7B42EA03221143A4
:105B8000C0F8211FBDF814103144497CBDF8142021
:105B900009043244927C41EA0221BDF814203244C7
:105BA000D27C1143C0F8291FBDF814103144097D7F
:105BB00080F8461FBDF814103144497D80F8451F18
:105BC000BDF814103144897D80F8441FBDF81410CD
:105BD0003144C97D80F8431FBDF814103144097E5B
:105BE00080F8421FBDF814103144497E80F8411FEF
:105BF000022084F8DC0CB4F86A06E0B1002016E05C
:105C00000020BDF8141001447754401C80B20528D0
:105C1000F7D3FEF7D2B8BDF814102944014431443B
:105C20008978BDF814200244B154401C80B2B4F805
:105C30006A168142EFD8B4F86A0600287EF44BA8B1
:105C40000BB0BDE8F08F94F8A6074FF47A7830B126
:105C500001287DD002287CD003287BD118E294F85B
:105C6000E206C0F3C3000E2874D2DFE800F0F707A5
:105C700013F61F2B2B374D789BA7F5E4F6A1F748B9
:105C800006F064FB002865D094F8E20620F0780066
:105C90001030DAE0F2A1F14806F058FB0028F2D00B
:105CA00094F8E20620F078001830CEE0EDA1EB4841
:105CB00006F04CFB0028E6D094F8E20620F07800CD
:105CC0002830C2E0E7A1E54806F040FB0028DAD022
:105CD00094F8E20620F078003830B6E0E1A1DF4821
:105CE00006F034FB0028CED09AF80100182805D918
:105CF00094F8E20620F078005030A6E094F8E2062E
:105D000020F078004030A0E0D7A1D44806F01EFB78
:105D10000028B8D05246511901F5805181F82B77EF
:105D20006D1CADB2142DF6D30021431833441B79FA
:105D3000551805F5805585F83037491C89B20F296B
:105D4000F3D300210320F3F709FD94F8E20602E003
:105D500085E02EE16EE020F07800483002E2C4A138
:105D6000BE4806F0F3FA00288DD05246511901F5CD
:105D7000805181F8E4766D1CADB2142DF6D300216C
:105D8000431833445B79551805F5805585F8E93695
:105D9000491C89B20F29F3D394F8E20620F0780069
:105DA0005030DFE1AFA1AD4806F0D0FA00288ED028
:105DB00094F8E20620F07800583046E094F8AA07FC
:105DC00050B194F8E20620F07800603084F8E206E2
:105DD000C4F8807684F87EB6A7A1A04806F0B6FA8B
:105DE000002827D0C4F8807684F87EB63044417904
:105DF00000793039303841EA0010C117FBF790FEC6
:105E000084F8AA079EA1954806F0A0FA002811D0B0
:105E100031184A78302A06D34978305C3038303926
:105E200041EA001001E0305C3038C117FBF778FE22
:105E300084F8AB07A7E18BA1884806F087FA002811
:105E400009D094F8E20620F0780084F8E206C4F85D
:105E5000807684F87EB696E187E12FE128E194F818
:105E6000E206C0F3C3000D284CD2DFE800F00817AB
:105E7000232D3860078087F44B8D98003EE779A189
:105E8000764806F063FAE8B3C4F8807684F87EB604
:105E900094F8E20620F07800083063E179A195E0FB
:105EA000C4F8807684F87EB694F8E20620F0780094
:105EB000103057E16BA1694806F048FA10B3C4F8F6
:105EC000807684F87EB6AEE06FA1644806F03EFAB4
:105ED000C0B194F8E20620F078002030B5E764A164
:105EE0005E4806F033FA68B15246511901F5805107
:105EF00081F8E4766D1CADB2142DF6D30021431861
:105F0000334400E039E05B79551805F5805585F894
:105F1000E936491C89B20F29F1D3C4F8807684F898
:105F20007EB694F8E20620F0780028301AE152A1FB
:105F30004A4806F00BFA00B394F8AA1731B194F866
:105F4000E21621F07801303184F8E216C4F8807648
:105F500084F87EB63044417900793039303841EAEE
:105F60000010C117FBF7DCFD84F8AA070BE13DA187
:105F70003A4806F0EBF9002880D104E194F8E206F3
:105F800020F07800483060E736A1344806F0DEF9AA
:105F900010B394F8E20620F07800603055E731A1A4
:105FA0002E4806F0D3F9B8B194F8E20620F0780054
:105FB000D8E094F8E206C0F3C30005280CD2DFE86D
:105FC00000F003040CD438005EE726A1234806F055
:105FD000BDF900287FF464AFD5E0C4F8807684F87A
:105FE0007EB6B07971793038303940EA0110C11786
:105FF000FBF796FD84F8AA0721A1184806F0A6F938
:1060000088B131184A78302A06D34978305C303864
:10601000303941EA001001E0305C3038C117FBF73D
:106020007FFD84F8AB0794F8E20620F07800183082
:1060300098E094F8E20620F0800084F8E20694F8F4
:10604000E20620F0780084F8E206069880F876747C
:10605000C0F8787497E08EE061000000347400208E
:106060006F6B00004F4B0000494D45493A0000005E
:1060700049434349443A00004353513A0000000069
:106080002C0000002200000052454144590000004D
:1060900094F8E206C0F3C300092874D2DFE800F0E8
:1060A0000807060E051143536500FFE5F2E5E5E537
:1060B00094F8E20620F078000830C6E6AFF25C0102
:1060C00003E735A1364806F041F958B3C4F88076A5
:1060D00084F87EB6D046411931440A7908EB0501AF
:1060E00001F5805181F8AC276D1CADB2142DF2D3AF
:1060F0002AA12C4806F02AF958B1002142460B1873
:10610000134403F5805383F8AB77491C89B2022905
:10611000F5D394F8E20620F07800303084F8E206F7
:1061200088F807B02FE0AFF2C4011D4806F00EF961
:1061300048B3C4F8807684F87EB694F8E20620F07E
:10614000780038300EE0AFF2E401154806F0FEF8B2
:10615000C8B1C4F8807684F87EB694F8E20620F0E0
:106160007800403084F8E2060DE0AFF208110C48E8
:1061700006F0ECF838B194F8E20640F0800084F8BC
:10618000E206C4F88486A4F86A7600203754401CDE
:1061900080B26428FAD353E5444843502C000000F1
:1061A00034740020502A00202DE9F74F86B00020DB
:1061B000019081460090FF4D00212954401C80B27F
:1061C0006428F8D3FC4890F87614A0F5405431B315
:1061D00094F8A51719B3002180F8761494F8E20614
:1061E00020F0800084F8E20694F8A60728B1012880
:1061F0000ED0022806D0032811D194F8E20620F030
:1062000078000AE094F8E20620F07800203004E0FC
:1062100094F8E20620F07800583084F8E20694F80A
:10622000E206DFF898B300067ED594F8A6060128AA
:106230007BD194F8A407012877D10020E04F804655
:1062400000EB400101EB081007EB0010039000F594
:1062500080500026029061E0039800EB061505F5DA
:10626000805595F8860D000655D595F8860D40F0B9
:10627000040085F8860D95F8860D00074BD595F836
:10628000860D20F0080085F8860D0020C7F839003B
:1062900008EB081101EB082007EBC00006EB061124
:1062A00000EBC10AC64842F23D2151441022293078
:1062B00005F68455F1F7C9FF0AF5085050F8351F67
:1062C000C7F81D104068C7F821002878387742F2D7
:1062D000502050F80A00C7F82500BA480168C7F8EE
:1062E0003D108088A7F841006868C7F84300B86D82
:1062F00081B20220F2F728FC00210620F3F72EFAE3
:10630000B86D798B884202D2B86D401CB865002107
:106310000520F3F723FA761C0298B6B290F85B0DCD
:10632000B04299D8414601E0FEE31AE00220F3F7BB
:1063300015FA08F1010080B28046042880D394F851
:10634000A607032803D094F8A607012803D19E4985
:106350000020C1F88802002084F8A4070B2084F8EC
:10636000A807944E00203A3E307000980DE001F0EE
:1063700043FDC4F8F003D4F8F003C0F300400190EB
:10638000D4F8F003C0F3420000900028EFD094F856
:10639000A607022811D194F8A50770B185485521A8
:1063A0004FF007090170FD214170AA218170002181
:1063B000C17001716122427181717E49F52201F83B
:1063C00009200020D4F8F013C0F10302D200D1401C
:1063D000784A09EB00031A44D170401C80B20428AB
:1063E000F0D394F8A50720B17748D0F80802B0B9E7
:1063F00006E07048089A4844C27109F1080533E084
:106400006F48007858B194F8A607032807D094F88D
:10641000A607012803D0012084F8A606FBE36849FB
:10642000644B00200A1802F5805292F82B5709EBB2
:1064300000021A44D571401C80B21428F2D3002007
:106440000A1802F5805292F8EC5709EB00021A4440
:10645000D576401C80B20A28F2D303EB09000899D4
:1064600080F8251009F12605002DD7D0089884F86A
:10647000670608981021FF2212287CD009DCA0F1C1
:106480000B0007281BD2DFE800F01A1AFD0DFC1BD9
:10649000FB00A22813DA4FF05902142801D0152866
:1064A0000DD1B9E384F8A8174849424A00202E18B4
:1064B0000B5C9355401C80B20A28F8D30A35B0E330
:1064C00094F8DC01C00773D0012080F31388BFF378
:1064D0004F8F3F4801683F4A01F4E061114301607A
:1064E000BFF34F8FFEE700EB4001354B01EB0A1085
:1064F00003EB0016039606F5805696F85A0D03280E
:1065000018D096F85A0D012814D096F85A0D022882
:1065100010D096F85A0D04280CD096F85A0D07287A
:1065200008D096F85A0D05287ED096F85A0D062800
:106530007BD063E11F4901204855ED1CA8B202221F
:1065400004900A54401C80B21D220A54401C85B29B
:106550000020B6E0039800EB081101F5805191F896
:10656000840D144A50556D1C91F8863DA8B2135401
:10657000401C85B200E050E291F8860D400707D438
:1065800091F8860D000703D491F8860D80077AD51F
:106590000020D1F8883DC0F10307FF00FB404719F8
:1065A000D355401C80B20428F3D32D1DABB213E0A9
:1065B00027E1000052020020A4520020BC640240E7
:1065C000A41200208D260020000040425CC4010877
:1065D0000CED00E00400FA050AEB0A1505EB0A21B0
:1065E0000CEBC10508EB081105EBC101029100207D
:1065F00001F50051D1F83552C0F10307FF00FD400D
:10660000C718D555401C80B20428F3D31B1D9BB27C
:106610000020D1F83952C0F10307FF00FD40C71830
:10662000D555401C80B201E05DE08CE00428F0D339
:106630001B1D9BB20020D1F85052C0F10207FF0091
:10664000FD40C718D555401C80B20328F3D3DB1C8E
:106650009FB20025029901F50050D0F83D0201F5E6
:106660000051D1F84112C5F10502D200F1F7DBFD6E
:10667000FD49EA1988546D1CADB2062DEAD303E03A
:1066800074E107E252E119E0B81D87B200250299D2
:1066900001F50050D0F8450201F50051D1F849123A
:1066A000C5F10502D200F1F7BEFDEF49EA198854A1
:1066B0006D1CADB2062DEAD3B81D85B208F10100FC
:1066C00080B2DFF8A8C396F85B1D804641453FF6CF
:1066D00041AF0498E449049A281A1144030A01F8C6
:1066E000023D48708AE0E04E02207055ED1CADB2CC
:1066F000A84600211FE0481C074670556D1C5A181B
:1067000002F58052A8B292F885253254401C82B21C
:10671000002003EB01110D1805F5805595F89155F2
:1067200000EB020C06F80C50401C80B21028F2D38B
:10673000103295B2B9B294F884058842DBD80021B2
:1067400006EB080055E0C84F03207855ED1CA8B2B1
:10675000022180463954401C80B20E213954401C1D
:1067600085B200219E463DE0039800EB0110A0F5A4
:106770001F7000F5005002787A556D1CAAB285781A
:10678000BD54521C807895B2400729D50AEB0A1CEB
:106790000CEB0A220EEBC20201EB0113002002EB0C
:1067A000C302131803F5005393F85B3200EB050C9A
:1067B00007F80C30401C80B20A28F2D30A35ABB27D
:1067C0000020151805F5005595F8745200EB030CE0
:1067D00007F80C50401C80B20228F2D39B1C9DB2DB
:1067E000491C89B296F85B0D8842BDD8002107EBA1
:1067F000080000F8021DA5EB080141700AF1010034
:1068000080B294F8241B824651453FF66CAE94F852
:10681000C80B00287ED0AD1CADB2AA46002276E09F
:10682000924B02EB420003EB001101F5805191F80D
:10683000D20B04280FD18C4E70556D1CA8B20125C7
:106840003554401C9D1805F5805580B295F8315D92
:106850003554401C85B291F8D20B984602280DD0D1
:1068600002EB420000EB021003EB001000F5805039
:106870001E4690F85A0D052836D046E07A4E022082
:1068800070556D1C94F88415A8B23154401C80B228
:1068900012213154401C85B2002120E0481C0746DB
:1068A000705508EB010303F580536D1C93F8853593
:1068B000A8B23354401C83B2002008EB01152918FC
:1068C00001F5805191F8911500EB030C06F80C10BE
:1068D000401C80B21028F2D310339DB2B9B294F8A4
:1068E00084058842DAD810E05F49052048556D1CC0
:1068F000A8B201230B54401CB31803F5805380B297
:1069000093F8313D0B54401C85B2521C92B294F85E
:10691000C80B00E085E1904282D8534800225044E1
:1069200000F8022DA5EB0A0141707AE17078401C55
:1069300070707078052803D294F8DC01C00706D087
:1069400084F8A81794F8DC01C00704D005E00D20F6
:1069500084F8A80701E084F8E0217088010A424821
:106960004155718828444170AD1C5AE184F8A8173C
:1069700094F8E1013C4F78550022DFF8F0C06D1C1F
:106980003CE094F8E10102EB021600EB001101EB90
:1069900000200CEBC00000EBC60000F5805090F822
:1069A0000C0A012828D194F8E10100EB400101EB29
:1069B00000100CEB001000EB021000F5805090F876
:1069C000540C78556D1CABB2002094F8E11101EB2A
:1069D000011505EB01210CEBC10101EBC6010144DE
:1069E00001F5805191F80D1A1D187955401C80B29F
:1069F0000A28EAD30A339DB2521C92B294F8E101FC
:106A000000EB400101EB00100CEB001000F5805092
:106A100090F82B0C9042B4D803E17078401C707051
:106A2000707805280ED294F8E10100EB400303EBE7
:106A300000130E4800EB031000F5805090F83C0C5A
:106A4000C00715D084F8A81794F8E10100EB4001C5
:106A500001EB0011054800EB011000F5805090F8A3
:106A60003C0CC00708D009E052020020A41200200C
:106A7000122084F8A80701E084F8E02194F8E111DD
:106A8000F748415571882844090A4170718881701E
:106A9000ED1CC6E0DFF8CC83012188F80710D8F898
:106AA00058100A22B1FBF2F2ED494A55D8F85800C5
:106AB0006D1C0A2804D900204FF00A0A029003E056
:106AC000D8F858A00022029201F805A022206D1CDF
:106AD000485500266D1C96E0D8F8580038B1D8F813
:106AE0005800801B401E81B20220F1F7C1FF98F8C8
:106AF0001C00DB4948556D1CAAB20020D8F81D3097
:106B0000C0F10305ED00EB4085184B55401C80B2E9
:106B10000428F3D3121D92B20020D8F82130C0F11E
:106B20000305ED00EB4000E0C6E085184B55401C26
:106B300080B20428F1D3121D92B20020D8F825307B
:106B4000C0F10205ED00EB4085184B55401C80B2AA
:106B50000328F3D3D21C97B20025414651F8290FE0
:106B60004968C5F10502D200F1F75DFBBC49EA199D
:106B700088546D1CADB2062DEFD3BF1DBFB20025EA
:106B8000414651F8310F4968C5F10502D200F1F7CD
:106B90004AFBB349EA1988546D1CADB2062DEFD3F8
:106BA000BF1D98F84230B8B24146AD4A1354401C5C
:106BB00098F8413080B21354401C98F8403080B2AD
:106BC0001354401C98F83F3080B21354401C91F885
:106BD0003E3080B21354401C91F83D3080B21354C3
:106BE000401C83B20020D1F84350C0F10307FF00DE
:106BF000FD40C718D555401C80B20428F3D31B1D97
:106C0000761C9DB2B6B202990020B6EB0A0288410A
:106C1000FFF662AF05E0DAE084F8A8179048425525
:106C20006D1C8F49A5EB090601EB0900320A80466D
:106C30004270867000238A460BE009EB030101EBEA
:106C40000A07F879DDE90021F2F704FDF8715B1C11
:106C50009BB29E42F1DC94F8E80328B1B1B2404601
:106C600000230422F3F7D2F9B1B256464046F2F7B8
:106C7000DFFA010A71556D1CA9B27054491C94F8D1
:106C8000A6078DB202280DD194F8A50750B1681F50
:106C9000010AF170307181B2701D01F0F4F9705584
:106CA0006D1CADB2CBF8005001216F48F2F716FB16
:106CB00009B02846BDE8F08F94F8A6076B4B6C4FDF
:106CC00042F21076A3F18509A3F1870CA3F10B081A
:106CD000A3F1720A30B1012877D0022876D00328B8
:106CE00075D13FE394F8E206C0F3C3000E286ED2DC
:106CF000DFE800F0071422303E4D5C6E7D8C9BDD9A
:106D0000ECFF00261F4603E0B85DA855761CB6B21E
:106D10005648F1F7B8FAB042F6D83DE3002404E053
:106D200019F804002855641CA4B250488538F1F7BE
:106D3000AAFAA042F4D8C9E30024664603E0305D15
:106D40002855641CA4B249488738F1F79CFAA04240
:106D5000F5D8BBE3002404E018F804002855641CAF
:106D6000A4B242480B38F1F78EFAA042F4D8ADE352
:106D70003E4E00241C3E03E0305D2855641CA4B246
:106D80003A481C38F1F77FFAA042F5D89EE3374E17
:106D900000242D3E03E0305D2855641CA4B2334826
:106DA0002D38F1F770FAA042F5D88FE32C4E00246D
:106DB000323E03E0305D2855641CA4B228483238C6
:106DC000F1F761FAA042F5D880E3A0E0DFE1C5E089
:106DD000264E00243C3E03E0305D2855641CA4B2DE
:106DE00022483C38F1F74FFAA042F5D86EE31F4E27
:106DF0000024163603E0305D2855641CA4B21B48FD
:106E00001630F1F740FAA042F5D85FE3174E0024A0
:106E10000A3603E0305D2855641CA4B213480A30DA
:106E2000F1F731FAA042F5D850E394F8A5070F4ED8
:106E3000643E022811D00020315C2954401C80B2ED
:106E40000D28F9D33846F1F71EFA002250EA020164
:106E500028D000211346034C1FE000240EE0000060
:106E600052020020A4120020B8640240AFCB0108F7
:106E70009D290020305D2855641CA4B2F848F1F724
:106E800002FAA042F6D821E3661806F5805696F875
:106E9000F9666F187E73491C89B20E1A73EB0206ED
:106EA000F2DBFFE2EF48F1F7EEF984B20EE3EC4ECD
:106EB0000024853603E0305D2855641CA4B2E84800
:106EC0008530F1F7E0F9A042F5D8FFE2DFF89083D2
:106ED0000027A8F1150805E00BE018F80700E855B1
:106EE0007F1CBFB2DE481538F1F7CDF9B842F4D8AF
:106EF00012E2002704E01AF80710E9557F1CBFB220
:106F0000D7480E38F1F7BFF9B842F4D804E294F844
:106F1000E206C0F3C3000D2820D2DFE800F007200E
:106F20002D3C4B5A69788796F3F1F000CC4F002640
:106F3000FF1F03E0B85DA855761CB6B2C848C01F55
:106F4000F1F7A1F9B042F5D8CBF800600121C648AD
:106F5000F2F7C4F94FF47A70C4F88406CAE2002448
:106F6000C24E03E0305D2855641CA4B2BF48F1F75F
:106F70008AF9A042F6D8A9E2BC4E0024AF3603E05D
:106F8000305D2855641CA4B2B848AF30F1F77BF9E6
:106F9000A042F5D89AE2B54E00240A3603E0305DEF
:106FA0002855641CA4B2B1480A30F1F76CF9A0422C
:106FB000F5D88BE2AD4E0024153603E0305D285540
:106FC000641CA4B2A9481530F1F75DF9A042F5D8C8
:106FD0007CE2A64E0024203603E0305D2855641C78
:106FE000A4B2A2482030F1F74EF9A042F5D86DE2E4
:106FF0009E4E0024293603E0305D2855641CA4B25F
:107000009A482930F1F73FF9A042F5D85EE2974E51
:107010000024383603E0305D2855641CA4B2934840
:107020003830F1F730F9A042F5D84FE28F4E002406
:10703000563603E0305D2855641CA4B28B485630A8
:10704000F1F721F9A042F5D840E294F8A507874C62
:107050006334022816D00020215C2954401C80B2E1
:107060001428F9D33846F1F70EF90446002680A11A
:10707000384605F06BF954EA060135D00021431E6D
:107080007C4A17E0002603E0A05DA855761CB6B246
:1070900076486330F1F7F7F8B042F5D828E0571892
:1070A00007F5805797F8F97605EB010C8CF814700A
:1070B000491C89B29942F2DB22212B18D974641C35
:1070C00046F1000108E0131803F5805393F8F836F1
:1070D0002F183B75401C80B2031B76EB0103F2DBDB
:1070E00065A16048F1F7C3F85E48F1F7CCF886B2C5
:1070F000CBF8006001215C48F2F7F0F8FAE12FE0EC
:107100000FE0FFE7594E0024933603E0305D285529
:10711000641CA4B255489330F1F7B5F8A042F5D8F5
:10712000D4E1D4F8841640F2E930814207D194F8D2
:10713000E20620F07800603084F8E20601E0C4F84E
:107140008406474E0024193E03E0305D2855641C38
:10715000A4B243481938F1F796F8A042F5D8B5E142
:10716000424F0026A43703E0B85DA855761CB6B29E
:107170003E48A430F1F787F8B042F5D8CBF800606C
:1071800001213948F2F7AAF843F69820E4E694F88A
:10719000E206C0F3C300052861D2DFE800F0031463
:1071A0006F8BD100002084F8A707044604E018F88C
:1071B00004002855641CA4B229485930F1F763F83B
:1071C000A042F4D882E1002184F8A7170846295488
:1071D000401C80B26428FAD384F8A7172349002002
:1071E0005B390A5C2A54401C80B20828F9D3DFF8C6
:1071F000849041F26771002709EB010809E009EB6F
:10720000070000F5805090F86707E91908727F1CA5
:10721000BFB24046F1F737F8B842F0D82C20E91950
:10722000087209371FFA87F841F28F71002709EBBE
:10723000010A0AE009EB070000F5805090F88F176B
:1072400008EB0702A9547F1CBFB25046F1F71BF8A8
:10725000B842EFD808A10348F1F709F86BE005E15F
:107260004BCB010852020020B864024086CC0108D2
:107270002C000000A41200200D0A000000269F4FE1
:1072800003E0B85DA855761CB6B29C48F0F7FBFF4A
:10729000B042F6D8CBF8006001219948F2F71EF809
:1072A00094F8E20620F07800183084F8E2064FF4F3
:1072B000FA6051E694F8A507DFF840820228A8F1A9
:1072C00029084FF0000018D000212954401C80B23A
:1072D0006428FAD384F8A717002018F8001029545E
:1072E000401C80B20E28F8D33846F0F7CCFF0104DA
:1072F000090C20D00020834A1AE084F8A707002751
:1073000004E018F80710E9557F1CBFB27B48293804
:10731000F0F7B9FFB842F4D8CBF80070E4E01318E6
:1073200003F5805393F8F9362F18BB73401C80B2D5
:107330008842F4D38EE77448F0F7A5FF5946D2E0AF
:10734000DFF8B881002708F10C0804E018F80700FE
:10735000E8557F1CBFB269480C30F0F794FFB84283
:10736000F4D8D9E794F8E206C0F3C30009287DD227
:10737000DFE800F005202D3B4958679EAF0000264E
:107380001F4603E0B85DA855761CB6B25B48C2380C
:10739000F0F779FFB042F5D8CBF8006001215848EA
:1073A000F1F79CFF94F8E20620F07800083084F8AA
:1073B000E206CFE5002404E019F804002855641C17
:1073C000A4B25248F0F75FFFA042F5D87EE0002457
:1073D000664603E0305D2855641CA4B24B48801E0D
:1073E000F0F751FFA042F5D870E0002404E018F84F
:1073F00004002855641CA4B244487A30F0F743FFD7
:10740000A042F4D862E03D4E00246D3E03E0305DC2
:107410002855641CA4B239486D38F0F734FFA042F7
:10742000F5D853E0354E00245E3E03E0305D28552C
:10743000641CA4B231485E38F0F725FFA042F5D8AD
:1074400044E094F8A5072D4E973E022812D0002064
:10745000315C2954401C80B20F28F9D33846F0F72C
:1074600012FF0104090C3FF41DAD00E042E00020D2
:10747000244A15E0002403E0305D2855641CA4B2C2
:107480001E489738F0F7FFFEA042F5D81EE013180B
:1074900003F5805393F8F9362C18E373401C80B23F
:1074A0008842F4D3AFF230211748F0F7E0FEF9E458
:1074B000124E0024543E03E0305D2855641CA4B2F3
:1074C0000E485438F0F7DFFEA042F5D8CBF8004064
:1074D00010E600201AF800102954401C80B207283A
:1074E000F8D35946401E086001210548F1F7F6FE21
:1074F000C4F8846609B00020BDE8F08F71CC0108A3
:10750000B8640240A4120020520200202ACB0108D5
:1075100070B5164C40F224452946204603F0E9F8A0
:10752000002821D02946204603F080F8104D002184
:107530002846F1F7D3FE61102846F1F7B9FE0D4950
:10754000012081F8A7072088A088281D0268C2F5BD
:10755000FA62A1F86A264FF4FA6101602846BDE894
:1075600070400121F1F7BABE70BD0000001001406B
:1075700088640240A422002010B5074C054920462B
:10758000F1F796FE00212046F1F7A8FE03490120FD
:10759000087010BD00800028B86402401802002066
:1075A0002DE9F04301218FB0880500F07BFBDFF867
:1075B00094904846F1F79CFE40200501039000247A
:1075C000CDE90545C60207940894CDE909464FF078
:1075D00000681E480B940C940D941B4FCDF800804E
:1075E0000E94CDE9017069464846F1F729FF012262
:1075F00010214846F1F70EFFDFF84890A9F1300955
:107600004846F1F775FE4FF4FA60CDE90340CDE945
:10761000054507940894CDE909460D480B940C9450
:107620000D94CDF800800E94CDE90170694648466E
:10763000F1F706FF01214846F1F750FE0FB0BDE813
:10764000F0830000B86402400410014052020020A0
:10765000347400207CB50121032000F023FB164E7A
:10766000072206213046F2F795FC072211463046E4
:10767000F2F790FC02218DF8051000258DF80650D8
:107680000124C0208DF8074000908DF80410694651
:107690003046F2F743FC202000908DF804408DF82E
:1076A000065003208DF805008DF8074069463046E6
:1076B000F2F734FC7CBD000000040240F0B589B054
:1076C0000025FFF7C7FFFFF76BFF4FF4E13000F035
:1076D0000FF900F0EFF80121402000F0FBFA012043
:1076E00000F07CFB4FF47A77384604F08FFC5E4C58
:1076F0000B2084F82C01002684F828612676A676D3
:107700006676E676276284F82860012384F82A30BA
:1077100084F8293084F82B30F80020632670A37099
:107720006370E370A7602673A3736373E373001140
:1077300060614E490E708E704B70CB704EF66027B4
:107740008F604B4A42F6F82CA1F27441A4F27C649B
:1077500005EB450002EB8000A0F5156000F5005038
:10776000067086704370C670C0F808C06D1C042D8A
:10777000EED394F8A307000706D094F8A30700F00F
:107780000F00401E84F8A50794F8A307000906D04F
:1077900094F8A307FF2303EB101084F8A60784F8DE
:1077A000AA6794F8A60768B1324B01280DD00228C9
:1077B00008D0032811D147F23050C1F87C04C3F837
:1077C00088620AE0C1F87C7407E0C1F87C74C3F8F1
:1077D000886243F69820C4F8840627482749006841
:1077E00008602548001D006848602348083000688C
:1077F00088600020131803F5805383F82B67401C22
:107800001428F7D3087A04AFCD7A8B7A4A7A87E8BE
:107810002D000879CD798B794A798DE82D001248B1
:107820008B780A7816A1AF3003F002F8002103200C
:10783000F1F794FF10B11D48C0F8886294F8A517BD
:107840001B4800294FF0200104D009B0BDE8F040EA
:10785000F2F7B7BBF2F7B7FB94F8E20640F080000E
:1078600084F8E20609B0F0BD202900201857002056
:10787000A412002000004042107AFF1F047C002068
:1078800025303278253032782530327825303278FC
:1078900025303278253032782530327825303278EC
:1078A0002530327825303278250000000000424231
:1078B0000004024038B546208DF8000002208DF803
:1078C000010001248DF802408DF803406846FBF763
:1078D00073FE25208DF800008DF8014000208DF802
:1078E00002008DF803406846FBF766FE38BD0000D5
:1078F0001FB504460121102000F010FA0020ADF859
:1079000004000094ADF80600ADF80800ADF80C00D6
:107910000C200D4CADF80A006946204602F020FF0D
:107920000121204602F085FE012240F2244120463A
:1079300002F0FEFE1021204602F078FE0122C02156
:10794000204602F080FE1FBD001001402DE9FC47DB
:107950000121592000F0A6F943F6F8700024DFF861
:10796000A0A000908DF8044002268DF807606946BB
:107970005046F2F7D3FAFC20DFF8889000908DF89B
:10798000044001258DF8075069464846F2F7C6FACB
:10799000DFF874804FF440478DF8044000978DF86D
:1079A000075069464046F2F7B9FA8DF804408DF861
:1079B00007600720154E009069463046F2F7AEFA90
:1079C00007213046F2F7FDFA39464046F2F7FBFA56
:1079D0004FF47C515046F2F7F6FAF8215046F2F790
:1079E000F0FAFC214846F2F7EEFA0948D0F82812DE
:1079F0000848012902D00470BDE8FC870570FBE748
:107A00000010024000180240000C0240000002403A
:107A100000004242A412002070B5FFF797FF6420D7
:107A200004F0F4FA2048D0F83C3201221F492048E3
:107A30000024E3B180F8A547D1F814021D4978B3BA
:107A40000C761D48D0F81C22D0F81832120142EAF8
:107A5000C302D0F8143242EA8302D0F81032D0F8D0
:107A60000C0242EA4302024318324A7070BDD1F858
:107A700018328BB180F8A527D1F80832D1F80C5212
:107A800043EA4503DB4380F8A63790F8A63703F0B6
:107A9000030380F8A637CFE7022380F8A537EBE78A
:107AA000FFE70A76CDE70000008041420000434234
:107AB000A4220020A4120020000042422DE9FC4133
:107AC0000121112000F0EEF801248DF8044000257A
:107AD0004CF204008DF806500326184F00908DF8E4
:107AE00005608DF8074069463846F2F717FA042119
:107AF0003846F2F766FA124890F8A617032903D021
:107B000090F8A607012812D18DF804408DF8065090
:107B100004200C4D00908DF805608DF807406946F3
:107B20002846F2F7FBF904212846F2F74AFA0648FC
:107B3000C0F8B842C0F8BC42BDE8FC810010024069
:107B4000A42200200000024000004242FFF7B6BF1E
:107B50002DE9FE4316200A9D16461F468DF80000AB
:107B60004B4800EB4114202109E09DF8000020441F
:107B700080F85B1F9DF80000401C8DF800009DF808
:107B800000002028F1D34FF0000840460BE09DF89C
:107B90000000394682003046F0F745FB084308D024
:107BA0009DF80000401C8DF800009DF80000102892
:107BB000EDD39DF80000A84216D8FDB19DF8000055
:107BC00020B99DF8000028448DF800009DF80000C1
:107BD000401C8DF800009DF800103020C1F11E01FE
:107BE000214481F85B0F00E045B101208DF80400CD
:107BF000C5F11E0121442E2081F85B0F404614E0A0
:107C00009DF80800394682003046F0F70CFB00F082
:107C10000F009DF808103030C1F11E01214481F899
:107C20005B0F9DF8080000F101008DF808009DF839
:107C30000800A842E4D39DF8040028441BE09DF806
:107C400008009DF80410401A820030463946F0F7CB
:107C5000EAFA00F00F009DF8081030309DF804207B
:107C6000A1EB0201C1F11E01214481F85A0F9DF8D8
:107C7000080000F101008DF808009DF800009DF853
:107C8000041008449DF808108842D8D8BDE8FE8347
:107C9000A41200204FF400610148F2F78BB90000F4
:107CA00000040240044A0029116801D0014300E0A9
:107CB000814311607047000030380240044A0029B7
:107CC000116801D0014300E081431160704700005A
:107CD00010380240044A0029116801D0014300E035
:107CE000814311607047000034380240044A002983
:107CF000116801D0014300E081431160704700002A
:107D000040380240044A0029116801D0014300E0D4
:107D1000814311607047000020380240044A002966
:107D2000116801D0014300E08143116070470000F9
:107D300044380240044A0029116801D0014300E0A0
:107D400081431160704700002438024070B5204B19
:107D50001968204C11F00C0104D06610042903D0DE
:107D6000082903D004601BE0066019E0184A121FBE
:107D70001168C1F38055116801F03F0115B1B6FBE0
:107D8000F1F101E0B4FBF1F114681268C4F3881456
:107D90006143C2F30142521C5200B1FBF2F1016097
:107DA00019680F2202EA11110B4A545C0168E14084
:107DB00041601C68072505EA9424145D21FA04F447
:107DC00084601B6805EA5333D25CD140C16070BD4A
:107DD000083802400024F400000000200549002873
:107DE000086802D040F0040001E020F004000860C0
:107DF0007047000000080650014800687047000006
:107E00000808065070B5012080F310880C4D102131
:107E10002846F2F7D6F808212846F2F7D4F8D720FA
:107E2000F0F74AFFFF20F0F747FF044610212846ED
:107E3000F2F7C9F8002181F31088204670BD0000D8
:107E40000000024070B5012080F31088194C00201A
:107E5000A080FFF7D7FF000609D4012004F0D6F870
:107E6000A088401C80B2A080C828F2D31EE0A08861
:107E7000C8281BD2104D10212846F2F7A2F808217D
:107E80002846F2F7A0F89F20F0F716FFFF20F0F742
:107E900013FFFF20F0F710FF607010212846F2F763
:107EA00092F8002080F31088607870BD002080F385
:107EB000108870BD220A00200000024070B5012128
:107EC00088B08803FFF712FF01210220FFF7EAFEC6
:107ED00000244FF400602F4E8DF8044000908DF880
:107EE000074069463046F2F719F801218DF8041071
:107EF00002258DF8055008038DF806408DF807100F
:107F0000009069463046F2F709F805220D21304607
:107F1000F2F740F805220E213046F2F73BF8052231
:107F20000F213046F2F736F84FF4604000908DF89C
:107F3000045003208DF805008DF806408DF80740A9
:107F400069463046F1F7EAFF134D284600F04AF83B
:107F5000ADF810406815ADF812001820ADF8140007
:107F60000720ADF81800ADF808404FF48270ADF866
:107F70000C40ADF80A00ADF80E40ADF8164002A96D
:107F8000284600F064F80121284600F021F808B0E6
:107F900070BD0000000402400038004070B50B4C7A
:107FA00005460221204600F047F80028F9D029466E
:107FB000204600F04AF80121204600F03DF8002854
:107FC000F9D0204600F03FF8C0B270BD0038004044
:107FD0000029018802D041F0400101E021F0400178
:107FE00001807047114910B588420AD184140121DB
:107FF0002046FFF79FFE2046BDE810400021FFF716
:1080000099BE0B49884202D10121041404E00949B8
:1080100088420AD10121C4132046FFF773FE20468F
:10802000BDE810400021FFF76DBE10BD00300140DB
:1080300000380040003C00400246002012890A42FD
:1080400000D001207047808970478181704730B52A
:1080500002884C8802F441530A88CD8822438C88D8
:108060002C4322430C8922434C8922438C8922438E
:10807000CC8922431A430280828B22F400628283DD
:10808000098A018230BD0246002003E012F8013B5C
:108090001844C0B2491E89B2F8D270472DE9F041A8
:1080A00001218D070024284601F000FFF0B3F1F70D
:1080B0009DFF284E002006F580533DE006EB84012D
:1080C00001F58051D1F8F8271278012AD1F8F82764
:1080D00003D05278012A08D02CE01070D1F8F8278C
:1080E0005070D1F8F827907030E0D1F8F8279278E6
:1080F00002BBD1F8F82757687F1C5760D1F8F827E2
:108100005268D1F8F877BF68BA4213D3D1F8F8773C
:108110000122BA70D1F8F827D278012A16D0D1F806
:10812000F8275070D1F8F827506000E008E0D1F847
:10813000F817C870641CE4B293F8F617A142BDD8D2
:108140002846BDE8F041012101F0FABDD1F8F81749
:108150004860EFE7A41200200CB5002225490092E8
:108160000192086840F4803008604FF4A06308680A
:1081700000F4003001900098401C0090019810B964
:1081800000989842F3D10868800330D5012001900F
:1081900018484030026842F0805202601648026877
:1081A00042F48042026013480830026802600268AC
:1081B000026002680260031F104A1A600A6842F0F7
:1081C00080720A600A689201FCD50D4A40F205618E
:1081D0001160016821F003010160016841F00201B2
:1081E00001600168C1F381010229FAD10CBD01923D
:1081F0000CBD0000003802400070004008544007E9
:10820000003C02407CB500229FED170A00928DEDE4
:10821000010A6D4601AC16E0835CA3F13006102E16
:1082200005D2009B1B010093865C303E07E0413B7A
:10823000062B0CD2009B1B010093865C373E1E432D
:10824000521CD2B200968A42E6D3002006E0BFEE6E
:10825000000A7CBD2A5C2254401CC0B2B0EB510F16
:10826000F8D39DED010A7CBD0000000030B5054645
:108270000022104611E0AB5CA3F13004102C02D2B6
:1082800044EA001007E0A3F14104062C08D20401DF
:10829000A3F137002043521CD2B28A42EBD330BD47
:1082A0004FF0FF3030BD00002DE9FE43534C4FF03E
:1082B0003809A07800263146F9F732FC0125082755
:1082C0000096CDE901750246182000234946FBF7C8
:1082D000C3FB00F1040808EB48004006000E082329
:1082E0002D2249460095FBF749FB607808F101080B
:1082F0000021F9F715FC0246009608EB4800CDE98D
:1083000001754006000E00234946FBF7A5FB80449B
:1083100008EB48004006000E08232D224946009530
:10832000FBF72CFB207808F101080021F9F7F8FB96
:108330000246009608EB4800CDE901754006000EA4
:1083400000234946FBF788FB804408EB48004006C1
:10835000000E0823202249460095FBF70FFB6079A9
:1083600008F101080021F9F7DBFB0246009608EB53
:108370004800CDE901754006000E00234946FBF791
:108380006BFB804408EB48004006000E08232D22BA
:1083900049460095FBF7F2FA207908F1010800211F
:1083A000F9F7BEFB0246009608EB4800CDE90175DF
:1083B0004006000E00234946FBF74EFB804408EBC5
:1083C00048004006000E08232D2249460095FBF781
:1083D000D5FAE07808F101080021F9F7A1FB02467F
:1083E000009608EB4800CDE901754006000E002319
:1083F0004946FBF731FBBDE8FE8300008D260020D7
:10840000024908710120C87170470000A4120020C1
:108410002DE9F04F002587B02F46F1F7D1FBF74E3D
:10842000F07900287ED0A94686F80790FBF700F97E
:1084300030794FF0080A4FF001084FF0100B06F5A5
:108440008054102881F00E84DFE810F010008D00B9
:10845000F9007F02FF0343044505FD06EB075608BC
:10846000AB086709060A4B0AEB0AE50BF1F7AEFD0C
:1084700001280AD0022808D0042806D0082804D1F0
:108480000220FFF7BDFF84F8E091CDE900B800219C
:1084900045461523DAA20846FBF7ABFB94F8E10149
:1084A00028B3CDE900A557460523DAA21421002000
:1084B000FBF79FFBCDF80090CDE9017594F8E12121
:1084C000002314211E20FBF7C7FACDE9007594F8AC
:1084D000E1010A2300EB400101EB001006EB001163
:1084E00041F632400A1814212820FBF782FB94F849
:1084F000E001FF2829D094F8E001CDE900050A2326
:1085000064221E211846FBF7B7F9CDF80090CDE99B
:1085100001A594F8E0214E4600232D213220FBF7DF
:108520009BFA00E0F5E300EB4000322101EB400054
:10853000C0B2082325222D210095FBF71FFA94F8DD
:10854000E001642809D001F08DBBCDE900A5152319
:108550002D21B2A2142001F061BA84F8E06102205A
:10856000FFF74EFFEFE7F1F731FD01280BD00228AE
:1085700009D0042802D0082805D101E0092000E034
:108580000420FFF73DFF94F8A40738B194F8A5073D
:1085900038B1012808D0022811D108E01523A3A280
:1085A00007E01523A4A204E01523A7A201E01523E8
:1085B000A8A2CDE900A800210846FBF71AFBF07835
:1085C000012802D002280CD101E0A64901E0A5490A
:1085D0001231CDE9001809231A460A210020FBF7C1
:1085E000BBFAA04818234838CDE9000844461A468B
:1085F00000216820FBF7B0FACDE900A45546152309
:1086000099A21A210020FBF7F4FACDE900541523B2
:108610009BA224210020FBF7ECFACDF80090CDE9D5
:108620000154B26D002324215420FBF715FAB06DDC
:1086300010B90220FFF7E4FEFFF736FE83E7F1F7FB
:10864000C5FC012806D002280ED0042814D0082822
:108650001BD125E00320FFF7D3FE94F8DC0120F0C6
:10866000800084F8DC0110E094F8DC0120F0800048
:1086700084F8DC01032006E094F8DC0120F080009F
:1086800084F8DC010920FFF7BBFE94F8A40778B159
:1086900094F8A507A8B1012816D002281CD120E023
:1086A00094F8DC0120F0800084F8DC010420EAE783
:1086B000CDE900A80021152375A20846FBF799FA19
:1086C00015E015235CA201E015235FA2CDE900A807
:1086D00000210846FBF78DFA94F867060F2803D0AF
:1086E00005E015235BA2F1E70120FFF789FEF07892
:1086F000012802D0022811D106E05A49CDE900181C
:1087000009231A460A2106E0564809231230CDE90A
:1087100000081A460A210020FBF71EFA94F8E0012F
:1087200010B10020FFF76CFE94F8A50758B394F839
:10873000A6674C4A5C32A2F12A00A2F10E05A2F112
:108740001C03A0F10E01022E07D094F8A667012E9B
:108750003FD094F8A667E6B315E04F4ED6F8006216
:10876000C6B394F8AA17322947D394F8AA173C291C
:108770003ED2CDE9005808230E220021592000E006
:108780005920FBF7E9F9374818234838CDE90008A4
:1087900045461A4600216820FBF7DEF9CDE900B511
:1087A0005F4610233DA214212820FBF722FACDE9D1
:1087B00000A5564615233BA224211220FBF719FAE7
:1087C00094F8DC0100060AD510232E213AA20020DD
:1087D00001E087E080E0CDE90075FBF70AFAFFF7DA
:1087E00063FD94F8E206000672D594F8A827A1E08C
:1087F00094F8AA1746296CD392E07CE0A4120020DA
:108800004669726D77617265446F776E6C6F6164F3
:1088100000000000506F72743A000000446F776EE1
:108820006C6F6164204661696C2100004E6F2053BB
:1088300069676E616C000000547970653A53746129
:1088400074696F6E00000000547970653A436C6F74
:1088500075640000547970653A436C6F75642D54EB
:1088600065737400D4EB01084F66666C696E652011
:108870005265636F72642055706C6F616400000014
:108880005265636F7264206E756D6265723A0000A6
:108890004F66666C696E650000004042424C55456B
:1088A000534B5900454E4552475920544543484E75
:1088B0004F4C4F4759000000557067726164652046
:1088C00045525220436865636B2047756E00000077
:1088D0002CE01DE00E2203E0CDE9001808230E2253
:1088E00000214DE794F8AA67202EBFF435AF94F825
:1088F000AA671A2E03D9CDE900280823EAE794F8DD
:10890000AA27172A3FF635AF94F8AA27142A03D9C5
:10891000CDE900380823DDE794F8AA27122ADBD92D
:10892000CDE9000808230E22002129E794F8E20689
:10893000C0F3C302F7A103A801F07AFF022303AA40
:10894000CDE900653821002005E6F1F73FFB01285D
:1089500006D002281CD0042835D008283ED138E0A3
:108960003F210FE0707918B17079401E707100E0FE
:108970007171707900EB8002C2EB8010304490F886
:108980006000F8B970796D1CADB2402D26D8E9E7CA
:10899000494614E06D1CADB2402D1FD870793F28B8
:1089A00003D27079401C707100E07171707900EB36
:1089B0008002C2EB8010304490F8600010B97079EA
:1089C0004028E7D30AE0707984F8DB0C84F8DC8C6B
:1089D00004E00220FFF714FD86F805903079344654
:1089E00003287DD160790122010906910021CB483D
:1089F00001F044F9CDF80090CDE901B86079454621
:108A00005F464E4600EB8001C1EB8010204490F899
:108A10006020002319465820FBF71EF8CDE90075A9
:108A20001023BFA219460020FBF7E3F8607900EBA2
:108A30008001C1EB80102044D0F861000021F9F7DB
:108A40006FF80699024601EB410000EB011004EBC0
:108A5000001101F58051884691F8700D002300F057
:108A60000300CDE90007102102951820FAF7F4FF62
:108A7000CDE900751023AFA220210020FBF7B9F843
:108A8000607900EB8001C1EB80102044D0F86500D4
:108A90000021F9F745F8024698F8700D0023C0F35D
:108AA0008100CDE90007202102951820FAF7D4FFB4
:108AB000607900EB8001C1EB8010204490F88300C6
:108AC0000021F9F72DF80096CDE901A50246574699
:108AD000382118200023FAF7BFFF00F1040800E056
:108AE00092E208EB480040063821000E08232D22B0
:108AF0000095FAF743FF607908F1010800EB800167
:108B0000C1EB8010204490F882000021F9F708F8AA
:108B10000246009608EB4800CDE901754006382171
:108B2000000E0023FAF798FF804408EB4800400647
:108B30003821000E08232D220095FAF71FFF6079D7
:108B400008F1010800EB8001C1EB8010204490F88F
:108B500081000021F8F7E4FF0246009608EB480088
:108B6000CDE9017540063821000E0023FAF774FFA5
:108B7000804408EB480040063821000E08232022DC
:108B80000095FAF7FBFE607908F1010800EB80011F
:108B9000C1EB8010204490F886000021F8F7C0FF58
:108BA0000246009608EB4800CDE9017540063821E1
:108BB000000E0023FAF750FF804408EB48004006FF
:108BC0003821000E08232D220095FAF7D7FE607990
:108BD00008F1010800EB8001C1EB8010204490F8FF
:108BE00085000021F8F79CFF0246009608EB48003C
:108BF000CDE9017540063821000E0023FAF72CFF5D
:108C0000804408EB480040063821000E08232D223E
:108C10000095FAF7B3FE607908F1010800EB8001D6
:108C2000C1EB8010204490F884000021F8F778FF11
:108C30000246009608EB4800CDE901754006382150
:108C4000000E0023FAF708FF7DE4F1F7BFF90128D1
:108C500006D0022809D004280ED008281ED121E011
:108C60007079D8B17079401E04E07079032815D26C
:108C70007079401C707111E0707930B1012806D014
:108C8000022806D0032809D105E0052004E00620CB
:108C900002E0072000E00820FFF7B2FB307904284B
:108CA00005D050E40220FFF7ABFB4846E2E71B4843
:108CB00004220021803800F0E1FFCDE900B970798D
:108CC0001649803901EB001270790007010E10235C
:108CD000FEE3F1F77BF9082802D10420FFF790FBAF
:108CE00030790528B0D10D4804220021403800F029
:108CF000C5FF94F8A50720B1012825D002283DD151
:108D000058E01023AFF2D042CDE900A81946002068
:108D100032E0F0E32530327800000000BEEC0108BC
:108D20004C3A2020202020202020202020202020FD
:108D300000000000503A2020202020202020202069
:108D4000202020200000000047461023AFF20852E8
:108D5000CDE900A819460020FAF74BFFCDE900A79E
:108D60001023FDA238210020FAF743FFCDE900A728
:108D70001123FB4A38211E20FAF73BFF94F8A50780
:108D800000288ED094F8A617F64841F23F72871853
:108D900041F22B7200EB020921B394F8A6070128D7
:108DA0005AD094F8A607022871D094F8A607032891
:108DB0007DD043E4CDE900A810235746EAA2194626
:108DC0000020FAF716FFCDE900781023E2A238213F
:108DD0000020FAF70EFFCDE9007811233821E64A8A
:108DE0001E20C9E7701900F5805090F8E40618B904
:108DF0006D1CADB2152DF5D3CDE900A844465546FE
:108E00001023DEA21A210020FAF7F3FECDE9005468
:108E100010233A461A212420FAF7EBFE707818281E
:108E20000AD9CDE900541023D6A224210020FAF754
:108E3000E0FE14234A460AE0CDE900541023D1A2F3
:108E400024210020FAF7D5FEC54A14232A322E2108
:108E5000CDE90054002077E5701900F5805090F8B6
:108E6000E40618B96D1CADB2152DF5D3CDE900A8F7
:108E7000444655461023C1A21A210020FAF7B9FE34
:108E800010231A213A46242020E000E00FE0CDE92B
:108E900000A8444655461023BCA21A210020FAF728
:108EA000A8FEAF4A102361321A211E200EE0CDE940
:108EB00000A8444655461023B6A21A210020FAF70E
:108EC00098FEA74A1023A6321A211220CDE9005499
:108ED000FAF78FFEA5E7F1F779F8012804D0022808
:108EE00007D008280FD10BE0707960B17079401E6F
:108EF00004E07079032806D27079401C707102E09A
:108F00000420FFF77DFA307906287DD10422002164
:108F1000A14800F0B3FE4FF00009CDF80090CDE974
:108F200001B844467279B346B046012349463E2013
:108F3000521CFAF791FDCDE900A45646102397A2E2
:108F400000214820FAF755FEDFF85CA2CDE900A425
:108F500008231A4600217820FAF7FEFDCDE90064C7
:108F6000102392A208214820FAF743FE0823CDE9F6
:108F700000A91A4619467820FAF7EEFDCDE90064FB
:108F800010238DA219460020FAF733FE98F8050049
:108F900000EB400101EB001108EB011000F58050DF
:108FA00090F8610D4FF01003012844D084A2CDE960
:108FB000006410211E20FAF71CFECDE90064A046D3
:108FC000102381A218210020FAF713FE9BF8050058
:108FD00000EB400101EB00100BEB001000F580509E
:108FE00090F85A0DCDE9006805289BF8050000EBC4
:108FF000400101EB00100BEB001000F580501CD07D
:1090000090F85A0D644900E00AE2403101EB001289
:109010000C2318213620FAF7ECFD0120CDE9006081
:10902000B04610236BA220210020FAF7E2FD0926AA
:109030004FF0200BF7E06AA2B9E790F8600D5649AF
:10904000C031E3E706EB46014FF07A09B9EB410F77
:1090500002D27F1CBFB20026607900EB400101EB19
:10906000001004EB001000EB051000F5805090F8A4
:10907000860D4FF0000AC009CDF800A0CDE90180AF
:10908000607900EB400101EB001004EB001000EBF5
:10909000051000F5805090F8842D0BEBC700C1B28D
:1090A00006EB46004006000E5346FAF7D5FC304466
:1090B00086B206EB4601B9EB410F02D27F1CBFB26C
:1090C0000026607900EB400101EB001004EB00107A
:1090D00000EB051000F5805090F8860D0823C009BC
:1090E00000900BEBC700C1B206EB46004006000E35
:1090F0002D22FAF743FC761CB6B206EB4601B9EB1B
:10910000410F02D27F1CBFB20026607900EB400104
:1091100001EB001004EB001000EB051000F580508F
:1091200090F8860DCDF800A0C009CDE901806079E6
:1091300000EB400101EB001004EB001000EB051008
:1091400000F5805090F8852D0BEBC700C1B206EBFF
:1091500046005C46400647E055524C3A000000008D
:10916000AA290020A4120020547970653A436C6F3C
:1091700075642D546173740058CB010841504E2022
:109180003A000000494D45493A0000005353494414
:109190003A00000049503A00FEEC01084F6E4C695D
:1091A0006E65203A2000000084EB01084F66664C93
:1091B000696E653A20000000547970653A0000003D
:1091C000525334383500000050726F746F636F6C07
:1091D0003A00000047756E2D416464723A00000049
:1091E0004C4F524100000000000E0023FAF734FCFF
:1091F000304486B206EB4601B9EB410F02D27F1C28
:10920000BFB200260120009004EBC700C1B206EBFC
:1092100046004006000E08233B22FAF7AFFB761CFF
:109220006D1CB6B2ADB2F74C607900EB400101EBBA
:10923000001004EB001000F5805090F85B0DA84280
:109240003FF600AFECE0F0F7C1FE012804D00228A1
:1092500007D008280FD10BE0707960B17079401EFB
:1092600004E07079032806D27079401C707102E026
:109270000420FFF7C5F830790728E3D10124F47101
:1092800004220021E04800F0F9FC0020CDE9000BA9
:1092900002947279014601234020521CFAF7DCFB4C
:1092A0000820CDE900041023D8A214210020FAF7E9
:1092B000A0FC0924A5E004EB44014FF07A09B9EBC6
:1092C000410F02D27F1CBFB200244FF0000A4FF0C2
:1092D00001080821CDF800A0CDE90118707900EB54
:1092E000400101EB001006EB001000EB051000F54B
:1092F000805090F8842D4FF0140B0BEBC700C1B2D7
:1093000004EB44004006000E5346FAF7A5FB204448
:1093100084B204EB44017A20B0EB410F02D27F1CEF
:10932000BFB200240BEBC700C1B204EB44004006FF
:10933000C146000E08232D22CDF80080FAF71EFB4F
:10934000641CA4B204EB44014FF07A08B8EB410F5F
:1093500002D27F1CBFB200240821CDF800A0CDE9C5
:109360000119707900EB001101EB002006EBC00041
:1093700005EB051100EBC10000F5005090F8580214
:10938000642110FB01F0020A0BEBC700C1B204EB31
:10939000440040065E46000E0023FAF75DFB2044C1
:1093A00084B204EB4401B8EB410F02D27F1CBFB280
:1093B000002406EBC700C1B204EB44004006000ED7
:1093C00008232522CDF80090FAF7D8FA641CA4B23D
:1093D00004EB4401B8EB410F02D27F1CBFB2002462
:1093E00006EBC700C1B204EB44004006000E0823A0
:1093F0003B22CDF80090FAF7C1FA641C6D1CA4B2B0
:10940000ADB2804E707900EB400101EB001006EB2D
:10941000001000F5805090F85B0DA8423FF64BAF6E
:1094200019E2F0F7D3FD082802D10420FEF7E8FF87
:1094300030790828F4D1744804220021403000F02B
:109440001DFCCDE900A847465446102372A2142102
:109450000020FAF7CEFBCDE9004710236F4A142114
:109460001220FAF7C6FBCDE9004710236CA21421A5
:109470005A20FAF7BEFBCDF80090CDE9014772788B
:10948000022314216C20FAF7E7FAB24605EB4500F7
:1094900000EB05110AEB011841F66C5010F80800BA
:1094A000C00723D005EB8501142000EB4106CDE970
:1094B0000047F1B205235BA20020FAF79AFBCDF832
:1094C0000090CDE9014701236A1CF1B21E2000E0A3
:1094D00065E0FAF7C1FA41F66251CDE9004708EBC1
:1094E0000102F1B20A232A20FAF783FB6D1CADB208
:1094F000042DCBD3B6E3B7E3F0F768FD012806D01F
:1095000002280BD0042811D0082830D133E070791C
:1095100010B17079401E25E0052023E07079052800
:1095200002D27079401C1DE048461BE07079062885
:109530001DD2DFE800F00305070911190A2014E025
:109540000B2012E00C2010E00D20FEF759FF94F8DC
:10955000A30700F00F0005E00E20FEF751FF94F87E
:10956000A3070009707102E00F20FEF749FF307970
:10957000092804D076E30220FEF742FFD4E7707991
:10958000214C0422803404EB0010002100F076FB13
:10959000CDE900B97079102304EB001200210020FE
:1095A0003CE2F0F713FD012806D0022809D0042878
:1095B0000ED0082864D167E0707910B37079401E2E
:1095C00004E0707903285BD27079401C707157E019
:1095D000707900EB400101EB001006EB001000F584
:1095E000805090F8610D012820D0707900EB400187
:1095F00001EB001006EB001000F5805090F8610DB3
:1096000040B33DE0A4120020EEED010847756E2D39
:10961000525353493A00000053563A005CC40108C3
:1096200048563A00506F72742D00000070794C4615
:1096300000EB400101EB001006EB001000F580503C
:1096400080F8619D71790220F0F788F8FC48C0F835
:10965000884215E07079444600EB400101EB0010B0
:1096600006EB001000F5805080F8618D7079F8F7F6
:1096700029FFF348C0F8884271790220F0F76EF8AC
:1096800030790A2805D0EDE20920FEF7B9FE4846F8
:109690009CE704220021EB4800F0F0FACDE900A895
:1096A000444655461523E8A214212820FAF7A1FACA
:1096B000CDF80090CDE901547279012314214620A0
:1096C000521CFAF7C9F9707900EB400101EB001068
:1096D00006EB001000F5805090F8610D01280CD0C9
:1096E000707900EB400101EB001006EB001000F573
:1096F000805090F8610D18B10AE01523D4A201E062
:109700001523D6A2CDE900541E210020FAF771FAE4
:109710001523D5A23221FFF79BBBF0F757FCD74C9E
:10972000012806D002280FD004281AD0082830D1EA
:109730001CE0707968B394F88D0410B17079F8F773
:10974000C1FE7079401E0AE07079032821D294F896
:109750008D0410B17079F8F7B5FE7079401C707106
:1097600017E084F88D8484F8818412E00920FEF7E4
:1097700047FE484686F8059084F8808494F88D1456
:1097800039B1AF49C1F8880284F88D047079F8F7CF
:1097900099FE30790B2832D1AA48042200214030AA
:1097A00000F06CFACDE900A8454657461523A6A25D
:1097B00012212820FAF71DFACDF80090CDE90175A5
:1097C0007279012312214620521CFAF745F9CDE99E
:1097D00000751523AAA21C210020FAF70AFACDE988
:1097E00000751523ACA226210020FAF702FACDE974
:1097F00000751523AEA230210020FAF7FAF994F88B
:109800008D04012827D1454686F8078094F8820404
:1098100080B18B49C1F8889284F8829470790121D3
:10982000F8F78CFFCDE900A51523A6A2382100206A
:10983000FAF7DFF994F88C0400280CD084F88C94A3
:10984000CDE900A51523A3A238210020FAF7D1F90C
:109850007B48C0F8885205E2F0F7B8FB012813D026
:10986000022811D0042802D008280DD109E0EFF712
:109870009FFB142803D0484684F8E80304E04046E0
:10988000FAE70920FEF7BCFD30790C287ED16D483F
:1098900004220021803000F0F1F9CDE900A845460E
:1098A000564615238FA21A210020FAF7A2F9CDE916
:1098B0000065152390A224210020FAF79AF9CDE93A
:1098C0000065152390A22E210020FAF792F994F852
:1098D000E8034FF0150310B191A2FFF731B896A23B
:1098E000FBE7F0F773FB012806D002280BD0042811
:1098F00012D0082857D165E0707910B17079401EF8
:1099000008E0032006E07079032802D27079401C39
:1099100000E04846707146E0717994F8A30761F35E
:10992000030084F8A30700210320EFF717FF70B3AB
:1099300094F8A357022004F5EE74FEF761FDEFF7EB
:1099400063FF84F8C75500210320EFF707FF207855
:1099500020F001002070207840F006002070A4F86C
:10996000029000210120EFF7F9FE94F8060520F09F
:10997000800084F8060594F8CA05A4F5EE74B0B129
:10998000012819D0022805D0032801E06AE10AE085
:1099900007D10CE094F8E20620F07800203084F83B
:1099A000E206FDF78BFE30790D280FD05AE194F8CE
:1099B000E20620F07800F2E794F8E20620F0780062
:1099C0005830ECE70920FEF71BFDA2E71D480422F2
:1099D0000021C03000F052F9CDE900B894F8A30797
:1099E0005D46584F00F00F0007EB00121023194698
:1099F0000020FAF7FEF894F8A307717900F00F0041
:109A0000884202D0CDE9005901E0CDE900587079D3
:109A10000C2307EB001220210020121DFAF7E9F8B1
:109A200020E1F0F7D3FA012806D0022805D0042857
:109A300004D0082803D1CBE086E08CE094E0CBE0B2
:109A400000004242FEEE0108504F52543A0000001E
:109A5000545950453A4C4F5241000000545950451A
:109A60003A525334383500005061737320456E7498
:109A70006572204368616E6765000000A452002093
:109A8000313A446970207377697463682031616E7C
:109A90006432204F4E000000323A496E7365727492
:109AA00020736C617665206D6F64756C65000000D5
:109AB000333A5061737320456E746572205374613C
:109AC0007274000053746174653A53656E64696E14
:109AD0006700000053746174653A436F6D706C6584
:109AE00074650000496E7365727420552D44697366
:109AF0006B204669727374005468616E2050617304
:109B00007320456E74657200466F726D61743A46DB
:109B1000415433323B4D41583A3332470000000044
:109B200046696E6420552D4469736B2C4F757470B3
:109B30007574696E6700000053746174653A496416
:109B40006C6500003EF00108707910B17079401E1C
:109B500008E0042006E07079042802D27079401CE5
:109B600000E04846707137E0717994F8A30761F31B
:109B7000071084F8A30700210320EFF7EFFD58B387
:109B80000220FEF73DFC94F8E20620F0800084F805
:109B9000E20694F8A60780B1012813D0022802D06B
:109BA000032807D109E094F8E20620F0780020307D
:109BB00084F8E206FDF782FDD3E794F8E20620F090
:109BC0007800F5E794F8E20620F078005830EFE7E7
:109BD0000920FEF715FCC4E730790E2842D1042293
:109BE0000021234800F04AF8CDE900B894F8A30713
:109BF0005D461F4F20F00F008037C2191023194611
